:10000000F0EF0020F5CC0000972C0000432E0000FC
:10001000672E0000176E0000BF6E0000E5D00000E4
:10002000E5D00000E5D00000E5D00000276F00001B
:100030000F830000E5D000006B830000277A0000EA
:10004000E5D00000E5D00000E5D00000E5D00000DC
:10005000E5D00000E5D00000E5D00000E5D00000CC
:10006000E5D00000E5D00000E5D00000E5D00000BC
:10007000E5D00000E5D00000E5D00000E5D00000AC
:10008000E5D00000E5D00000E5D00000E5D000009C
:10009000E5D00000E5D00000E5D00000E5D000008C
:1000A000E5D00000E5D00000E5D00000E5D000007C
:1000B000C98E0000E5D00000E5D00000E5D00000CA
:1000C000E5D00000E5D00000E5D00000E5D000005C
:1000D000E5D00000E5D00000E5D00000E5D000004C
:1000E000E5D00000E5D00000E5D00000E5D000003C
:1000F000E5D00000E5D00000E5D00000E5D000002C
:10010000E5D00000E5D00000E5D00000E5D000001B
:10011000E5D00000E5D00000E5D00000E5D000000B
:10012000E5D00000E5D00000E5D00000E5D00000FB
:10013000E5D00000E5D00000E5D00000E5D00000EB
:10014000E5D00000E5D00000E5D00000E5D00000DB
:10015000E5D00000E5D00000E5D00000E5D00000CB
:10016000E5D00000E5D00000E5D00000E5D00000BB
:10017000E5D00000E5D00000E5D00000E5D00000AB
:10018000E5D00000E5D00000E5D00000E5D000009B
:10019000E5D00000E5D00000E5D00000E5D000008B
:1001A000E5D00000E5D00000E5D00000E5D000007B
:1001B000E5D00000E5D00000E5D00000E5D000006B
:1001C000E5D00000E5D00000E5D00000E5D000005B
:1001D000E5D00000E5D00000E5D00000E5D000004B
:1001E000E5D00000E5D00000E5D00000E5D000003B
:1001F000E5D00000E5D00000E5D000004F7A000017
:10020000E5D00000E5D00000E5D00000E5D000001A
:10021000E5D00000E5D00000E5D00000E5D000000A
:10022000E5D00000E5D00000E5D00000E5D00000FA
:10023000E5D00000E5D00000E5D00000E5D00000EA
:10024000E5D00000E5D00000E5D00000E5D00000DA
:10025000E5D00000E5D00000E5D00000E5D00000CA
:10026000E5D00000E5D00000E5D00000E5D00000BA
:10027000E5D00000E5D00000E5D00000E5D00000AA
:10028000E5D00000E5D00000E5D00000E5D000009A
:10029000E5D00000E5D00000E5D00000E5D000008A
:1002A000E5D00000E5D00000E5D00000E5D000007A
:1002B000E5D00000E5D00000E5D00000E5D000006A
:1002C000E5D00000E5D00000E5D00000E5D000005A
:1002D000E5D00000E5D00000E5D00000E5D000004A
:1002E000E5D00000E5D00000E5D00000E5D000003A
:1002F000E5D00000E5D00000E5D00000E5D000002A
:10030000E5D00000E5D00000E5D00000E5D0000019
:10031000E5D00000E5D00000E5D00000E5D0000009
:10032000E5D00000E5D00000E5D00000E5D00000F9
:10033000E5D00000E5D00000E5D00000E5D00000E9
:10034000E5D00000E5D00000E5D00000E5D00000D9
:10035000E5D00000E5D00000E5D00000E5D00000C9
:10036000E5D00000E5D00000E5D00000E5D00000B9
:10037000E5D00000E5D00000E5D00000E5D00000A9
:10038000E5D00000E5D00000E5D00000E5D0000099
:10039000E5D00000E5D00000E5D00000E5D0000089
:1003A000E5D00000E5D00000E5D00000E5D0000079
:1003B000E5D00000E5D00000E5D00000E5D0000069
:1003C000E5D00000E5D00000E5D00000E5D0000059
:1003D000E5D00000E5D00000E5D00000E5D0000049
:1003E000E5D00000E5D00000E5D00000E5D0000039
:1003F000E5D00000E5D00000E5D00000E5D0000029
:1004000048573031424C30313031000031303A31D0
:10041000333A32300000000044656320313120322D
:10042000303234000000000052502D303100000006
:1004300000000000000000000000000000000000BC
:10044000010000200A00D2B2002A05D0022A09D0F9
:1004500005D3032A09D00AE01022100007E0182271
:10046000100004E02822100001E048221000C0B271
:1004700070472DE9F04704000D00206810F1800658
:100480005FF000085FF0000AD4F8009000275046A3
:10049000C0B2002819D0022809D00FD303281BD1DD
:1004A000D9F8000C400E10F00300070014E0D9F852
:1004B000000C800D10F0030007000DE0D9F8000CCF
:1004C000C00C10F00300070006E0D9F8000C000C87
:1004D00010F003000700FFE73800C0B2FFF7B0FFDD
:1004E0000100C9B289083800C0B2002807D10A004B
:1004F000D2B2280080B2424316EB820636E03800C2
:10050000C0B201280FD10800C0B22A0092B22B005D
:100510009BB25FF0150C93FBFCF35B0002FB003019
:1005200016EB800622E03800C0B202280FD1080086
:10053000C0B22A0092B22B009BB25FF00C0C93FB6E
:10054000FCF39B0002FB003016EB80060EE0080077
:10055000C0B22A0092B22B009BB25FF0070C93FB53
:10056000FCF35B0002FB003016EB80063000BDE8B8
:10057000F087010000200A00D2B2002A082A0ED912
:10058000093A0ED0521E0FD0521E10D0521E11D05A
:10059000521E12D0521E13D0521E14D016E0080064
:1005A00014E00C22100011E0102210000EE01422C2
:1005B00010000BE01822100008E02022100005E0D7
:1005C0003022100002E040221000FFE7C0B2704766
:1005D0002DE9F84304000D0000275FF00009290011
:1005E00089B22000FFF745FF0600D6F800805FEAD9
:1005F000184818F00F084046C0B2FFF7BAFFC0B263
:10060000BDE8F28330B400241300DBB2002B0BD022
:10061000036853F4C0030360456815F0604521F09A
:1006200060431D4345600BE0036833F4C00303607F
:1006300043686FF39C437F4D15EA81451D43456038
:1006400030BC7047026832F47022026002680B000E
:10065000DBB21B0413F470231A4302607047026874
:1006600022F000420260026832F0804202600A001A
:10067000D2B2002A07D0026852F00042026002683B
:1006800052F08042026070470A00D2B2002A06D1BE
:10069000026832F070620260026802600BE00A00D9
:1006A000D2B2012A07D1026832F070620260026899
:1006B00052F080620260704710B44168496C11F0DA
:1006C0000101C9B2002909D05B494268116441683F
:1006D000496C11F00101C9B20029F8D1017C00294F
:1006E00020D101214268536933F080530C00E4B2F9
:1006F000240714F080542343536144686469240F31
:1007000014F00104E4B2002C39D10121426853698C
:1007100033F080530C00E4B2240714F080542343D8
:1007200053612CE0017C01290CD1012142685369FD
:1007300033F000530C00E4B2640714F00054234378
:1007400053611CE0017C02290CD1012142685369EC
:1007500033F080430C00E4B2A40714F08044234338
:1007600053610CE0017C032909D1012142685369DE
:1007700023F000430C00E4B253EAC473536110BC8D
:10078000704710B42C4A43681A64017C002920D1B8
:1007900001214268136933F400730C00E4B264026F
:1007A00014F400742343136144682469640A14F048
:1007B0000104E4B2002C3BD101214268136933F4F7
:1007C00000730C00E4B2640214F400742343136158
:1007D0002EE0017C01290CD101214268136933F418
:1007E00080630C00E4B2A40214F480642343136118
:1007F0001EE0017C02290CD101214268136933F407
:1008000000630C00E4B2E40214F4006423431361B7
:100810000EE0017C03290BD101214268136933F4F6
:1008200080530C00E4B2240314F480542343136176
:1008300010BC70470000FC1F7775637030B402680D
:10084000803200230024B4F5007F06D202EB84033B
:10085000190000230B60641CF5E70023802B08D2ED
:1008600002EB830414F50064210000240C605B1C7F
:10087000F4E700240B2C08D202EB840313F5206369
:10088000190000230B60641CF4E700230B2B08D233
:1008900002EB830414F52364210000240C605B1C2C
:1008A000F4E70024352C08D202EB840303F6A86396
:1008B000190000230B60641CF4E7036813F5005370
:1008C0000025B5F5207F06D203EB8502110000223A
:1008D0000A606D1CF5E700220468D2B204EB8202C4
:1008E00012F540520024802C06D202EB840319003A
:1008F00000230B60641CF6E730BC704770B4039CA7
:10090000049D6E7846742E780674016042608360A0
:10091000C46070BC7047002181600021016100212A
:100920004161002181610021C1600021C16100217C
:100930004162002181620021C16200210162012126
:1009400001700021C170002141715FF0FF314163EE
:100950008163C163002180F84410002141700021AF
:100960008170002180F83010002180F845100021AE
:1009700080F84710002180F84810002180F85110BD
:10098000002180F85010002180F85210002180F8DA
:100990005310002180F849100021C1647047F0B461
:1009A00000210268136833F080430C00E4B2A4070E
:1009B00014F0804423431360002405682E6836F049
:1009C00080562700FFB23F0717F080573E432E6046
:1009D00001680968090E11F00101C9B20029F7D1B7
:1009E000F0BC7047F8B5040020680068000D10F0F6
:1009F0000100C0B2002815D0002021680A6822F04A
:100A000000420300DBB252EAC3720A602068006849
:100A1000000D10F00100C0B2002803D02000FFF745
:100A2000B0FEF3E7012021680A6832F0007203008B
:100A3000DBB25B0613F000731A430A60206800689B
:100A4000400E10F00100C0B20028F7D1012021684B
:100A50000A6832F080420300DBB29B0713F0804348
:100A60001A430A60012325682E6836F080561F005D
:100A7000FFB23F0717F080573E432E6020680068A2
:100A8000000E10F00100C0B20028F7D02068006806
:100A9000C00E10F00100C0B20028EFD0F1BDF8B5D3
:100AA00004000D0016003100C9B289B22000FFF722
:100AB000E0FC07002A7A69683800FFF7A3FDA97AED
:100AC0003800FFF7BFFDE97A3800FFF7C8FD697A03
:100AD0003800FFF7D9FD287B002804D03100C9B2C7
:100AE000200001F0CAFD687A012808D12869310088
:100AF00022680B00DBB202EB8303C3F88008F1BD70
:100B00002DE9F04F86B0040000208DF8070000208A
:100B10008DF8060000208DF8050000208DF80400F7
:100B2000002500260020039000275FF0000E5FF0F4
:100B3000000C5FF000081000C0B299465FFA89F916
:100B400019F101095FEA59095FEA490919EB4009FE
:100B5000B9F1810F80F07C811800C0B250FA82F0A8
:100B60000128C0F275811000C0B200280CD0D00757
:100B700002D5501C050000E01500D00706D55FF037
:100B800001098DF8069001E0002005001800C0B2B0
:100B9000002817D01800C0B2401C40084019B0F11E
:100BA00001098DF804909DF80400402803D35FF0FC
:100BB0003F098DF80490D80708D55FF001098DF83A
:100BC000059003E0B5F101098DF804909DF80490BB
:100BD0008DF80190D4F80090D9F80CAC3AF47C5A16
:100BE0009DF80100000210F47C5050EA0A0ACDF88A
:100BF00008A00298C9F80C0C8DF80050D4F800A099
:100C0000DAF80CBC3BF4FE0B9DF80000000410F475
:100C1000FE0050EA0B0BCAF80CBC0020804691F88D
:100C200049901FFA88F81FFA89F9C84580F0A28018
:100C30005FF01408D1F84C9082461FFA8AFA08FB3C
:100C40000AFAD14499F80990B9F1010F40F0908067
:100C5000D1F84C9082461FFA8AFA08FB0AFAD1446E
:100C600099F80890B9F1010F40F082801EF1010E51
:100C70005FF0000A5FF00009CDF800A0D1F84CB099
:100C800082461FFA8AFA08FB0AFADA44DAF804A064
:100C9000DDF800B05AEA0B0A5646D1F84CA083465C
:100CA0001FFA8BFB08FB0BF8D044D8F8108028F013
:100CB000604858EA0909CDF80C900596ADF808C0CF
:100CC000D4F800A04FF44059BDF808800AEB88081A
:100CD000DDF814B048F809B01CF1010CADF800C003
:100CE000DDF80C80CDF81080BDF80080ADF80280F2
:100CF000D4F80080BDF802C008EB8C0CDDF810B011
:100D00004CF809B0BDF800C01CF1010C93465FFA25
:100D10008BFBDE452CD19DF80680B8F1000F26D064
:100D20000596ADF808C0D4F800A0BDF808800AEB1D
:100D30008808DDF814B048F809B01CF1010CADF8D2
:100D400000C0DDF80C80CDF81080BDF80080ADF853
:100D50000280D4F80080BDF802C008EB8C0CDDF8EE
:100D600010B04CF809B0BDF800C01CF1010C01E056
:100D7000401C53E75FF00008404691F8499080B26C
:100D80001FFA89F948455FD25FF01409C86CC24662
:100D90001FFA8AFA09FB0AFA5044407A012850D116
:100DA000C86CC2461FFA8AFA09FB0AFA5044007A54
:100DB000002846D17F1C0020D1F84CA0C3461FFA62
:100DC0008BFB09FB0BFBDA44DAF804A050EA0A407B
:100DD000D1F84CA0C3461FFA8BFB09FB0BF9D14499
:100DE000D9F810905FEA49595FEA595959EA000069
:100DF00006000296ADF800C020684FF44059BDF8D7
:100E000000A000EB8A0ADDF808B04AF809B01CF12E
:100E1000010C9A465FFA8AFA574512D19DF80500EF
:100E200000280DD00296ADF800C02068BDF800A0E3
:100E300000EB8A0ADDF808B04AF809B01CF1010C91
:100E400002E018F1010897E75FF001098DF80790BB
:100E50009DF8070006B0BDE8F08F2DE9F44F85B08E
:100E600005000C0000208DF80600002600208DF8FB
:100E7000050000208DF8040000208DF801000020FE
:100E80008DF80000002100225FF0000C00275FF0C9
:100E9000000E5FF000089DF81400401C4008400060
:100EA00099465FFA89F919F1010910EB5900812877
:100EB00080F039829DF8140050FA83F00128C0F2C6
:100EC00032829DF81400002815D09DF81400C00748
:100ED00008D59DF8149019F101095FEA59098DF8B8
:100EE00000900CE09DF814905FFA89F95FEA5909C7
:100EF0008DF8009003E05FF000098DF80090180075
:100F0000C0B2002824D09DF8000099465FFA89F904
:100F100019F101095FEA590919F101095FEA590953
:100F200019EB0000B0F101098DF801909DF8010066
:100F3000402803D35FF03F098DF8019013F0030FB1
:100F40000CD013F00309D9F104098DF8059005E0E0
:100F50009DF80000B0F101098DF801909DF8019015
:100F60008DF80390D5F80090CDF808900298D0F84D
:100F70000C9C39F47C599DF80300000210F47C505D
:100F800050EA0909CDF80C900398DDF80890C9F8EB
:100F90000C0C9DF800908DF802902868D0F80CACED
:100FA0003AF4FE0A9DF802905FEA094919F4FE0935
:100FB00059EA0A0AC0F80CAC5FF00009484694F8F8
:100FC000498080B21FFA88F8404580F0BD805FF00C
:100FD0001408E06CCA461FFA8AFA08FB0AFA504461
:100FE000407A012840F0AD80E06CCA461FFA8AFAC8
:100FF00008FB0AFA5044007A012840F0A2807F1CC6
:101000003000C0B2002849D1012006005FF0000A7C
:1010100000200200E06CCB461FFA8BFB08FB0BFBA9
:101020005844406850EA0A0A51469DF81400874225
:1010300040F0878052F08042E06CCA461FFA8AFA7C
:1010400008FB0AF84044406802430492ADF80AE005
:10105000D5F800804FF4405ABDF80A0008EB800034
:10106000DDF810B040F80AB01EF1010EADF802E054
:101070000391BDF802E0ADF808E02868BDF808E08B
:1010800000EB8E0EDDF80CB04EF80AB0BDF802E0B1
:101090001EF1010E5FF0000A564655E0E06CCA46AC
:1010A0001FFA8AFA08FB0AFA5044406881420FD2BC
:1010B00052F080421000E26CCA461FFA8AFA08FB1E
:1010C0000AF84244D2F80480020058EA02020CE016
:1010D000080050F080400200E06CCA461FFA8AFA0D
:1010E00008FB0AF84044406801000492ADF80AE0A9
:1010F000D5F800804FF4405ABDF80A0008EB800094
:10110000DDF810B040F80AB01EF1010EADF802E0B3
:101110000391BDF802E0ADF808E02868BDF808E0EA
:1011200000EB8E0EDDF80CB04EF80AB0BDF802E010
:101130001EF1010E5FF0000A56469DF814A05745B7
:1011400002D019F1010939E75FF00008404694F830
:10115000499080B21FFA89F9484580F07F805FF09E
:101160001409E06CC2461FFA8AFA09FB0AFA5044D5
:10117000407A01286FD1E06CC2461FFA8AFA09FB57
:101180000AFA5044007A002865D11CF1010C3000A5
:10119000C0B2002819D101200600002050F0804084
:1011A000D4F84CA0C3461FFA8BFB09FB0BF9D144C2
:1011B000D9F8049059EA000949461800C0B284459C
:1011C00049D1C1468DF8049048E04805400DD4F857
:1011D0004CA0C3461FFA8BFB09FB0BFBDA44DAF881
:1011E00004A050450AD2E06CC2461FFA8AFA09FBF5
:1011F0000AF94844406851EA004113E04805400DAF
:1012000002005FF08040D4F84CA0C3461FFA8BFB6D
:1012100009FB0BF9D144D9F8049059EA000959EABD
:101220000249494602917046D5F80090DDF808A0C1
:1012300083461FFA8BFB09EB8B0B1BF5405BCBF84E
:1012400000A01EF1010E5FF0000A56469A465FFAB2
:101250008AFAD44502D018F1010877E79DF8050015
:10126000002805D0022822D003D3032831D056E02D
:1012700055E0D4F84C909DF804A0142000FB0AFA25
:1012800009EB0A00406851EA004102917046D5F826
:101290000090DDF808A083461FFA8BFB09EB8B0B4F
:1012A0001BF5405BCBF800A01EF1010E37E0029168
:1012B0007046D5F80090DDF808A083461FFA8BFB36
:1012C00009EB8B0B1BF5405BCBF800A01EF1010E68
:1012D00025E00491ADF80AE0D5F800904FF4405AAB
:1012E000BDF80A0009EB8000DDF810B040F80AB044
:1012F0001EF1010EADF802E00391BDF802E0ADF879
:1013000008E02868BDF808E000EB8E0EDDF80CB0B0
:101310004EF80AB0BDF802E01EF1010EFFE75FF0E3
:1013200001098DF806909DF8060006B0BDE8F08F23
:101330002DE9F84F85B005000B00140000208DF852
:101340000600002600208DF8050000208DF804001E
:1013500000208DF8010000208DF8000000210022FF
:1013600000275FF0000C5FF0000E5FF00008200027
:10137000C0B2401C400840009DF8149019F10109CA
:1013800010EB5900812880F001829DF8140050FA7A
:1013900084F00128C0F2FA812000C0B2002813D0E6
:1013A000E00709D5A1465FFA89F919F101095FEA59
:1013B00059098DF800900BE0A1465FFA89F95FEAC0
:1013C00059098DF8009003E05FF000098DF8009056
:1013D0009DF81400002827D09DF800009DF8149077
:1013E00019F101095FEA590919F101095FEA59097F
:1013F00019EB0000B0F101098DF801909DF8010092
:10140000402803D35FF03F098DF801909DF8140048
:1014100010F0030F0ED09DF8149019F00309D9F1C4
:1014200004098DF8059005E09DF80000B0F1010970
:101430008DF801909DF801908DF80390D5F80090FB
:10144000CDF808900298D0F80C9C39F47C599DF89E
:101450000300000210F47C5050EA0909CDF80C900A
:101460000398DDF80890C9F80C0C9DF800908DF8F1
:1014700002902868D0F80CAC3AF4FE0A9DF802906D
:101480005FEA094919F4FE0959EA0A0AC0F80CACE6
:101490005FF00009484693F8498080B21FFA88F847
:1014A000404580F0A4805FF01408D86CCA461FFA4B
:1014B0008AFA08FB0AFA5044407A012840F09480E6
:1014C000D86CCA461FFA8AFA08FB0AFA5044007A16
:1014D000012840F089801CF1010C3000C0B20028C6
:1014E00048D1012006005FF0000A002002005AF0F7
:1014F000004AD86CCB461FFA8BFB08FB0BFB584409
:10150000406850EA0A0A51462000C0B284456BD1B7
:10151000D86CCA461FFA8AFA08FB0AF840444068A9
:1015200002430491ADF80AE0D5F800804FF4405A28
:10153000BDF80A0008EB8000DDF810B040F80AB0F2
:101540001EF1010EADF802E00392BDF802E0ADF825
:1015500008E02868BDF808E000EB8E0EDDF80CB05E
:101560004EF80AB0BDF802E01EF1010E5FF0000A6D
:1015700056463CE01000DA6CCA461FFA8AFA08FBAD
:101580000AF84244D2F80480020058EA02020491A8
:10159000ADF80AE0D5F800804FF4405ABDF80A00D3
:1015A00008EB8000DDF810B040F80AB01EF1010E23
:1015B000ADF802E00392BDF802E0ADF808E028685B
:1015C000BDF808E000EB8E0EDDF80CB04EF80AB066
:1015D000BDF802E01EF1010E5FF0000A5646A24679
:1015E0005FFA8AFAD44502D019F1010952E75FF097
:1015F0000008404693F8499080B21FFA89F948459F
:1016000055D25FF01409D86CC2461FFA8AFA09FB5A
:101610000AFA5044407A012846D1D86CC2461FFAD3
:101620008AFA09FB0AFA5044007A00283CD17F1C50
:101630003000C0B2002819D101200600002050F06F
:101640000040D3F84CA0C3461FFA8BFB09FB0BF9F3
:10165000D144D9F8049059EA000949469DF814008C
:10166000874221D1C1468DF8049020E0D86CC24653
:101670001FFA8AFA09FB0AF94844406851EA004116
:1016800002917046D5F80090DDF808A083461FFA55
:101690008BFB09EB8B0B1BF5405BCBF800A01EF11D
:1016A000010E5FF0000A564618F10108A1E79DF807
:1016B0000500012804D065D3032831D01ED361E092
:1016C000D3F84C909DF804A0142000FB0AFA09EB13
:1016D0000A00406851EA004102917046D5F8009036
:1016E000DDF808A083461FFA8BFB09EB8B0B1BF57B
:1016F000405BCBF800A01EF1010E43E00291704662
:10170000D5F80090DDF808A083461FFA8BFB09EBA3
:101710008B0B1BF5405BCBF800A01EF1010E31E0F6
:10172000D3F84C909DF804A0142000FB0AFA09EBB2
:101730000A00406851EA00410491ADF80AE0D5F88A
:1017400000904FF4405ABDF80A0009EB8000DDF824
:1017500010B040F80AB01EF1010EADF802E003919E
:10176000BDF802E0ADF808E02868BDF808E000EB3D
:101770008E0EDDF80CB04EF80AB0BDF802E01EF196
:10178000010EFFE75FF001098DF806909DF8060055
:1017900006B0BDE8F08F2DE9F04704000D000026EB
:1017A000002700205FF000085FF000095FF0000AEA
:1017B000504695F84910C0B2884227D21421E86CEF
:1017C0005246D2B24A431044407A01281BD1E86CF9
:1017D0005246D2B24A431044007A002801D17F1CFD
:1017E00000E0761CE86C5246D2B201FB02F10844DC
:1017F000807AFEF7BEFE814640464946C0B2C9B275
:10180000884200D2C8461AF1010AD1E76879012856
:1018100018D100204146C9B21031042291FBF2F1E7
:10182000491E0A002368D3F80CCC3CF0F84C9646CD
:101830005FFA8EFE5FEA8E6E1EF0F84E5EEA0C0CCA
:10184000C3F80CCC95F85500002803D0022813D01B
:1018500009D31AE03B00DBB23200D2B229002000EB
:10186000FFF74EF911E03B00DBB23200D2B22900A3
:101870002000FFF7F2FA08E03B00DBB23200D2B200
:1018800029002000FFF754FDFFE7BDE8F0872DE9B0
:10189000F24F88B0040000208DF805002568286804
:1018A00030F000509DF80510490711F00051084331
:1018B00007900798286001208DF804002668D6F864
:1018C0000C0C20F000409DF8041050EAC170069006
:1018D0000698C6F80C0C2768D7F8140C50F0006076
:1018E000C7F8140C00208DF80300D4F80080D8F855
:1018F000100C20F000409DF8031050EAC1700590D4
:101900000598C8F8100C00208DF80200D4F800905B
:10191000D9F8100C30F080409DF80210890711F0C2
:101920008041084304900498C9F8100C00208DF8F9
:101930000100D4F800A0DAF8100C30F000509DF847
:101940000110490711F00051084303900398CAF8A9
:10195000100C00208DF80000D4F800B0DBF8100C5B
:1019600030F080509DF80010090711F080510843B5
:1019700002900298CBF8100C08992000FFF70BFF9B
:1019800000202168D1F80C2C520952010300DBB26F
:1019900013F01F031A43C1F80C2C09B0BDE8F08FF7
:1019A0002DE9F04F8BB004000D0000208DF80100F0
:1019B0002000FEF781FE01208DF8030026683068C4
:1019C00020F000409DF8031050EAC1700490049884
:1019D000306028788DF800002768786830F400506F
:1019E0009DF80010490311F4005108430390039837
:1019F00078602000FEF7F6FF5FF00108D4F8009051
:101A0000D9F8000030F400004146C9B2C90511F40C
:101A10000001084302900298C9F800005FF0010A33
:101A2000D4F800B0DBF8340030F080505146C9B231
:101A3000090711F08051084301900198CBF8340058
:101A40002000FEF7FBFE95F83000FEF7F9FC8DF85C
:101A500002009DF80200002809D04FF400709DF8A4
:101A60000210B0FBF1F1607C41438DF801109DF84C
:101A700001008DF8030021680868C009C0019DF8C5
:101A8000032012F07F02104309900998086095F82E
:101A900059008DF800002268506830F080009DF8F1
:101AA0000030DB0113F08003184308900898506061
:101AB00001232668306D20F000401F00FFB250EA7D
:101AC000C770079007983065A868401EADF80A00F7
:101AD0002768386D6FF35E50BDF80AC0DFF8C8E9BB
:101AE0001EEA4C5E5EEA0000069006983865E868DB
:101AF000401EADF80800D4F800E0DEF8500030F4E5
:101B0000F810BDF808C05FEA0C4C1CF4F81C5CEA45
:101B1000000005900598CEF850002869401EADF8E9
:101B20000600D4F80080D8F8500030F47C40BDF8AE
:101B300006C05FEA8C2C1CF47C4C5CEA000004902C
:101B40000498C8F850006869401EADF80400D4F845
:101B50000090D9F8500030F47870BDF804C05FEA06
:101B60004C1C1CF4787C5CEA000003900398C9F8D4
:101B70005000A869B0F1010AD4F800C0DCF850B0F8
:101B80005FEA5B1B5FEA4B1B504680B210F01F0000
:101B900050EA0B0BCCF850B06878002800F0B981FF
:101BA00068788DF803002168086830F400609DF8BB
:101BB0000320D20212F4006210430A900A980860CF
:101BC00001222368D3F8000C20F000401600F6B282
:101BD00050EAC67009900998C3F8000CE869401EE5
:101BE000ADF80C002668D6F8040C6FF31D50BDF854
:101BF0000C70DFF8B8C81CEA075C5CEA00000890CB
:101C00000898C6F8040C286A401EADF80A00276838
:101C1000D7F8040C30F4E020BDF80AC05FEA0C4CA1
:101C20001CF4E02C5CEA000007900798C7F8040C4D
:101C3000686AADF80800D4F800E0DEF8040C30F46F
:101C4000F840BDF808C05FEA8C2C1CF4F84C5CEA44
:101C5000000006900698CEF8040CA86A401EADF865
:101C60000600D4F80080D8F8040C30F0E000BDF88D
:101C700006C05FEA4C1C1CF0E00C5CEA000005901A
:101C80000598C8F8040CE86A401EADF80400D4F8C2
:101C90000090D9F8040CC008C000BDF804C01CF0C6
:101CA000070C5CEA000004900498C9F8040C95F84D
:101CB00030008DF800005FF0000CD4F800A0DAF8D6
:101CC000000CE3465FFA8BFBBBF1000F24D0BBF1A5
:101CD000020F0DD016D3BBF1030F27D130F0C06037
:101CE00001009DF80000400610F0C06008431DE0B0
:101CF00030F4400001009DF80000800510F4400021
:101D0000084313E030F4C01001009DF80000C00447
:101D100010F4C010084309E030F4403001009DF891
:101D20000000000410F440300843FFE7CAF8000C3C
:101D300095F8301001222368D3F8006C1700FFB229
:101D4000002F22D0022F0CD015D3032F27D136F02D
:101D5000C06630000E00F6B2760616F0C066064386
:101D60001DE036F4400630000E00F6B2B60516F45B
:101D70004006064313E036F4C01630000E00F6B2FB
:101D8000F60416F4C016064309E036F44036300077
:101D90000E00F6B2360416F440360643FFE7C3F8E9
:101DA000006C95F830005FF0020E2768D7F800CC81
:101DB000F0465FFA88F8B8F1000F2DD0B8F1020FA5
:101DC00010D01CD3B8F1030F33D13CF0C06C614686
:101DD00084465FFA8CFC5FEA4C6C1CF0C06C5CEAD9
:101DE000010C26E03CF4400C614684465FFA8CFC12
:101DF0005FEA8C5C1CF4400C5CEA010C19E03CF4DA
:101E0000C01C614684465FFA8CFC5FEACC4C1CF433
:101E1000C01C5CEA010C0CE03CF4403C614684468A
:101E20005FFA8CFC5FEA0C4C1CF4403C5CEA010C51
:101E3000FFE7C7F800CC95F8301003222368D3F8E9
:101E4000006C90465FFA88F8B8F1000F24D0B8F122
:101E5000020F0DD016D3B8F1030F27D136F0C066AC
:101E600030000E00F6B2760616F0C06606431DE09E
:101E700036F4400630000E00F6B2B60516F4400601
:101E8000064313E036F4C01630000E00F6B2F60436
:101E900016F4C016064309E036F4403630000E0052
:101EA000F6B2360416F440360643FFE7C3F8006C7A
:101EB00095F84500002820D195F847002168D1F811
:101EC000002C32F400420300DBB2DB0313F40043C6
:101ED0001A43C1F8002C95F848302668D6F8007CE3
:101EE00037F4F8579C465FFA8CFC5FEA0C2C1CF424
:101EF000F85C5CEA0707C6F8007CA87821684A6BA2
:101F000032F480520300DBB21B0313F480531A43F4
:101F10004A63E878002843D0207C00280BD10020B9
:101F20002168D1F80C2C22F000420300DBB252EA07
:101F3000C372C1F80C2C012021680A6832F00052EB
:101F40000300DBB25B0713F000531A430392039ABA
:101F50000A602A6C02922268029B93646B6B019365
:101F60002368019E1E61AE6B27687E61D5F83CC078
:101F7000D4F800E0CEF818C095F84480D4F800906A
:101F8000D9F800A03AF4803AC3465FFA8BFB5FEAC7
:101F90000B4B1BF4803B5BEA0A0AC9F800A09AE0ED
:101FA0002879002808D0207C002840F0948029005F
:101FB0002000FFF76CFC8EE000212268136833F0EC
:101FC00000530800C0B2400710F0005003431360F4
:101FD000207C002863D100208DF800002068D0F814
:101FE0000C1C21F000419DF8002051EAC2710491BF
:101FF0000499C0F80C1C2168D1F8142C52F000622E
:10200000C1F8142C00222368D3F8106C26F0004687
:102010001700FFB256EAC7760396039EC3F8106C0A
:1020200000262768D7F810EC3EF0804EB4465FFAE1
:102030008CFC5FEA8C7C1CF0804C5CEA0E0ECDF8C8
:1020400008E0DDF808C0C7F810CC5FF0000ED4F847
:102050000080D8F8109C39F00059F4465FFA8CFCE7
:102060005FEA4C7C1CF0005C5CEA0909CDF8049046
:10207000DDF804C0C8F810CC5FF0000CD4F8009074
:10208000D9F810AC3AF0805AE3465FFA8BFB5FEA6E
:102090000B7B1BF0805B5BEA0A0AC9F810AC686B2B
:1020A00021680861AA6B23685A61EE6B2768BE61DC
:1020B00095F844C0D4F800E0DEF8008038F48038A9
:1020C000E1465FFA89F95FEA094919F4803959EA6A
:1020D0000808CEF8008069792268136833F4004359
:1020E0000800C0B2C00310F400400343136095F829
:1020F000450000281BD0002021680A6832F4003215
:102100000300DBB25B0413F400331A430A600123BB
:102110002668776837F480579C465FFA8CFC5FEA44
:102120000C3C1CF4805C5CEA070777601AE0012035
:1021300021680A6832F400320300DBB25B0413F456
:1021400000331A430A6000232668776837F4805703
:102150009C465FFA8CFC5FEA0C3C1CF4805C5CEAF9
:102160000707776095F846102268536833F0080334
:102170000800C0B2C00010F008000343536095F897
:10218000500000282ED0012021680A6832F4800215
:102190000300DBB29B0513F480031A430A6001239A
:1021A0002668376837F080679C465FFA8CFC5FEAE8
:1021B0008C6C1CF0806C5CEA070737605FF0010CE8
:1021C000D4F800E0DEF8008038F48028E1465FFAB9
:1021D00089F95FEA894919F4802959EA0808CEF893
:1021E00000802DE0002021680A6832F4800203009C
:1021F000DBB29B0513F480031A430A6000232668B0
:10220000376837F080679C465FFA8CFC5FEA8C6C1D
:102210001CF0806C5CEA070737605FF0000CD4F8B4
:1022200000E0DEF8008038F48028E1465FFA89F9A2
:102230005FEA894919F4802959EA0808CEF8008034
:1022400001212268506830F04000069006985060E6
:1022500095F851008DF806002368186830F4805016
:102260009DF80660360316F48056304305900598B5
:10227000186095F852008DF805002668706830F4F3
:1022800000409DF80570FF0317F4004738430490A1
:102290000498706095F853008DF8040027687868FA
:1022A00030F480409DF804C05FEA8C3C1CF4804C04
:1022B0005CEA000003900398786095F854008DF86C
:1022C0000300D4F800E0DEF8000030F400109DF8C0
:1022D00003C05FEA4C5C1CF4001C5CEA0000029046
:1022E0000298CEF8000095F854008DF80000D4F85C
:1022F00000C0DCF8048038F400689DF80000C002DB
:1023000010F4006050EA0808CCF8048095F854A056
:10231000D4F80090D9F804B03BF4806B5046C0B2BA
:10232000800210F4806050EA0B0BC9F804B02879E1
:1023300000282ED100200026300095F84910C0B2A8
:1023400088425DD200201427E96C3200D2B27A4371
:1023500031F80280404680B2E96C3200D2B27A4352
:10236000895AEA6C3300DBB27B431A445288511815
:1023700088420CDA4246D2B2E86C3100C9B27943E5
:1023800001442000FEF78BFB18F10108E2E7761C00
:10239000D2E700200026300095F84910C0B28842EC
:1023A0002ED200201427E96C3200D2B27A4331F8E1
:1023B0000280404680B2E96C3200D2B27A43895A38
:1023C000EA6C3300DBB27B431A44528851188842CE
:1023D00014DAE86C3100C9B279430844407A002825
:1023E00009D14246D2B2E86C3100C9B27943014406
:1023F0002000FEF754FB18F10108DAE7761CCAE763
:1024000095F856008DF800002668706B30F4004097
:102410009DF80010C90311F400410843029002988E
:10242000706395F85870D4F80080D8F8340030F410
:1024300040703900C9B2090211F44071084301909B
:102440000198C8F8340095F85790D4F800A0DAF84D
:1024500034B03BF0C00B4846C0B2800110F0C00061
:1024600050EA0B0BCAF834B0200000F089F8207C49
:10247000002807D12879012804D15FF0704120009D
:1024800000F000FB2000FEF78AFA002021680A68AD
:1024900032F400020300DBB2DB0513F400031A433D
:1024A0000A600BB0BDE8F08F0000E07F0000F03F55
:1024B00038B504000D00297889B22000FDF7D9FF56
:1024C000016851F04061016031BDF8B504000D00B4
:1024D000297889B22000FDF7CCFF10F10806297891
:1024E00089B22000FEF774F8002100221100C9B261
:1024F000814244D212F0030F0AD1002131603168C9
:102500001300DBB22B441B7A51EA0361316034E0E3
:102510001100C9B2042391FBF3F703FB1711012942
:1025200008D131681300DBB22B441B7A51EA034116
:10253000316022E01100C9B2042391FBF3F703FBE1
:102540001711022908D131681300DBB22B441B7A22
:1025500051EA0321316010E01100C9B2042391FB5C
:10256000F3F703FB1711032907D133681100C9B230
:102570002944097A0B433360361D521CB6E7F1BD7E
:10258000F0B4417C032937D15FF0FF310A00022605
:102590000368002E0AD0022E04D005D3032E07D1E3
:1025A0001A6705E05A6703E0DA6201E01A63FFE7A1
:1025B0000C0001270568002F0AD0022F04D005D394
:1025C000032F07D12C6705E06C6703E0EC6201E0A4
:1025D0002C63FFE700230268002B0AD0022B04D0F3
:1025E00005D3032B07D1116705E0516703E0D162E2
:1025F00001E01163FFE73EE0417C022925D15FF055
:10260000FF310A0001250368002D0AD0022D04D0F5
:1026100005D3032D07D11A6705E05A6703E0DA6294
:1026200001E01A63FFE700260468002E0AD0022E9C
:1026300004D005D3032E07D1216705E0616703E0CD
:10264000E16201E02163FFE715E0417C012912D13D
:102650005FF0FF3100230268002B0AD0022B04D068
:1026600005D3032B07D1116705E0516703E0D16261
:1026700001E01163FFE7F0BC7047F0B400240A00EA
:10268000D2B2202392FBF3F503FB152201239340E2
:102690000D00EDB2402D1ADB1C0002260568002E4D
:1026A00010D0022E06D009D3032E0FD1AF6E2743D0
:1026B000AF660BE0EF6E2743EF6607E06F6A2743D4
:1026C0006F6203E0AF6A2743AF62FFE738E00C00B8
:1026D000E4B2202C1ADB1C0001260568002E10D065
:1026E000022E06D009D3032E0FD1AF6E2743AF665B
:1026F0000BE0EF6E2743EF6607E06F6A27436F62D8
:1027000003E0AF6A2743AF62FFE719E01C00002631
:102710000568002E10D0022E06D009D3032E0FD14B
:10272000AF6E2743AF660BE0EF6E2743EF6607E01F
:102730006F6A27436F6203E0AF6A2743AF62FFE728
:10274000F0BC70472DE9F14F2DED068B8AB008EEF5
:10275000101A08EE902A9A469FED840A01200590EF
:10276000012004905FF00809032001900221142049
:1027700008909FED7F9AF5EE009A9DF86C00002876
:1027800010D040F2FF3007905E24032006901F20F7
:102790000290DDF8088018EB040818F101085FF0DA
:1027A000080B0FE040F2FF3007902624032006902C
:1027B00007200290DDF8088018EB040818F10108E2
:1027C0005FF0080BF8EE680A01250798A84246DB7F
:1027D000B8EE480A01EE105AB8EEC11A80EE010AAE
:1027E000B8EE681A80EE011ABDEEC11A8DED001A1E
:1027F0000098002802D00098584500DA2FE09DED9F
:10280000001AB8EEC11A80EE011AF8EE681A71EEDD
:10281000611AF5EE401AF1EE10FA04DDF8EE681ACE
:1028200071EE611A03E0F8EE681A71EEC11A0098B1
:10283000804512DBF4EE610AF1EE10FA0DDB05952E
:1028400000988146F0EE610A0898009A904204DBF5
:10285000F4EE491AF1EE10FA01D46D1CB5E75046BA
:1028600080B200EE100AB8EE400A20EE290AA14517
:1028700000DA4C4626000698864227DB721C42F29C
:102880001070424392FBF9F0524692B2821A012A2A
:1028900005DB524692B2821A00EE902A04E05246BC
:1028A00092B2121A00EE902A524692B290420DDB7A
:1028B000B8EEE01AB4EE401AF1EE10FA04D5019623
:1028C000F8EEE00AB0EE600A761ED4E70198B9EBA4
:1028D0000000401E03909FED27AA01270398B842ED
:1028E00023DB42F2107000FB07F090FBF9F0BDF81B
:1028F0006810411A012905DBBDF86810411A00EE85
:10290000101A04E0BDF86810091A00EE101AF8EE6B
:10291000C00AF4EE4A0AF1EE10FA04D50497B8EEB4
:10292000C00AB0EE40AA7F1CD8E70598109908604D
:10293000019800F09FF95FF033320F4B00F0ACF9D3
:1029400000F080FA10998860019910988068091A3F
:102950001098C16003981099086104981099486014
:102960000AB0BDEC068BBDE8F18F0000000000004E
:10297000CDCCCC3D00401C463333E33F70B4130054
:10298000DBB2012B3ED1CB000DD501230468D4F876
:10299000105C35F080551E00F6B2360716F08056F2
:1029A0003543C4F8105C8B000DD501230468D4F8BE
:1029B000105C35F000551E00F6B2760716F0005692
:1029C0003543C4F8105C4B000DD501230468D4F8DE
:1029D000105C35F080451E00F6B2B60716F0804652
:1029E0003543C4F8105C00294AD501230468D4F8A3
:1029F000105C25F000451E00F6B255EAC675C4F815
:102A0000105C3DE0CB000DD500230468D4F8105CC9
:102A100035F080551E00F6B2360716F08056354365
:102A2000C4F8105C8B000DD500230468D4F8105C4A
:102A300035F000551E00F6B2760716F00056354305
:102A4000C4F8105C4B000DD500230468D4F8105C6A
:102A500035F080451E00F6B2B60716F080463543C5
:102A6000C4F8105C00290BD500230468D4F8105C6E
:102A700025F000451E00F6B255EAC675C4F8105C94
:102A800070BC7047CA0004D502685FF08053C2F87A
:102A9000143C8A0004D502685FF00053C2F8143C6D
:102AA0004A0004D502685FF08043C2F8143C002954
:102AB00004D502685FF00043C2F8143C704702007E
:102AC00000200B00B3F1805F09D0B3F1005F12D09A
:102AD000B3F1804F1BD0B3F1004F24D02DE0136829
:102AE000D3F8143C1B0F13F00103DBB2002B01D011
:102AF0000123180021E01368D3F8143C5B0F13F096
:102B00000103DBB2002B01D00123180015E013688C
:102B1000D3F8143C9B0F13F00103DBB2002B01D060
:102B20000123180009E01368D3F8143CDB0FDBB273
:102B3000002B01D001231800FFE7C0B2704701004D
:102B400000200A68D2F8142C520C12F00102D2B202
:102B5000002A01D001221000C0B2704701000020FD
:102B60000A68D2F8142C120C12F00102D2B2002A18
:102B700001D001221000C0B2704701000022086895
:102B8000D0F8140C10F03F00C0B270472DE9F047A8
:102B900004000D00206810F5005A5FF000090026BF
:102BA000DAF800703F0C17F00F07DAF80000A5F80C
:102BB0004A003800C0B2FDF7DCFC85F84800DAF8BE
:102BC0000000C0F3405818F001081AF10400414613
:102BD000C9B2002904D0016821F06041696003E0B6
:102BE0000168C1F38A416960001D5FF00009494630
:102BF00095F84820C9B2914232D219F0030F06D19C
:102C00000168090E4A46D2B22A44117225E04946AB
:102C1000C9B2042291FBF2F302FB1311012906D180
:102C20000168090C4A46D2B22A44117215E049469D
:102C3000C9B2042291FBF2F302FB1311022906D15F
:102C40000168090A4A46D2B22A44117205E00168B5
:102C50004A46D2B22A441172001D19F10109C6E791
:102C6000061D3068E8645FF080512000FFF70AFF1E
:102C7000BDE8F08710F0004160B148BF4042B0FAB3
:102C800080F29040D21CC2F5846241EA025202EB0B
:102C9000D02140057047FEE730B540F2FF7C1CEACA
:102CA00011541DBF1CEA1355644565453FE0641986
:102CB00081EA030C6FF35F530CF0004C43F4801374
:102CC000C90241F0004141EA505EC5021100A5FB76
:102CD000020200284FF00000EEFB01204FF000013F
:102CE000E3FB052118BF42F00102401800214941D1
:102CF000E3FB0E01A4F580640D0302D2921840415B
:102D0000494154F1010470DD450872F1004250F16F
:102D1000000051EB0451A1F5801102D441EA0C01ED
:102D200030BD40F2FF7E4CEA0E51002030BD0CEA6F
:102D30001355644518BF654581EA030C0CF0004C3F
:102D400041D050EA410E1CBF52EA430E02E06146F8
:102D5000002030BD24422C441BD15FEA050EF6D082
:102D6000090302BF01460020AEF1140EB1FA81F54D
:102D7000AEEB050401FA05FE0C35C5F1200100FAA1
:102D800005F5C8404EEA000E6FF35F5343F480131D
:102D90009CE733F00043B3FA83F504BFB2FA82FE36
:102DA00075440B3D641BB5F1200E2FBF02FA0EF3E4
:102DB000AB40C5F1200E22FA0EFE38BF43EA0E03E7
:102DC000AA40641C7CE750EA410E14BF52EA430E4D
:102DD0006FF000014FF4001515EB430F8EBF19463D
:102DE00015EB410F9DE7B4D830BDD4F10104B4F127
:102DF00020050FDAC4F12005520828BF42F0010275
:102E000010FA05FE01FA05F57244E2BFE0402843DE
:102E1000E1400FE0352C9ADCC5F1200452EA400273
:102E200020FA05F218BF42F0010231FA05F0A14084
:102E30000A43002172F1004250F1000051EB0C01F5
:102E400030BDFEE7400D40F21E4C40EAC120BCEB15
:102E5000115C40F0004003D48CF30701C840704778
:102E60006FEAE1707047FEE7020010688068C0F307
:102E70004000C0B200280AD01068C068C0F340000B
:102E8000C0B2002803D010690860012000E00020D3
:102E9000704730B4020000231468A56835F00205BD
:102EA0001800C0B2400010F002000543A560087889
:102EB000002812D0012013689C6834F00204050039
:102EC000EDB26D0015F002052C439C601068C068DF
:102ED000C0F34000C0B20028F8D0012030BC7047D9
:102EE000020010688068C0F38000C0B200280AD0D9
:102EF0001068C068C0F38000C0B2002803D0906999
:102F00000860012000E000207047F0B502000023B7
:102F10001468A56835F004051800C0B2800010F0F0
:102F200004000543A5600878002842D09069224B30
:102F3000984201D2002312E09069204B984201D2BE
:102F400001230CE090691E4B984201D2022306E057
:102F500090691C4B984201D2032300E0042318001F
:102F6000C0B2042801D1002024E0180014682568AC
:102F700035F00C050600F6B2B60016F00C06354327
:102F8000256001261768D7F808C03CF0040CB64647
:102F90005FFA8EFE5FEA8E0E1EF0040E5EEA0C0CE7
:102FA000C7F808C01068C068C0F38000C0B200282D
:102FB000F8D00120F0BD000000093D0000127A00A9
:102FC00000366E01015A620202001068806810F03B
:102FD0000100C0B200280AD01068C06810F00100DB
:102FE000C0B2002803D050690860012000E0002032
:102FF000704730B4020000231468A5686D086D00A6
:103000001800C0B210F001000543A5600878002840
:1030100011D0012013689C68640864000500EDB2BB
:1030200015F001052C439C601068C06810F0010089
:10303000C0B20028F8D0012030BC7047F8B50400B9
:103040000D00002620688068C0F3C000C0B20028D0
:1030500069D02068C068C0F3C000C0B2002862D048
:103060002068406810F00300C0B2002803D0022896
:103070000DD006D311E069462000FFF7F5FE0600EB
:103080000BE069462000FFF79FFF060005E0694658
:103090002000FFF725FF0600FFE73000C0B2002840
:1030A00001D1002041E0012220684068C0F3810086
:1030B000C0B2002805D0022809D005D3032809D0C2
:1030C0000BE00120020008E00220020005E00420DD
:1030D000020002E008200200FFE720684168090AB8
:1030E00011F07F01C9B2002901D18021FFE72068DA
:1030F0004068C0F30210C0B2002801D10820FFE7E9
:1031000023685B681B0C13F00103DBB25B1C009FA0
:103110004F435F4300FB02FC5FEA4C0CB7FBFCF73C
:103120002F6001273E003000C0B2F2BDF0B40200B3
:1031300000201468A56835F008050300DBB2DB0049
:1031400013F008031D43A56001234E78002E03D021
:10315000022E19D00CD323E0022014686568AD0854
:10316000AD000600F6B216F003063543656019E0BF
:10317000012014686568AD08AD000600F6B216F0CF
:103180000306354365600DE0002014686568AD08EE
:10319000AD000600F6B216F003063543656001E0A7
:1031A000002003001800C0B2002801D1002088E0F0
:1031B000C868012801D100240FE0C868022801D1A5
:1031C00001240AE0C868042801D1022405E0C86887
:1031D000082801D1032400E0FF242000C0B2FF280A
:1031E00001D100206DE025001668776837F00C07E4
:1031F0002800C0B2800010F00C00074377604888B8
:10320000002817D04888812814DA4888802801D1FE
:10321000002500E04D881668776837F4FE472800DF
:10322000C0B2000210F4FE4007437760086900282E
:1032300002D119E0002044E00869092814D2086985
:10324000082801D1002000E0086915686E6836F092
:1032500070060700FFB23F0117F070073E436E6033
:103260008F68012F02D104E000202AE0886802283C
:1032700010D18868451E1668776837F480372800B3
:10328000C0B2000410F4803007437760087800284B
:1032900002D114E0002014E001201568AE6836F079
:1032A00008060700FFB2FF0017F008073E43AE60B4
:1032B0001068C068C0F3C000C0B20028F8D0180081
:1032C000C0B2F0BC70477CB504000D0000260020A1
:1032D0000090A0684068C0F38000C0B2002817D0FA
:1032E00069462000FFF7FCFD06003000C0B2002850
:1032F0000ED0A068016911F0070101208840412823
:1033000004D20099B1FBF0F0286001E000210E002A
:103310003000C0B276BDF0B40300002000229C68EB
:10332000656835F004051600F6B2B60016F004061E
:10333000354365608E88012E01D100241EE08A8805
:10334000022A01D1012419E08A88042A01D1022429
:1033500014E08A88082A01D103240FE08A88102A01
:1033600001D104240AE08A88202A01D1052405E03D
:103370008A88402A01D1062400E007242200D2B224
:10338000072A0CD022009D682E69F608F600170067
:10339000FFB217F007073E432E61012738000A7875
:1033A000002A01D0012200E000229D686E6836F0FC
:1033B00004061700FFB2BF0017F004073E436E601B
:1033C000C0B2F0BC70477CB504000D0000260020A0
:1033D0000090A0684068C0F3C000C0B2002817D0B9
:1033E00069462000FFF77CFD06003000C0B20028CF
:1033F0000ED0A0680069C0F3021101208840412866
:1034000004D20099B1FBF0F0286001E000210E0029
:103410003000C0B276BDF0B40300002000229C68EA
:10342000656835F008051600F6B2F60016F00806D5
:10343000354365608E88012E01D100241EE08A8804
:10344000022A01D1012419E08A88042A01D1022428
:1034500014E08A88082A01D103240FE08A88102A00
:1034600001D104240AE08A88202A01D1052405E03C
:103470008A88402A01D1062400E007242200D2B223
:10348000072A0DD022009D682E6936F070061700BD
:10349000FFB23F0117F070073E432E61012738004D
:1034A0000A78002A01D0012200E000229D686E689F
:1034B00036F008061700FFB2FF0017F008073E437A
:1034C0006E60C0B2F0BC70477CB504000D000026F1
:1034D00000200090A0684068C0F30010C0B200282F
:1034E00017D069462000FFF76FFD06003000C0B21C
:1034F00000280ED0A068016A11F007010120884061
:10350000412804D20099B1FBF0F0286001E00021CD
:103510000E003000C0B276BDF0B4030000200022DF
:103520009C68656835F010051600F6B2360116F095
:103530001006354365608E88012E01D100241EE0FF
:103540008A88022A01D1012419E08A88042A01D13B
:10355000022414E08A88082A01D103240FE08A8813
:10356000102A01D104240AE08A88202A01D10524E6
:1035700005E08A88402A01D1062400E007242200C1
:10358000D2B2072A0CD022009D682E6AF608F600F7
:103590001700FFB217F007073E432E6201273800DD
:1035A0000A78002A01D0012200E000229D686E689E
:1035B00036F010061700FFB23F0117F010073E4328
:1035C0006E60C0B2F0BC70477CB504000D000026F0
:1035D00000200090A0684068C0F34010C0B20028EE
:1035E00017D069462000FFF7EFFC06003000C0B29C
:1035F00000280ED0A068006AC0F3021101208840A4
:10360000412804D20099B1FBF0F0286001E00021CC
:103610000E003000C0B276BDF0B4030000200022DE
:103620009C68656835F020051600F6B2760116F044
:103630002006354365608E88012E01D100241EE0EE
:103640008A88022A01D1012419E08A88042A01D13A
:10365000022414E08A88082A01D103240FE08A8812
:10366000102A01D104240AE08A88202A01D10524E5
:1036700005E08A88402A01D1062400E007242200C0
:10368000D2B2072A0DD022009D682E6A36F070064D
:103690001700FFB23F0117F070073E432E6201276B
:1036A00038000A78002A01D0012200E000229D683B
:1036B0006E6836F020061700FFB27F0117F0200772
:1036C0003E436E60C0B2F0BC70477CB504000D0094
:1036D000002600200090A0684068C0F38010C0B2AF
:1036E000002817D069462000FFF7BEFB0600300017
:1036F000C0B200280ED0A068016B11F007010120B4
:103700008840412804D20099B1FBF0F0286001E024
:1037100000210E003000C0B276BDF0B403000020DE
:1037200000229C68656835F040051600F6B2B601C7
:1037300016F04006354365608E88012E01D10024C5
:103740001EE08A88022A01D1012419E08A88042A0D
:1037500001D1022414E08A88082A01D103240FE051
:103760008A88102A01D104240AE08A88202A01D1FB
:10377000052405E08A88402A01D1062400E00724B8
:103780002200D2B2072A0CD022009D682E6BF608C8
:10379000F6001700FFB217F007073E432E6301271C
:1037A00038000A78002A01D0012200E000229D683A
:1037B0006E6836F040061700FFB2BF0117F04007F1
:1037C0003E436E60C0B2F0BC70477CB504000D0093
:1037D000002600200090A0684068C0F3C010C0B26E
:1037E000002817D069462000FFF73EFB0600300096
:1037F000C0B200280ED0A068006BC0F302110120F7
:103800008840412804D20099B1FBF0F0286001E023
:1038100000210E003000C0B276BDF0B403000020DD
:1038200000229C68656835F080051600F6B2F60146
:1038300016F08006354365608E88012E01D1002484
:103840001EE08A88022A01D1012419E08A88042A0C
:1038500001D1022414E08A88082A01D103240FE050
:103860008A88102A01D104240AE08A88202A01D1FA
:10387000052405E08A88402A01D1062400E00724B7
:103880002200D2B2072A0DD022009D682E6B36F09E
:1038900070061700FFB23F0117F070073E432E631A
:1038A000012738000A78002A01D0012200E0002216
:1038B0009D686E6836F080061700FFB2FF0117F0B2
:1038C00080073E436E60C0B2F0BC70477CB5040018
:1038D0000D00002600200090A0684068000A10F04B
:1038E0000100C0B2002817D069462000FFF7A6FBF0
:1038F00006003000C0B200280ED0A068016C11F0A4
:10390000070101208840412804D20099B1FBF0F062
:10391000286001E000210E003000C0B276BDF0B496
:103920000300002000229C68656835F4807516004D
:10393000F6B2360216F48076354365608E88012E25
:1039400001D100241EE08A88022A01D1012419E055
:103950008A88042A01D1022414E08A88082A01D125
:1039600003240FE08A88102A01D104240AE08A88FF
:10397000202A01D1052405E08A88402A01D10624A5
:1039800000E007242200D2B2072A0CD022009D6852
:103990002E6CF608F6001700FFB217F007073E433B
:1039A0002E64012738000A78002A01D0012200E0A5
:1039B00000229D686E6836F480761700FFB23F02E1
:1039C00017F480773E436E60C0B2F0BC70477CB5A0
:1039D00004000D00002600200090A0684068400A06
:1039E00010F00100C0B2002817D069462000FFF790
:1039F00025FB06003000C0B200280ED0A068006C85
:103A0000C0F3021101208840412804D20099B1FB83
:103A1000F0F0286001E000210E003000C0B276BD59
:103A2000F0B40300002000229C68656835F400753E
:103A30001600F6B2760216F40076354365608E887D
:103A4000012E01D100241EE08A88022A01D101241E
:103A500019E08A88042A01D1022414E08A88082AFD
:103A600001D103240FE08A88102A01D104240AE03E
:103A70008A88202A01D1052405E08A88402A01D1BC
:103A8000062400E007242200D2B2072A0DD022002B
:103A90009D682E6C36F070061700FFB23F0117F0DC
:103AA00070073E432E64012738000A78002A01D0AF
:103AB000012200E000229D686E6836F4007617004F
:103AC000FFB27F0217F400773E436E60C0B2F0BCD5
:103AD000704770B504000D0000262068C068C0F370
:103AE0000110C0B2002805D002280FD008D3032847
:103AF00012D017E029002000FFF7B6F9060011E008
:103B000029002000FFF7ECF906000BE02900200057
:103B1000FFF794FA060005E029002000FFF754FAA9
:103B20000600FFE73000C0B270BD70B402004878F4
:103B3000022801D100230FE04878002801D1012399
:103B40000AE04878032801D1022305E048780128DB
:103B500001D1032300E0FF231800C0B2FF2801D1E8
:103B6000002014E0180014682569AD08AD000600B7
:103B7000F6B216F00306354325611068C068C0F33D
:103B800001101C00C0B2E4B2A042F6D1012070BC0A
:103B900070477CB504000D00002669462000FFF741
:103BA00098FF01000800C0B2002801D100200BE0FE
:103BB00020680069C0F30310009AC0B2401CB2FB39
:103BC000F0F028600800C0B276BD30B402008888EA
:103BD000002811D0888811280EDA8888431E1468BE
:103BE000256935F0F0051800C0B2000110F0F000B2
:103BF00005432561012000E0002030BC70477CB502
:103C000004000D00002669462000FFF7C2FF0100F6
:103C10000800C0B2002801D100200CE0A0680068B4
:103C2000000A10F00F00009AC0B2401CB2FBF0F086
:103C300028600800C0B276BD30B402008888002831
:103C400011D0888811280EDA8888431E9468256868
:103C500035F470651800C0B2000210F470600543BE
:103C60002560012000E0002030BC70477CB50400D6
:103C70000D00002669462000FFF78BFF01000800B9
:103C8000C0B2002801D1002015E0E068006910F002
:103C90000100C0B200280AD0A068006810F01F0020
:103CA000009AC0B2401CB2FBF0F0286001E0002096
:103CB00001000800C0B276BD30B402008888002838
:103CC00020D0888809281DDA8888431E94682568D2
:103CD0006D096D011800C0B210F01F00054325608A
:103CE0000878002801D0012300E00023D46825696A
:103CF0006D086D001800C0B210F001000543256189
:103D0000012000E0002030BC70477CB504000D00AD
:103D1000002669462000FFF73CFF01000800C0B202
:103D2000002801D1002016E0A068406810F00100D2
:103D3000C0B200280BD0A0680068000F10F0070088
:103D4000009AC0B2401CB2FBF0F0286001E00020F5
:103D500001000800C0B276BD70B40300002000244A
:103D60009D686E68760876002200D2B212F00102D9
:103D700016436E608A88002A11D08A88092A0EDAD2
:103D80008A88521E9C68256835F0E0451600F6B218
:103D9000360716F0E04635432560012630000A78E4
:103DA000002A01D0012200E000229C6865686D08AD
:103DB0006D001600F6B216F0010635436560C0B21C
:103DC00070BC70477CB504000D00A0684068C0F36B
:103DD0004000C0B2002801D100209AE00026002057
:103DE0000090A0688068C0F30210C0B2002843D1E0
:103DF000A068806810F00700C0B200280BD002282D
:103E000015D00ED304281ED017D3062827D020D3D0
:103E100007282AD02FE069462000FFF727FF060079
:103E200066E069462000FFF75BF8060060E069463F
:103E30002000FFF7C9F806005AE069462000FFF7A6
:103E400013F8060054E069462000FFF7F7F8060073
:103E50004EE069462000FFF79CFE060048E06946F8
:103E60002000FFF7CCFE060042E069462000FFF785
:103E7000ACFC06003CE03BE0A0688068C0F30210A8
:103E8000C0B201280AD033D3032813D00CD305289D
:103E90001CD015D3072825D01ED329E06946200061
:103EA000FFF791FA060023E069462000FFF78FFD37
:103EB00006001DE069462000FFF786FB060017E0BC
:103EC0006946200000F0EAF9060011E0694620008A
:103ED00000F0BFF906000BE06946200000F094F9FD
:103EE000060005E06946200000F0DEF90600FFE765
:103EF0003000C0B201280AD1A0688068000A10F022
:103F000007000099C0B2401CB1FBF0F028603000FF
:103F1000C0B276BDF0B503000A00012000219C6804
:103F2000656835F002050E00F6B2760016F002065E
:103F3000354365605678002E39D0012E55D0022EBB
:103F400071D0032E00F08D80052E00F00281072E27
:103F500000F01981092E00F0DE800B2E00F00681A2
:103F60000D2E00F09C800E2E00F0B7800F2E40F03A
:103F7000178100219C68A56835F070050E00F6B227
:103F8000360116F070063543A56000269F68D7F805
:103F900008C05FEADC0C5FEACC0CB6465FFA8EFE26
:103FA0001EF0070E5EEA0C0CC7F808C0FAE000210C
:103FB0009C68A56835F070050E00F6B2360116F063
:103FC00070063543A56001269F68D7F808C05FEAF0
:103FD000DC0C5FEACC0CB6465FFA8EFE1EF0070ED4
:103FE0005EEA0C0CC7F808C0DCE000219C68A568FC
:103FF00035F070050E00F6B2360116F07006354346
:10400000A56002269F68D7F808C05FEADC0C5FEA6B
:10401000CC0CB6465FFA8EFE1EF0070E5EEA0C0C64
:10402000C7F808C0BEE000219C68A56835F070059F
:104030000E00F6B2360116F070063543A560032671
:104040009F68D7F808C05FEADC0C5FEACC0CB64684
:104050005FFA8EFE1EF0070E5EEA0C0CC7F808C071
:10406000A0E000219C68A56835F070050E00F6B24E
:10407000360116F070063543A56004269F68D7F810
:1040800008C05FEADC0C5FEACC0CB6465FFA8EFE35
:104090001EF0070E5EEA0C0CC7F808C082E0002193
:1040A0009C68A56835F070050E00F6B2360116F072
:1040B00070063543A56005269F68D7F808C05FEAFB
:1040C000DC0C5FEACC0CB6465FFA8EFE1EF0070EE3
:1040D0005EEA0C0CC7F808C064E000219C68A56883
:1040E00035F070050E00F6B2360116F07006354355
:1040F000A56006269F68D7F808C05FEADC0C5FEA77
:10410000CC0CB6465FFA8EFE1EF0070E5EEA0C0C73
:10411000C7F808C046E000219C68A56835F0700526
:104120000E00F6B2360116F070063543A56007267C
:104130009F68D7F808C05FEADC0C5FEACC0CB64693
:104140005FFA8EFE1EF0070E5EEA0C0CC7F808C080
:1041500028E001219C68A56835F070050E00F6B2D4
:10416000360116F070063543A5601BE002219C68FD
:10417000A56835F070050E00F6B2360116F070062F
:104180003543A5600EE003219C68A56835F07005F5
:104190000E00F6B2360116F070063543A56001E058
:1041A000002108000100C9B2002915D0918800291A
:1041B00010D0918809290DDA9188491E9C68A5685C
:1041C00035F4E0650E00F6B2360216F4E0663543CB
:1041D000A56001E0002108001178002901D001212B
:1041E00000E000219C68656835F002050E00F6B21B
:1041F000760016F0020635436560C0B2F0BD0200DD
:10420000D069086001207047020050684068C0F320
:10421000C000C0B2002804D04FF47A7008600120BA
:1042200000E00020704730B402000878002801D078
:10423000012300E000235468656835F00805180084
:10424000C0B2C00010F0080005436560012030BC1A
:104250007047020050684068C0F30010C0B20028E8
:1042600004D04FF4FA400860012000E000207047BD
:1042700030B402000878002801D0012300E00023B8
:104280005468656835F010051800C0B2000110F0E0
:10429000100005436560012030BC704702005FF4E8
:1042A000FA3008600120704770B504000D00002648
:1042B00060684068C0F34000C0B2002801D100200F
:1042C0001AE060680068C0F30010C0B2002805D191
:1042D00029002000FFF7BDFF06000BE060680068C2
:1042E000C0F30010C0B2012804D129002000FFF75C
:1042F00086FF06003000C0B270BD70B4030000201D
:1043000000245D686E6836F002062200D2B25200C8
:1043100012F0020216436E600A78002A01D00122D0
:1043200000E000225C68656835F002051600F6B210
:10433000760016F0020635436560C0B270BC704767
:1043400070B504000D00002660680068000B10F0D6
:104350000100C0B2002805D129002000FFF74FFC62
:1043600006000CE060680068000B10F00100C0B2AD
:10437000012804D15FF4FA302860012006003000E3
:10438000C0B270BD70B4020000204B780E2B0DD16E
:1043900000235468256835F480551E00F6B23603B4
:1043A00016F480563543256001263000C0B270BC3B
:1043B000704770B504000D00002660684068C0F3C7
:1043C0008010C0B2002801D100202EE06068006893
:1043D000400B10F00700C0B2002806D0022810D011
:1043E00009D3042819D012D31DE029002000FFF7BB
:1043F000ECF9060017E029002000FEF7E4FF0600B4
:1044000011E029002000FFF7E2FA06000BE0290086
:104410002000FFF7D9F8060005E05FF4FA302860C5
:1044200001200600FFE73000C0B270BD70B4030089
:10443000012000225C68656835F040051600F6B280
:10444000B60116F04006354365604E78052E13D050
:10445000072E2BD0092E02D00B2E1AD033E00022CB
:104460005C68256835F460451600F6B2760316F4EC
:1044700060463543256028E001225C68256835F4F4
:1044800060451600F6B2760316F4604635432560A3
:104490001BE002225C68256835F460451600F6B220
:1044A000760316F46046354325600EE003225C680F
:1044B000256835F460451600F6B2760316F46046BA
:1044C0003543256001E0002210000A78002A01D05F
:1044D000012200E000225C68656835F040051600A6
:1044E000F6B2B60116F0400635436560C0B270BC46
:1044F00070477CB504000D00002600200090606825
:104500004068C0F38000C0B2002801D1002054E010
:1045100060680068000C10F00700C0B200280BD0E3
:10452000022815D00ED304281ED017D3062827D072
:1045300020D307282AD02FE069462000FFF745F94D
:10454000060029E069462000FEF73DFF060023E053
:1045500069462000FFF73BFA06001DE0694620008F
:10456000FFF732F8060017E069462000FFF796FED5
:10457000060011E069462000FFF746FE06000BE04A
:1045800069462000FFF765FE060005E06946200049
:10459000FFF735FE0600FFE73000C0B200280AD062
:1045A00060680068000D10F00700C0B2401C009960
:1045B000B1FBF0F028603000C0B276BD70B40300EB
:1045C000012000225C68656835F004051600F6B22B
:1045D000B60016F00406354365604E78052E13D0FC
:1045E000072E2BD0092E02D00B2E1AD033E000223A
:1045F0005C68256835F4E0251600F6B2360416F43A
:10460000E0263543256028E001225C68256835F402
:10461000E0251600F6B2360416F4E0263543256090
:104620001BE002225C68256835F4E0251600F6B22E
:10463000360416F4E026354325600EE003225C685C
:10464000256835F4E0251600F6B2360416F4E026A7
:104650003543256001E0002210008A88002A10D02E
:104660008A88092A0DDA8A88521E5C68256835F422
:10467000E0051600F6B2360516F4E006354325606F
:1046800001E0002210000A78002A01D0012200E097
:1046900000225C68656835F004051600F6B2B600C5
:1046A00016F0040635436560C0B270BC704770B543
:1046B00004000D0000266068406810F00100C0B2E0
:1046C000002801D100201AE060680068C0F34010A3
:1046D000C0B2002805D129002000FFF7E5FD060043
:1046E0000BE060680068C0F34010C0B2012804D13C
:1046F00029002000FFF788FD06003000C0B270BD21
:1047000070B40300002000245D686E6876087600AF
:104710002200D2B212F0010216436E600A78002A1B
:1047200001D0012200E000225C6865686D086D0020
:104730001600F6B216F0010635436560C0B270BCD3
:10474000704770B504000D00002660680068000E18
:1047500010F00100C0B2002805D129002000FFF7A9
:104760004EFA06000CE060680068000E10F00100D0
:10477000C0B2012804D129002000FFF78FFD0600F8
:104780003000C0B270BD70B4020000204B780E2B18
:104790000BD100235468256835F080751E00F6B2F1
:1047A000360616F0807635432560C0B270BC70477F
:1047B00070B504000D00002660680068400E10F01F
:1047C0000100C0B2002805D129002000FFF717FA28
:1047D00006000CE060680068400E10F00100C0B2F6
:1047E000012804D129002000FFF758FD0600300001
:1047F000C0B270BD70B4020000204B780E2B0BD1FC
:1048000000235468256835F000751E00F6B2760660
:1048100016F0007635432560C0B270BC704770B5A5
:1048200004000D00002660680068800E10F0010092
:10483000C0B2002805D129002000FFF7E0F90600EA
:104840000CE060680068800E10F00100C0B2012822
:1048500004D129002000FFF721FD06003000C0B27E
:1048600070BD70B4020000204B780E2B0BD10023DA
:104870005468256835F080651E00F6B2B60616F05D
:10488000806635432560C0B270BC704770B50400C7
:104890000D00002660680068C00E10F00100C0B274
:1048A000002805D129002000FFF7A9F906000CE037
:1048B00060680068C00E10F00100C0B2012804D189
:1048C00029002000FFF7EAFC06003000C0B270BDEE
:1048D00070B4020000204B780E2B0BD100235468DB
:1048E000256835F000651E00F6B2F60616F0006683
:1048F00035432560C0B270BC704770B504000D0030
:10490000002660680068000F10F00100C0B20028A7
:1049100005D129002000FFF772F906000CE060685D
:104920000068000F10F00100C0B2012804D1290076
:104930002000FFF7B3FC06003000C0B270BD70B4B9
:10494000020000204B780E2B0BD100235468256801
:1049500035F080551E00F6B2360716F08056354306
:104960002560C0B270BC704770B504000D00002611
:1049700060684068000A10F00100C0B2002804D04E
:1049800029002000FFF73BF906003000C0B270BDDF
:1049900030B402000878002801D0012300E0002391
:1049A0005468656835F480751800C0B2000210F4D0
:1049B000807005436560012030BC704770B504000D
:1049C0000D00002660684068400A10F00100C0B287
:1049D000002804D029002000FFF711F9060030005C
:1049E000C0B270BD30B402000878002801D00123A5
:1049F00000E000235468656835F400751800C0B203
:104A0000400210F4007005436560012030BC70471F
:104A100070B504000D00002660684068800A10F040
:104A20000100C0B2002804D029002000FFF7E7F8F9
:104A300006003000C0B270BD30B402000878002813
:104A400001D0012300E000235468656835F48065D7
:104A50001800C0B2800210F4806005436560012038
:104A600030BC704770B504000D00002660684068D7
:104A7000C00A10F00100C0B2002804D029002000B4
:104A8000FFF7BDF806003000C0B270BD30B40200C0
:104A90000878002801D0012300E0002354686568ED
:104AA00035F400651800C0B2C00210F40060054380
:104AB0006560012030BC704770B504000D00002611
:104AC00060684068000B10F00100C0B2002804D0FC
:104AD00029002000FFF793F806003000C0B270BD37
:104AE00030B402000878002801D0012300E0002340
:104AF0005468656835F480551800C0B2000310F49E
:104B0000805005436560012030BC704738B5040013
:104B10000D00E0680069C0F34000C0B2002801D178
:104B2000002003E029002000FFF733F832BD30B445
:104B300002000878002801D0012300E00023D46897
:104B4000256935F002051800C0B2400010F00200DF
:104B500005432561012030BC704738B504000D00C5
:104B6000E0680069C0F38000C0B2002801D10020D5
:104B700003E029002000FFF70CF832BD30B402003A
:104B80000878002801D0012300E00023D4682569BB
:104B900035F004051800C0B2800010F00400054391
:104BA0002561012030BC704738B504000D00E06875
:104BB0000069C0F3C000C0B2002801D1002003E0AA
:104BC00029002000FEF7E5FF32BD30B4020008786E
:104BD000002801D0012300E00023D468256935F0C6
:104BE00008051800C0B2C00010F008000543256198
:104BF000012030BC704738B504000D00E068006942
:104C0000C0F34010C0B2002801D1002003E0290009
:104C10002000FEF7BEFF32BD30B402000878002845
:104C200001D0012300E00023D468256935F0200578
:104C30001800C0B2400110F020000543256101209A
:104C400030BC704738B504000D00E0680069000F03
:104C500010F00100C0B2002801D1002003E02900BB
:104C60002000FEF796FF32BD30B40200087800281D
:104C700001D0012300E00023D468256935F0805578
:104C80001800C0B2000710F08050054325610120D4
:104C900030BC704738B504000D00E0680069400F73
:104CA00010F00100C0B2002801D1002003E029006B
:104CB0002000FEF76EFF32BD30B4020008780028F5
:104CC00001D0012300E00023D468256935F00055A8
:104CD0001800C0B2400710F00050054325610120C4
:104CE00030BC704738B504000D00E0680069800FE3
:104CF00010F00100C0B2002801D1002003E029001B
:104D00002000FEF77CFF32BD30B402000878002896
:104D100001D0012300E00023D468256935F08045E7
:104D20001800C0B2800710F08040054325610120C3
:104D300030BC704738B504000D00E0684069800E53
:104D400010F00100C0B2002801D1002003E02900CA
:104D50002000FEF7C5F832BD30B402000878002804
:104D600001D0012300E00023D468656935F0806537
:104D70001800C0B2800610F0806005436561012014
:104D800030BC704738B504000D00E0684069000E83
:104D900010F00100C0B2002801D1002003E029007A
:104DA0002000FEF761F832BD30B402000878002818
:104DB00001D0012300E00023D468656935F08075D7
:104DC0001800C0B2000610F0807005436561012034
:104DD00030BC704738B504000D00E0684069C00E73
:104DE00010F00100C0B2002801D1002003E029002A
:104DF0002000FEF739F832BD30B4020008780028F0
:104E000001D0012300E00023D468656935F0006516
:104E10001800C0B2C00610F00060054365610120B3
:104E200030BC704738B504000D00E0684069400EA2
:104E300010F00100C0B2002801D1002003E02900D9
:104E40002000FEF7FBF832BD30B4020008780028DD
:104E500001D0012300E00023D468656935F00075B6
:104E60001800C0B2400610F00070054365610120D3
:104E700030BC704770B504000D00E0680069400E5A
:104E800010F00100C0B2002801D1002023E001266B
:104E9000E068006810F00300C0B2002805D00228C6
:104EA0000DD007D303280FD013E029002000FEF710
:104EB0008CFC0FE029002000FEF785FA0AE02900AB
:104EC0002000FEF784FD05E029002000FEF77CFBB2
:104ED00000E00020C0B270BDF0B40300002000224A
:104EE000DC68256935F000751600F6B2760616F016
:104EF0000076354325614E78092E01D100240FE05C
:104F00004A78052A01D101240AE04A780B2A01D106
:104F1000022405E04A78072A01D1032400E0FF2497
:104F20002200D2B2FF2A0CD02200DD682E68B6081B
:104F3000B6001700FFB217F003073E432E600127AB
:104F400038000A78002A01D0012200E00022DD6842
:104F50002E6936F000761700FFB27F0617F0007753
:104F60003E432E61C0B2F0BC704770B504000D0026
:104F7000E0680069400C10F00100C0B2002801D1C7
:104F8000002024E00126E0680068000D10F0030016
:104F9000C0B2002805D002280DD007D303280FD0B7
:104FA00013E029002000FEF710FC0FE0290020008C
:104FB000FEF709FA0AE029002000FEF708FD05E0E7
:104FC00029002000FEF700FB00E00020C0B270BD09
:104FD000F0B4030000200022DC68256935F40035B8
:104FE0001600F6B2760416F40036354325614E7885
:104FF000092E01D100240FE04A78052A01D10124AD
:105000000AE04A780B2A01D1022405E04A78072AEF
:1050100001D1032400E0FF242200D2B2FF2A0DD0E8
:105020002200DD682E6836F440161700FFB23F05F7
:1050300017F440173E432E60012738000A78002AF3
:1050400001D0012200E00022DD682E6936F400362E
:105050001700FFB27F0417F400373E432E61C0B241
:10506000F0BC704770B504000D00E0680069800C6A
:1050700010F00100C0B2002801D1002024E0012678
:10508000E0680068800D10F00300C0B2002805D071
:1050900002280DD007D303280FD013E029002000E9
:1050A000FEF793FB0FE029002000FEF78CF90AE0E1
:1050B00029002000FEF78BFC05E029002000FEF708
:1050C00083FA00E00020C0B270BDF0B403000020FD
:1050D0000022DC68256935F480251600F6B2B60496
:1050E00016F48026354325614E78092E01D100241F
:1050F0000FE04A78052A01D101240AE04A780B2AF8
:1051000001D1022405E04A78072A01D1032400E0F6
:10511000FF242200D2B2FF2A0DD02200DD682E68C3
:1051200036F440061700FFB2BF0517F440073E43B0
:105130002E60012738000A78002A01D0012200E001
:105140000022DD682E6936F480261700FFB2BF0406
:1051500017F480273E432E61C0B2F0BC704770B593
:1051600004000D00E0680069C00C10F00100C0B23E
:10517000002801D1002024E00126E0680068000E2C
:1051800010F00300C0B2002805D002280DD007D3CC
:1051900003280FD013E029002000FEF716FB0FE0D4
:1051A00029002000FEF70FF90AE029002000FEF791
:1051B0000EFC05E029002000FEF706FA00E00020C2
:1051C000C0B270BDF0B4030000200022DC68256985
:1051D00035F400251600F6B2F60416F40026354321
:1051E00025614E78092E01D100240FE04A78052A66
:1051F00001D101240AE04A780B2A01D1022405E0FA
:105200004A78072A01D1032400E0FF242200D2B209
:10521000FF2A0DD02200DD682E6836F04076170098
:10522000FFB23F0617F040773E432E60012738005B
:105230000A78002A01D0012200E00022DD682E69F0
:1052400036F400261700FFB2FF0417F400273E4390
:105250002E61C0B2F0BC7047F0B4049C059D0160A3
:1052600042608360C4602E6806616E684661AE6805
:105270008661EE68C661002600273E00F6B2032E66
:105280000DD23E00F6B205EB86063669BC465FFAE3
:105290008CFC00EB8C0CCCF820607F1CEDE7F0BCA4
:1052A0007047F8B504000E0015003000C0B2342875
:1052B00001DB002011E00027354A3000C0B252F86F
:1052C0003000002807D0290020003300DBB252F85C
:1052D0003320904707003800C0B2F2BD2DE9F64FE9
:1052E00085B083460C002000C0B2342801DB0020CA
:1052F0004AE00025264A2000C0B202EBC000406808
:1053000000283FD0234EDBF80070C7F88060DFF83C
:105310008880DBF8040004900498C0F84080DFF82F
:105320007C90DBF80C0003900398C0F84090DFF805
:1053300070A0DBF8080002900298C0F880A00699DF
:1053400058462300DBB202EBC302526890470500C7
:105350000020DBF80010C1F880000022DBF80430E8
:105360000193019B1A640023DBF80CE0CDF800E008
:10537000DDF800C0CCF840305FF0000CDBF808E04E
:10538000CEF880C02800C0B207B0BDE8F08F0000A2
:10539000A8C30000E42386FA9C1FC5C1777563701B
:1053A000656D4353BFF34F8FDFF8AC110A6812F4F9
:1053B000E062DFF8A80102430A60BFF34F8F00BF2D
:1053C000FDE70160426083607047020000200B002F
:1053D000DBB20E2B01DBC0B2BCE00B00DBB2002B5A
:1053E00017D0022B2BD01FD3042B3ED032D3062B49
:1053F00051D045D3082B64D058D30A2B79D06CD325
:105400000C2B00F08E80C0F080800D2B00F095807A
:105410009FE013685B6813F00103DBB2012B01D13D
:10542000012000E0002094E013685B68C3F34003B0
:10543000DBB2012B01D1012000E0002089E01368DC
:105440005B68C3F38003DBB2012B01D1012000E0D4
:1054500000207EE013685B68C3F3C003DBB2012B5E
:1054600001D1012000E0002073E013685B68C3F302
:105470000013DBB2012B01D1012000E0002068E025
:1054800013685B68C3F34013DBB2012B01D1012029
:1054900000E000205DE013685B68C3F38013DBB2BB
:1054A000012B01D1012000E0002052E013685B686D
:1054B000C3F3C013DBB2012B01D1012000E00020B7
:1054C00047E013685B681B0A13F00103DBB2012B92
:1054D00001D1012000E000203BE013685B685B0A1B
:1054E00013F00103DBB2012B01D1012000E0002009
:1054F0002FE013685B689B0A13F00103DBB2012BFA
:1055000001D1012000E0002023E013685B68DB0A82
:1055100013F00103DBB2012B01D1012000E00020D8
:1055200017E013685B681B0B13F00103DBB2012B60
:1055300001D1012000E000200BE013685B685B0BE9
:1055400013F00103DBB2012B01D1012000E00020A8
:10555000FFE7C0B2704700000CED00E00400FA0560
:10556000F8B504000D00DFF8A40CA1680864DFF8AA
:10557000A02C63681A642E00F6B2002E00F08C8016
:10558000022E00F0AD80C0F09980042E00F0CC8097
:10559000C0F0B880062E00F0EB80C0F0D780082E57
:1055A00000F00A81C0F0F6800A2E00F03181C0F0D0
:1055B00015810C2E00F06681C0F047810E2E00F0A0
:1055C0009B81C0F07C81102E00F0D081C0F0B181B1
:1055D000122E00F00582C0F0E681142E00F0388211
:1055E000C0F01A82162E00F06B82C0F04D82182E89
:1055F00000F09E82C0F080821A2E00F0D182C0F0AE
:10560000B3821C2E00F00483C0F0E6821E2E00F050
:105610003783C0F01983202E00F06A83C0F04C83DA
:10562000222E00F09D83C0F07F83242E00F0D083D3
:10563000C0F0B283262E00F00384C0F0E583282E4C
:1056400000F03684C0F018842A2E00F06984C0F07F
:105650004B842C2E00F09C84C0F07E842E2E00F013
:10566000CF84C0F0B184302E00F00285C0F0E48415
:10567000322E00F03585C0F01785342E00F0688595
:10568000C0F04A85362E00F09B85C0F07D85372E10
:1056900000F0B28500F0B3BD0120A1680200D2B2D3
:1056A000520012F002028A600022A3681600F6B2CD
:1056B000760016F002069E6000F0A1BD0120A168F0
:1056C0000200D2B2920012F004028A600022A368A3
:1056D0001600F6B2B60016F004069E6000F08FBD0C
:1056E0000120A1680200D2B2520112F020028A60A9
:1056F0000022A3681600F6B2760116F020069E601E
:1057000000F07DBD0120A1680200D2B2920112F02A
:1057100040028A600022A3681600F6B2B60116F0B5
:1057200040069E6000F06BBD0120A1680200D2B26D
:10573000120212F480728A600022A3681600F6B288
:10574000360216F480769E6000F059BD0120A168F3
:105750000200D2B2520212F400728A600022A368E0
:105760001600F6B2760216F400769E6000F047BD91
:105770000120A1680200D2B2920212F480628A6013
:105780000022A3681600F6B2B60216F480669E6088
:1057900000F035BD0120A1680200D2B2D20212F49D
:1057A00000628A600022A3681600F6B2F60216F4C0
:1057B00000669E6000F023BD0120A1680200D2B205
:1057C000120312F480528A600022A3681600F6B217
:1057D000360316F480569E6000F011BD012061680A
:1057E0000A6A520852000300DBB213F001031A43A5
:1057F0000A6200236668376A7F087F009C465FFA6A
:105800008CFC1CF0010C5CEA0707376200F0F7BC67
:10581000012061680A6A32F002020300DBB25B0019
:1058200013F002031A430A6200236668376A37F0EE
:1058300002079C465FFA8CFC5FEA4C0C1CF0020CE1
:105840005CEA0707376200F0DABC012061680A6A87
:1058500032F004020300DBB29B0013F004031A438E
:105860000A6200236668376A37F004079C465FFACD
:105870008CFC5FEA8C0C1CF0040C5CEA07073762B6
:1058800000F0BDBC012061680A6A32F00802030022
:10589000DBB2DB0013F008031A430A6200236668D8
:1058A000376A37F008079C465FFA8CFC5FEACC0C3D
:1058B0001CF0080C5CEA0707376200F0A0BC01206E
:1058C00061680A6A32F010020300DBB21B0113F0B8
:1058D00010031A430A6200236668376A37F010071C
:1058E0009C465FFA8CFC5FEA0C1C1CF0100C5CEA16
:1058F0000707376200F083BC012061680A6A32F052
:1059000020020300DBB25B0113F020031A430A629A
:1059100000236668376A37F020079C465FFA8CFCE4
:105920005FEA4C1C1CF0200C5CEA0707376200F0B1
:1059300066BC012061680A6A32F040020300DBB2F3
:105940009B0113F040031A430A6200236668376A1A
:1059500037F040079C465FFA8CFC5FEA8C1C1CF019
:10596000400C5CEA0707376200F049BC012061681F
:105970000A6A32F480720300DBB21B0213F48073F4
:105980001A430A6200236668376A37F480779C46B8
:105990005FFA8CFC5FEA0C2C1CF4807C5CEA070745
:1059A000376200F02CBC012061680A6A32F4007290
:1059B0000300DBB25B0213F400731A430A62002394
:1059C0006668376A37F400779C465FFA8CFC5FEABA
:1059D0004C2C1CF4007C5CEA0707376200F00FBC1B
:1059E000012061680A6A32F480620300DBB29B0224
:1059F00013F480631A430A6200236668376A37F437
:105A000080679C465FFA8CFC5FEA8C2C1CF4806CEF
:105A10005CEA07073762F2E3012061680A6A32F440
:105A200000620300DBB2DB0213F400631A430A6274
:105A300000236668376A37F400679C465FFA8CFC7F
:105A40005FEACC2C1CF4006C5CEA07073762D6E3F3
:105A5000012061680A6A32F480520300DBB21B0342
:105A600013F480531A430A6200236668376A37F4D6
:105A700080579C465FFA8CFC5FEA0C3C1CF4805C0F
:105A80005CEA07073762BAE3012061680A6A32F408
:105A900000520300DBB25B0313F400531A430A62A3
:105AA00000236668376A37F400579C465FFA8CFC1F
:105AB0005FEA4C3C1CF4005C5CEA070737629EE33B
:105AC000012061680A6A32F480420300DBB29B0362
:105AD00013F480431A430A6200236668376A37F476
:105AE00080479C465FFA8CFC5FEA8C3C1CF4804C3F
:105AF0005CEA0707376282E3012061680A6A32F4D0
:105B000000420300DBB2DB0313F400431A430A62D2
:105B100000236668376A37F400479C465FFA8CFCBE
:105B20005FEACC3C1CF4004C5CEA0707376266E392
:105B3000012061680A6A32F480320300DBB21B0480
:105B400013F480331A430A6200236668376A37F415
:105B500080379C465FFA8CFC5FEA0C4C1CF4803C5E
:105B60005CEA070737624AE3012061680A6A32F497
:105B700000320300DBB25B0413F400331A430A6201
:105B800000236668376A37F400379C465FFA8CFC5E
:105B90005FEA4C4C1CF4003C5CEA070737622EE3DA
:105BA000012061680A6A32F480220300DBB29B04A0
:105BB00013F480231A430A6200236668376A37F4B5
:105BC00080279C465FFA8CFC5FEA8C4C1CF4802C8E
:105BD0005CEA0707376212E3012061680A6A32F45F
:105BE00000220300DBB2DB0413F400231A430A6231
:105BF00000236668376A37F400279C465FFA8CFCFE
:105C00005FEACC4C1CF4002C5CEA07073762F6E232
:105C1000012061680A6A32F480120300DBB21B05BE
:105C200013F480131A430A6200236668376A37F454
:105C300080179C465FFA8CFC5FEA0C5C1CF4801CAD
:105C40005CEA07073762DAE2012061680A6A32F427
:105C500000120300DBB25B0513F400131A430A625F
:105C600000236668376A37F400179C465FFA8CFC9D
:105C70005FEA4C5C1CF4001C5CEA07073762BEE27A
:105C8000012061680A6A32F480020300DBB29B05DE
:105C900013F480031A430A6200236668376A37F4F4
:105CA00080079C465FFA8CFC5FEA8C5C1CF4800CDD
:105CB0005CEA07073762A2E2012061680A6A32F4EF
:105CC00000020300DBB2DB0513F400031A430A628F
:105CD00000236668376A37F400079C465FFA8CFC3D
:105CE0005FEACC5C1CF4000C5CEA0707376286E2D2
:105CF000012061680A6A32F080720300DBB21B0681
:105D000013F080731A430A6200236668376A37F01B
:105D100080779C465FFA8CFC5FEA0C6C1CF0807C00
:105D20005CEA070737626AE2012061680A6A32F0BA
:105D300000720300DBB25B0613F000731A430A62C1
:105D400000236668376A37F000779C465FFA8CFC60
:105D50005FEA4C6C1CF0007C5CEA070737624EE29D
:105D6000012061680A6A32F080620300DBB29B06A0
:105D700013F080631A430A6200236668376A37F0BB
:105D800080679C465FFA8CFC5FEA8C6C1CF0806C30
:105D90005CEA0707376232E2012061680A6A32F082
:105DA00000620300DBB2DB0613F000631A430A62F1
:105DB00000236668376A37F000679C465FFA8CFC00
:105DC0005FEACC6C1CF0006C5CEA0707376216E2F5
:105DD000012061680A6A32F080520300DBB21B07BF
:105DE00013F080531A430A6200236668376A37F05B
:105DF00080579C465FFA8CFC5FEA0C7C1CF0805C50
:105E00005CEA07073762FAE1012061680A6A32F04A
:105E100000520300DBB25B0713F000531A430A621F
:105E200000236668376A37F000579C465FFA8CFC9F
:105E30005FEA4C7C1CF0005C5CEA07073762DEE13D
:105E4000012061680A6A32F080420300DBB29B07DE
:105E500013F080431A430A6200236668376A37F0FA
:105E600080479C465FFA8CFC5FEA8C7C1CF0804C7F
:105E70005CEA07073762C2E1012061684A6A32F0D2
:105E800004020300DBB29B0013F004031A434A62CE
:105E900000236668776A37F004079C465FFA8CFC3B
:105EA0005FEA8C0C1CF0040C5CEA07077762A6E141
:105EB000012061684A6A32F008020300DBB2DB00AD
:105EC00013F008031A434A6200236668776A37F0C2
:105ED00008079C465FFA8CFC5FEACC0C1CF0080CAF
:105EE0005CEA070777628AE1012061684A6A32F05A
:105EF00010020300DBB21B0113F010031A434A62C5
:105F000000236668776A37F010079C465FFA8CFCBE
:105F10005FEA0C1C1CF0100C5CEA070777626EE16C
:105F2000012061684A6A32F020020300DBB25B01A3
:105F300013F020031A434A6200236668776A37F039
:105F400020079C465FFA8CFC5FEA4C1C1CF0200C7E
:105F50005CEA0707776252E1012061684A6A32F021
:105F600040020300DBB29B0113F040031A434A6274
:105F700000236668776A37F040079C465FFA8CFC1E
:105F80005FEA8C1C1CF0400C5CEA0707776236E184
:105F9000012061684A6A32F080020300DBB2DB0153
:105FA00013F080031A434A6200236668776A37F069
:105FB00080079C465FFA8CFC5FEACC1C1CF0800CCE
:105FC0005CEA070777621AE1012061684A6A32F4E5
:105FD00080620300DBB29B0213F480631A434A62BF
:105FE00000236668776A37F480679C465FFA8CFC0A
:105FF0005FEA8C2C1CF4806C5CEA07077762FEE099
:10600000012061684A6A32F400620300DBB2DB02FD
:1060100013F400631A434A6200236668776A37F410
:1060200000679C465FFA8CFC5FEACC2C1CF4006C89
:106030005CEA07077762E2E0012061684A6A32F4AD
:1060400080520300DBB21B0313F480531A434A62ED
:1060500000236668776A37F480579C465FFA8CFCA9
:106060005FEA0C3C1CF4805C5CEA07077762C6E0E0
:10607000012061684A6A32F400520300DBB25B031C
:1060800013F400531A434A6200236668776A37F4B0
:1060900000579C465FFA8CFC5FEA4C3C1CF4005CA9
:1060A0005CEA07077762AAE0012061684A6A32F475
:1060B00080420300DBB29B0313F480431A434A621D
:1060C00000236668776A37F480479C465FFA8CFC49
:1060D0005FEA8C3C1CF4804C5CEA070777628EE038
:1060E000012061684A6A32F480120300DBB21B05AA
:1060F00013F480131A434A6200236668776A37F400
:1061000080179C465FFA8CFC5FEA0C5C1CF4801CD8
:106110005CEA0707776272E0012061684A6A32F040
:1061200080720300DBB21B0613F080731A434A62CD
:1061300000236668776A37F080779C465FFA8CFCAC
:106140005FEA0C6C1CF0807C5CEA0707776256E023
:10615000012061684A6A32F000720300DBB25B061C
:1061600013F000731A434A6200236668776A37F0B7
:1061700000779C465FFA8CFC5FEA4C6C1CF0007C5C
:106180005CEA070777623AE0012061684A6A32F008
:1061900080620300DBB29B0613F080631A434A62FD
:1061A00000236668776A37F080679C465FFA8CFC4C
:1061B0005FEA8C6C1CF0806C5CEA070777621EE07B
:1061C000012061684A6A32F000620300DBB2DB063C
:1061D00013F000631A434A6200236668776A37F057
:1061E00000679C465FFA8CFC5FEACC6C1CF0006C8C
:1061F0005CEA0707776202E0FFF7D4F8FFE70020C8
:10620000A1680864002263681A64F1BD9C1FC5C1BF
:10621000777563702DE9F04798B004005FF00008CF
:106220005FF000095FF0000A0025002600274022E9
:10623000002108A800F0E5FD6846DFF8A01620223E
:1062400000F0FAFD082140F20112002003008C4604
:10625000DBB25FFA8CFC634514D25FF0FF330DF1C3
:10626000200C86465FFA8EFE4CF83E3000230DF17E
:10627000200C86465FFA8EFE0CEBCE0CACF8043098
:10628000401CE3E7002318008C46C0B25FFA8CFC88
:10629000604553D202200600300080B2824247D3CC
:1062A0002068EC469E465FFA8EFE5CF82EC0B0FB7E
:1062B000FCF0B4461FFA8CFCB0FBFCF005006068F3
:1062C000854218D108A89C465FFA8CFC00EBCC00F4
:1062D000868008A89C465FFA8CFC00EBCC0083719A
:1062E00000200DF1200C9E465FFA8EFE4CF83E0019
:1062F000012007001CE06068854217D208A89C4670
:106300005FFA8CFC00EBCC00868008A89C465FFA04
:106310008CFC00EBCC0083716068401B0DF1200CFD
:106320009E465FFA8EFE4CF83E0001E0761CB3E715
:106330003800C0B2002801D15B1CA4E75FF0000C5C
:1063400008A8E6465FFA8EFE50F83EE05FF00108CE
:1063500043468946DBB25FFA89F94B450ED2434684
:10636000DBB250F83330734505D24346DBB250F808
:1063700033309E46C44618F10108E9E708ABE14610
:106380005FFA89F903EBC9039B88022B15DA2068B1
:106390006B4689465FFA89F903EB890353F8043C9D
:1063A000B0FBF3F0B0FBF2F005000800C0B2401EF5
:1063B000A060901EE060256118E008ABE1465FFA3E
:1063C00089F903EBC9039B79A36008ABE1465FFA47
:1063D00089F903EBC9039B889B1EE3606368E14670
:1063E0005FFA89F950F839001B1A236118B0BDE82B
:1063F000F0872DE9F04F87B004000D0000200090D9
:106400005FF000085FF000092000006E009000219E
:10641000684600F0D4FC0021684600F0C3FC697BAC
:10642000684600F08FFC697A684600F06AFCA97A39
:10643000684600F05DFC686803902868029002A836
:10644000FFF7E8FE049E059FBA46A346DBF840101E
:10645000090A09025046C0B2014301910198CBF8E4
:1064600040003100C9B2684600F056FCE889411E80
:1064700089B2684600F0BBFCA87B800604D5E97EA3
:10648000684600F06AFC03E00021684600F065FC05
:10649000E97A684600F04BFC687D002805D00228A8
:1064A00029D010D303283ED04BE00021684600F0ED
:1064B00093FCE97F684600F075FC95F8201068466B
:1064C00000F07DFC4AE00121684600F06BFC0021F1
:1064D000684600F074FC287C002804D1002168463E
:1064E00000F07AFC06E0287C012803D101216846EF
:1064F00000F072FC32E0287C002804D100216846BC
:1065000000F06AFC06E0287C012803D101216846DE
:1065100000F062FC0121684600F044FC002168465E
:1065200000F04DFC1AE00021684600F055FCE97FC0
:10653000684600F037FC95F82010684600F03FFCF4
:106540000CE00021684600F047FCE97F684600F057
:1065500029FC95F82010684600F031FC0098206670
:1065600007B0BDE8F08FF0B40D7A03005C6A2A0032
:10657000D2B2012A03D154F001025A6202E0620849
:1065800052005A620E7B91F90B2096400200576A26
:1065900037F47067B4465FFA8CFC5FEA0C2C1CF48D
:1065A000706C5CEA07075762F0BC70472DE9FF4F3B
:1065B000030092F800C01E00F7696046C0B20128CF
:1065C00003D157F00100F06102E078084000F0616B
:1065D00050781C00E56986465FFA8EFEBEF1010F19
:1065E00003D155F00206E66102E035F00206E661ED
:1065F00096781F00D7F824C0B6465FFA8EFEBEF12B
:10660000010F03D15CF00800786202E03CF0080062
:106610007862D0781C00256A86465FFA8EFEBEF14D
:10662000010F03D155F48076266202E035F48076BE
:1066300026621F000026D7F824C05FEACC7C01D573
:1066400001200600F6B2002E0DD155791800446ADB
:106650002E00F6B2012E03D154F00406466202E089
:1066600034F004064662D7791D002E693800C0B2A6
:10667000012803D156F00400286102E036F004003E
:10668000286190798DF80100180004699DF801C017
:10669000BCF1010F03D154F00805056102E034F0AC
:1066A000080505614D788DF800500193019D2D6C12
:1066B00035F47F459DF8006055EA06250395039D56
:1066C000019E35648D781E00376C37F47F07AC4629
:1066D0005FFA8CFC57EA0C470297029F3764CF7829
:1066E0009C46DCF840E02EF07F4EB8465FFA88F812
:1066F0005EEA086ECCF840E091F804809946D9F83B
:1067000024A03AF0700AC3465FFA8BFB5FEA0B1BCA
:106710001BF0700B5BEA0A0AC9F824A091F805B0D7
:10672000BBF1000F07D0BBF1020F3ED028D3BBF165
:10673000030F4FD073E08879002801D0012000E0DA
:1067400000201C00656A0600F6B2002E03D055F04A
:106750008066666202E035F08066666200261F0091
:10676000D7F824C03CF0407CB6465FFA8EFE5FEA64
:106770000E6E1EF0407E5EEA0C0CC7F824C072E07C
:1067800001201C00656A35F040750600F6B2360639
:1067900016F040763543656201261F00D7F824C005
:1067A0005CF0806EC7F824E05DE002201C00656AA2
:1067B00035F040750600F6B2360616F040763543E1
:1067C000656201261F00D7F824C05CF0806EC7F810
:1067D00024E048E08879002801D0012000E0002072
:1067E0001C00656A0600F6B2002E03D055F08066E4
:1067F000666202E035F08066666203261F00D7F805
:1068000024C03CF0407CB6465FFA8EFE5FEA0E6E16
:106810001EF0407E5EEA0C0CC7F824C023E08879A5
:10682000002801D0012000E000201C00656A06005D
:10683000F6B2002E03D055F08066666202E035F0B5
:106840008066666200261F00D7F824C03CF0407CBA
:10685000B6465FFA8EFE5FEA0E6E1EF0407E5EEA7E
:106860000C0CC7F824C0BDE8FF8FDFF8841301606B
:10687000DFF8801341600121017200214172002183
:1068800081720021C172002101730121417308212D
:10689000C1810021C17500210176002141760021CE
:1068A00081760021C1760021017700214177002106
:1068B000C177002180F82010002181770221017426
:1068C0000A2141740A2181740A21C17400210175D1
:1068D000002141750021817570470000D4CF000070
:1068E0002DE9F84F84B004000D00002627683869B0
:1068F00003900398400840003861D4F80080D8F82D
:1069000010000290029850F48070C8F81000D4F87B
:106910000090D9F810000190019850F40070C9F867
:10692000100000BF00BF00BF29002068FFF71BFE5A
:1069300015F1170215F110012068FFF737FE5FF01F
:10694000010AD4F800B0DBF810000090009850F075
:106950000100CBF8100029002068FFF74AFD05B0C0
:10696000BDE8F08F2DE9F04101600268136953F42E
:10697000807414610468256955F400762661012647
:106980000768D7F810C05CF0020EC7F810E000BF2F
:1069900000BF00BF5FF0000ED0F80080C8F810E024
:1069A000BDE8F08170B40300002000220C00012C2F
:1069B00014D0022C1AD0B4F5807F1FD0B4F5007F1C
:1069C00025D0B4F5806F2BD0B4F5006F31D0B4F57D
:1069D000805F37D0B4F1807F3DD045E01C68002552
:1069E000666916F00106F6B232003DE01C6800252B
:1069F0006669C6F34006F6B2320035E01C68002531
:106A00006669360A16F00106F6B232002CE01C6800
:106A100000256669760A16F00106F6B2320023E018
:106A20001C6800256669B60A16F00106F6B2320047
:106A30001AE01C6800256669F60A16F00106F6B22F
:106A4000320011E01C6800256669360B16F001065D
:106A5000F6B2320008E01C6800256669360E16F0B2
:106A60000106F6B23200FFE7002A01D0012420001F
:106A7000C0B270BC70472DE9FE4F04000D00160037
:106A80001F00DDF830805FF001090020216800223E
:106A9000CB6D13F01F03D3F110038DF804303300D6
:106AA0009DF804C09BB21FFA8CFC634580F099806E
:106AB000002000905FF0000B0020ADF80600206879
:106AC000006E00900021684600F061F901216846DF
:106AD00000F050F90021684600F071F90021684685
:106AE00000F060F92900C9B2C900491E89B26846A0
:106AF00000F07DF90098216808665FF0000A5046B2
:106B0000310080B289B288425FD220680021426998
:106B100012F00102D2B2002A07D11BF1010B40F2A0
:106B2000E9308345F1D3002081462800C0B2012816
:106B300005D1504680B2385C2168486610E02800D4
:106B4000C0B2022806D1504680B237F81000216842
:106B5000486605E0504680B257F820002168486634
:106B60000020834622680021106FC0F340000028F7
:106B700001D001200100C9B2002907D01BF1010B8F
:106B800040F2E9308345EDD3002081462800C0B2B1
:106B9000012806D12068406F514689B208F80100EB
:106BA00010E02800C0B2022806D12068406F51468C
:106BB00089B228F8110005E02068406F514689B27B
:106BC00048F821001AF1010A99E70021684600F00F
:106BD000DEF80021684600F0CDF8009821680866CC
:106BE00001E0002081464846C0B2BDE8FE8F0000AB
:106BF000000E270740420F0070B4020000200B0077
:106C0000012B11D0022B1AD0B3F5807F22D0B3F51F
:106C1000007F2BD0B3F5806F34D0B3F5006F3DD03B
:106C2000B3F5805F46D051E0012415680023AE69BA
:106C30002640A64201D101263300180046E0022476
:106C400015680023AE692640A64201D10126330013
:106C500018003BE04FF4807415680023AE692640AD
:106C6000A64201D10126330018002FE04FF4007432
:106C700015680023AE692640A64201D101263300E3
:106C8000180023E04FF4806415680023AE692640A5
:106C9000A64201D101263300180017E04FF400642A
:106CA00015680023AE692640A64201D101263300B3
:106CB00018000BE04FF4805415680023AE6926409D
:106CC000A64201D1012633001800FFE7C0B270BC14
:106CD000704730B40A0003689C6D34F4F814150052
:106CE000EDB22D0415F4F8152C439C6530BC7047AB
:106CF000026822F000420B00DBB252EAC37202606B
:106D00007047026832F080420B00DBB29B0713F041
:106D100080431A4302607047026832F060520B00F1
:106D2000DBB2DB0613F060531A430260704702685F
:106D300032F040720B00DBB21B0613F040731A43B3
:106D400002607047026832F400020B00DBB2DB0520
:106D500013F400031A430260704702680B00DBB2B1
:106D6000012B03D152F48003036002E032F480036C
:106D70000360704702680B00DBB2012B03D152F4B1
:106D80000013036002E032F40013036070470268EE
:106D900032F480120B00DBB21B0513F480131A438C
:106DA0000260704702680B00DBB2012B03D152F482
:106DB0000023036002E032F400230360704702689E
:106DC0000B00DBB2012B03D152F48023036002E0FD
:106DD00032F4802303607047026832F440320B00C3
:106DE000DBB21B0413F440331A430260704702689D
:106DF000120B12030B009BB21B051B0D1A43026002
:106E0000704710B5044610460A460146204600F079
:106E100057F8204610BDFEE762B38B0708D0521E1C
:106E200011F8013B00F8013B00F024808B07F6D1FC
:106E3000830740F0208000BF103A07D330B4B1E898
:106E40003810103AA0E83810F9D230BC530724BFEC
:106E5000B1E80810A0E8081044BF51F8043B40F81E
:106E6000043BD20724BF31F8022B20F8022B44BF89
:106E70000B7803707047121F17D35B0009D151F8CC
:106E8000043B20F8023B1B0C121F20F8023BF6D2F9
:106E90000BE051F8043B00F8013B1B0A20F8023BD1
:106EA0001B0C121F00F8013BF3D238BF121D521EFB
:106EB00024BF11F8013B00F8013BF8D87047FEE70A
:106EC00062F30F2262F31F42401810F0030308D050
:106ED000C91A1FD3DB0748BF00F8012D28BF20F8CF
:106EE000022D130030B414461546103928BF20E98E
:106EF0003C00FAD8490728BF20E90C0048BF40F8F9
:106F0000042D890028BF20F8022D48BF00F8012D6C
:106F100030BC7047C91818BF00F8012DCB0728BF37
:106F200000F8012D7047FEE7010008000200D2B210
:106F3000802A01DB7F221000C0B2704701000800E8
:106F4000C0B2F12805DB0800C0B2FA2801DA01203E
:106F500006E00800C0B2802801DA080000E0002046
:106F6000C0B270472DE9FC4104000D0016001F005F
:106F70005FF000083F208DF800009DF8001055F0EC
:106F8000F00001408DF800108DF801603800C0B2AB
:106F9000FFF7CAFF8DF802002078002813D00320E5
:106FA00080464046C0B2082807DA002069464246BB
:106FB000D2B2885418F10108F3E708226946E06864
:106FC000A36D984704E003226946E068A36D9847E3
:106FD00040B2BDE8F6817CB50400002500200F21F9
:106FE0008DF800109DF80010E28A52F0F002114076
:106FF0008DF8001000263000C0B2E18A80B28842CD
:107000000AD220693100C9B2405C69463200D2B26E
:1070100011444870761CEEE72078002817D0002035
:1070200005002800C0B2E18AD1F10701884208DAE0
:107030006846E18A51FA85F10844CC2141706D1C03
:10704000EFE708226946E068A36D984706E0E28A08
:10705000521CD2B26946E068A36D984740B276BD33
:107060003EB504001F208DF800009DF80000E18A65
:1070700089B2090A51F0F00108408DF80000E08A59
:107080008DF80100002000252800C0B206280ADA89
:1070900020692900C9B2405C69462A00D2B2114475
:1070A00088706D1CF0E708226946E068A36D984778
:1070B000010049B2002904D1218B891D21830121BE
:1070C000A17640B23EBDFEB5040000212F208DF810
:1070D00000009DF80000A27E52F0F00210408DF8F2
:1070E0000000E58A208B2D1A280080B2082801DBD9
:1070F0000720050000263000C0B2290080B289B206
:1071000088420BD22069218B51FA86F1405C694696
:107110003200D2B211444870761CECE72078002887
:1071200019D0002000273800C0B2290089B2D1F15F
:107130000701884209DA6846290089B251FA87F1C5
:107140000844CC2141707F1CEDE708226946E068C5
:10715000A36D984705E06A1CD2B26946E068A36D4A
:107160009847010049B200290AD1218B691821836F
:10717000A17E491CA176A17E102901DB0021A17608
:1071800040B2FEBDF8B504000D00160000272878B7
:1071900010F00F0F07D03000C0B2401E297811F058
:1071A0000F01884208DA606D002802D0A448616DA2
:1071B00088477FF0060017E0287810F00F00A4F849
:1071C000420000210800C0B2B4F8422080B29042D0
:1071D00009D20800C0B228444078E26B0B00DBB251
:1071E000D054491CEEE70020F2BD2DE9F041040027
:1071F0000D00160000273000C0B2082808D0606DCE
:10720000002802D08F48616D88477FF006003AE081
:107210002878000210F47060697810EB010840468D
:1072200080B2082808DA606D002802D08648616DB7
:1072300088477FF0060026E0B4F84000414689B256
:10724000884208D2606D002802D08048616D88476E
:107250007FF0020017E0A4F8428000210800C0B2CD
:10726000062809DA0800C0B228448078E26B0B00D7
:10727000DBB2D054491CF1E70620A4F844000120F9
:1072800084F846000020BDE8F0812DE9F0410400BB
:107290000D001600002794F84600297811F00F0120
:1072A000884202D07FF0030042E0B4F84280B4F894
:1072B0004400B8EB0008404680B2082801DB0720F4
:1072C00080463000C0B2401E414689B2884208DA8A
:1072D000606D002802D05E48616D88477FF006002F
:1072E00026E000210800C0B2424680B292B290422D
:1072F0000BD2E06BB4F8442052FA81F20B00DBB2FF
:107300002B445B788354491CECE7B4F8440018EB39
:107310000000A4F8440094F84600401C84F846009D
:1073200094F84600102802DB002084F84600002074
:10733000BDE8F08170B504000D0016003000C0B249
:10734000032808DA606D002802D04248616D884742
:107350007FF0060000E0002070BD70B504000D0055
:10736000160033009BB22A00E168200000F001F80B
:1073700070BD2DE9F8430400894615001E005FF03A
:107380000008002C02D15FF0FF3056E0A08A3100E7
:1073900089B2884208D2606D002802D02E48616D03
:1073A00088477FF0020048E094F83400012808D1B3
:1073B000606D002802D02948616D88477FF0010088
:1073C0003BE0E6820020208300273800C0B2310075
:1073D00080B289B2884208D23800C0B2285C2169E4
:1073E0003A00D2B288547F1CEFE7E08A082804DA1A
:1073F0002000FFF7F0FD80461DE02000FFF730FE83
:107400008046404640B2002815D10020A0830020CD
:10741000A0770020E077E06D8047C4E90801E06DC7
:107420008047643051F10001C4E90A010020206363
:10743000012084F83400404640B2BDE8F2830000E9
:10744000F4CE000020CF0000ECCD000024CE0000E0
:1074500094CF0000B4CF00005CCE000090CE0000BE
:107460002DE9FE4304000D0091461E003000C0B21D
:10747000022803DB3000C0B2092800DB2AE100202B
:10748000002108003200C0B2D2B2904209D20800F6
:10749000C0B219F800006A460B00DBB2D054491C98
:1074A000EFE75FF000084046C0B23100C9B2D1F149
:1074B0000801884209DA002069463200D2B252FA45
:1074C00088F2885418F10108EDE79DF80000C0B279
:1074D0000009002806D0022861D01FD3032800F03D
:1074E000AB80F7E094F85100012804D17FF005004B
:1074F00084F8500002E0002084F850003200D2B23C
:1075000069462000FFF73EFE0700380040B2002821
:1075100003D1A563022084F85100DBE094F8510008
:10752000012804D17FF0050084F8500002E000201B
:1075300084F850003200D2B269462000FFF755FEB1
:10754000070038007FF0020140B288420DD17FF081
:10755000070084F85000002084F851000023002226
:1075600002212000FFF7FEFCB4E0380040B2002802
:1075700014D1A563012084F85100607884F8470095
:10758000012394F8472000212000FFF7EBFCE06D79
:107590008047643051F10001C4E912019AE094F887
:1075A0005100012804D07FF0050084F8500091E0DC
:1075B000A06B854240F08E803200D2B26946200036
:1075C000FFF763FE07007FF003003900020049B2B5
:1075D000914205D184F85000002084F8510079E0F0
:1075E000380040B2002826D1E06D8047643051F168
:1075F0000001C4E91201B4F84400B4F84210884212
:1076000003D3022084F8510015E06078002812D0DE
:1076100094F84700401E84F8470094F8470000287B
:1076200009D1607884F84700012394F847200021AD
:107630002000FFF797FC4DE094F83400012849D171
:107640003200D2B269462000FFF774FE070038000E
:1076500040B200283DD1E06D8047643051F1000117
:10766000C4E90A019DF8000010F00F00022806D1BD
:107670007FF007002063022084F8340029E09DF8A1
:10768000000010F00F0001280CD1E07F401CE077D3
:10769000E07F02281DDB7FF006002063022084F8D3
:1076A000340016E09DF8000010F00F0F11D19DF886
:1076B0000100002803D14FF6FF70A08302E09DF87F
:1076C0000100A0839DF80200FFF738FCA07700209E
:1076D000E077FFE7BDE8F783F0B40400049D0026DF
:1076E00094F85100022802D07FF0040028E0A06B3B
:1076F000A768B84201D1012000E000200870B4F86A
:1077000042701800BC4680B21FFA8CFC604500D263
:107710001F005FF0000C60463E0080B2B6B2B0427F
:1077200009D2E06B6646B6B2805D6646B6B2905549
:107730001CF1010CEFE72F80002084F8510000209D
:10774000F0BC70470A7802704A7842704A6842601A
:107750008A688260CA68C2600A6902618A8A828213
:107760000022C282002202830022827600228283CB
:10777000002282770022C27700220023C0E908237A
:1077800000220023C0E90A2300220263002280F8BD
:1077900034208A69C2638A8BA0F840200022A0F8B6
:1077A00042200022A0F84420002280F84620002237
:1077B00080F8472000220023C0E91223002280F82D
:1077C0005020002280F851200A6A42654A6A826588
:1077D0008A6AC265704770B5040094F834000128C5
:1077E0004DD14FF6FF76A08BB04202D0A08B00287F
:1077F00036D0A07F00280BD0A07F002830D0E06DCD
:107800008047D4E90823101A73EB0101002927D51A
:107810002000FFF758FC0500280040B200281CD1CA
:10782000A08BB04202D0A08B401EA083E06D8047A9
:10783000643051F10001C4E90A01E06D8047A27F84
:10784000002380185941C4E90801208BE18A88424D
:1078500006D3002084F8340002E0022084F83400CB
:10786000E06D8047D4E90A23101A73EB0101002967
:1078700005D57FF001002063022084F8340094F8DD
:10788000510001280FD1E06D8047D4E91223101A6E
:1078900073EB0101002906D57FF0020084F8500047
:1078A000002084F8510070BD10B4020012B2002A0A
:1078B00006D40A01DFF81438040024B21A5509E08E
:1078C0000A01DFF80C38040024B214F00F0423443A
:1078D00003F8042C10BC704710B50400601EB0F112
:1078E000807F01D3012011E0601EDFF8E8170860F7
:1078F0000F215FF0FF30FFF7D7FF0020DFF8D81728
:1079000008600720DFF8D4170860002010BD0022AF
:107910000260416001220272002242727047017AC5
:1079200000290FD0417A00290CD1016842689142A8
:1079300008D20168491C016001684268914201D186
:1079400001214172704770B504000D001600B4F8B3
:107950008C1804F6A800FFF7DAFF94F878000128E5
:1079600006D0320092B2290014F11800FFF7F5FC9E
:1079700070BDFEB504000D001600082100226F4600
:107980003800FFF79DFA3000C0B2782805D0B4F86F
:107990008C1804F6A800FFF7BAFF94F879000028C5
:1079A00014D03000C0B211280FD03000C0B212285D
:1079B0000BD03000C0B2312807D03000C0B27E28D2
:1079C00003D03000C0B27F2800D10CE07F208DF8BA
:1079D00000008DF801508DF802600322694614F111
:1079E0001800FFF7BAFCF7BD10B5040014F50860E5
:1079F000D0E90001401C71F1FF3114F50862C2E9C1
:107A0000000114F50960FFF78AFF04F69C00FFF7F8
:107A100086FF04F6A800FFF782FF10BDDFF8C0065E
:107A2000D0E90001704780B5DFF8B8060168491C4D
:107A30000160DFF8AC06D0E90023521C73F1FF337C
:107A4000C0E90023DFF8A006FFF7CEFF01BD2DE956
:107A5000F04794B0DFF894465FF080512068FBF760
:107A60002EF8012843D12068FBF778F82068FBF74F
:107A700066F800283BD1DFF878562068FBF77DF8E0
:107A800028702878002832D069462068FBF77EF8F5
:107A90009DF8485002AE4C274FF49858DFF85496A2
:107AA00019F808007843484410F1040A2A0031000C
:107AB0005046FFF7B1F919F808007843019949F8E1
:107AC000001019F8080007FB00F709EB07009DF804
:107AD000481080F8441019F80800401C09F8080004
:107AE00019F80800202802D3002009F808005FF0E8
:107AF00000512068FAF7E3FF012804D15FF000513C
:107B00002068FAF7BFFF5FF080412068FAF7D7FFDF
:107B1000012804D15FF080412068FAF7B3FF5FF0DD
:107B200000412068FAF7CBFF012804D15FF0004143
:107B30002068FAF7A7FF14B0BDE8F0872DE9F047F9
:107B40000400002541F20136DFF8A87517F59850BA
:107B50000078B95D884216D05FF04C08B95D4C20C2
:107B6000414307EB0109A246424649465046FFF70A
:107B700053F9B85D401CB855B85D202801D30020EA
:107B8000B855012005002800C0B2BDE8F0872DE9F6
:107B9000F84F94B004000D001600002700205FF09D
:107BA0000008DFF85415404691F84920C0B29042D1
:107BB0000ED2CA6C4346DBB21420434302EB0300EF
:107BC0004068844201D1474602E018F10108E8E725
:107BD0001420CA6C3B00DBB24343D25A8DF800201C
:107BE0008DF84860C96C3A00D2B200FB02F008443C
:107BF00040680190B1465FFA89F9AA460DF1080B79
:107C00004A4651465846FFF707F9DFF8E0B469469F
:107C1000DBF80000FAF759FC6946DBF80000FAF7D8
:107C200047FC002015B0BDE8F08F7FB50020029022
:107C3000DFF8B844DFF8C85415F19800206015F556
:107C4000A07601220121300000F0FEFA012201217C
:107C5000300000F02EFB00220121300000F038FB44
:107C600015F5A47601220721300000F0EDFA01227B
:107C70000721300000F01DFB00220721300000F03A
:107C800027FB15F5987605220021300000F0DCFA7C
:107C900005220121300000F0D7FADFF85C640120F2
:107CA0003070002070700020B07001203071002012
:107CB00086F83000012086F8440002AA0E2115F152
:107CC0001800FDF7EEFA707801280DD1012001901F
:107CD0004FF4FA60009041F64C53DFF828240299E3
:107CE00016F11C00FAF72EFD0020019040F6C4109A
:107CF000009041F64C53DFF81024029916F1080069
:107D0000FAF720FD31002068F9F74AFE01225FF002
:107D100080512068FAF732FE6F2000F01FFB7FBD14
:107D2000F0B4040020000025002696420BD2DFF8B4
:107D3000DC538F5D474007F0FF0755F8275095EA61
:107D40001020761CF1E71D00EDB2012D02D15FF08D
:107D5000FF35281AF0BC704738B50124DFF8B0535E
:107D60000D212800FDF731FB002815D10121280045
:107D7000FDF72BFB01280CD1DFF898030168DFF831
:107D80009823914202D00020040007E00021016006
:107D900004E00020040001E0002004002000C0B244
:107DA00032BDF8B50024002500F0CEFACF480068B7
:107DB000F8F718FE5FF480300668D8480768D8489E
:107DC0000760D8490E600A6882F30988096881F360
:107DD00008885FF48031D44A116000688047F1BDA3
:107DE000C1494870704780B500F0AEFA3721C848E5
:107DF000FDF7B6FB01BD80B50020009003230622ED
:107E0000C021012000F0E4FA01BD38B504000D00E6
:107E10002A0092B22100B448FFF795FD31BD38B574
:107E200004000D002A00D2B22100C9B2AE48FFF70B
:107E3000A0FD31BD10B504002000C0B2012802D160
:107E400000F076FA01E000F07FFA10BD2DE9F04F66
:107E50009BB00020009000F077FADFF8A482404643
:107E600000F08CFB18F5FC7000F050FC41F204307F
:107E70000790002006909F4D069A07992800FFF76B
:107E80001FF85FF080095FF0000A9B4E35005246F4
:107E900049462800FFF714F800F087FDA3490020A9
:107EA00000F0CBFF01208DF804000120ADF80800A0
:107EB00018F1180B01AA20215846FDF70FFA01AA64
:107EC00021215846FDF70AFA01AA22215846FDF75A
:107ED00005FA01AA23215846FDF700FA01AA242138
:107EE0005846FDF7FBF901208DF8040003208DF8BA
:107EF00005000120ADF8080001AA0B215846FDF746
:107F0000EDF901208DF804000B208DF8050001AA81
:107F100033215846FDF7E2F9050018F5F070006EC0
:107F2000009003216846FEF7F7FE00F095FF00F091
:107F300083FA3000F8F7EFFC042086F849007C480B
:107F4000F064FFF772FE18F59876012205213000E3
:107F500000F07AF901220521300000F0AAF902228E
:107F60000521300000F0F9F800220521300000F072
:107F7000AFF918F5A07601220721300000F064F96E
:107F800001220721300000F094F90122072130007E
:107F900000F09EF9674E01220221300000F054F9F2
:107FA00000220221300000F084F94F4F624938006E
:107FB00001F072F8614918F17C0001F0FBFADFF87A
:107FC000808142460C215846FDF76BF9D8F8000035
:107FD0004FF47A71B0FBF1F0FFF77EFC4FF6FF70C3
:107FE00000F0BCF900F0A4F9D8F8002055490020B1
:107FF00000F023FF3B49086800284DD000200860AE
:10800000DFF84481D8F80000401CC8F80000D8F818
:1080100000000A21B0FBF1F201FB1200002801D19F
:1080200000F0A4F90221300000F061F9002802D12B
:10803000012001F016FBD8F800004FF4FA71B0FBF4
:10804000F1F201FB120000280CD1032000F09CF992
:1080500005002B0022003D49002000F0EEFE641CCC
:1080600026480570D8F8000041F2883188420BD3C9
:108070000020C8F8000036490868002802D1012015
:10808000086001E000200860012001F087FB380053
:1080900001F057FC01F072FB08A8FFF74FFD012823
:1080A000A8D1089840F23271884204D0089840F272
:1080B000DF7188429ED19DF8643009AA089917F1B2
:1080C0001800FFF7CDF995E70000000000E400E09C
:1080D00018ED00E014E000E018E000E010E000E03F
:1080E000000000203413002008000020D0300020C1
:1080F000FE3500204C1D0020503000206C04FF1F76
:108100003811002080841E0020A1070060A5000017
:10811000BC120020F0EF002055AAAA55040001006F
:10812000D8300020D430002008ED00E090D00000CE
:108130004CCD0000701200203804FF1F4CCF00000F
:10814000401300203CD000003813002058D000001D
:108150003C1300200160426070472DE9F043202964
:1081600070D21300DBB2002B03D0022B47D023D3F5
:1081700068E000230C00056855F8246036F002061C
:108180001F00FFB27F0017F002073E4345F824604E
:1081900000278C46D0F800E05EF82C805FEA580893
:1081A0005FEA4808B9465FFA89F919F0010959EA06
:1081B00008084EF82C8045E001230C00056855F8AE
:1081C000246036F002061F00FFB27F0017F002079E
:1081D0003E4345F8246000278C46D0F800E05EF866
:1081E0002C805FEA58085FEA4808B9465FFA89F9C7
:1081F00019F0010959EA08084EF82C8022E0002302
:108200000C00056855F8246036F002061F00FFB226
:108210007F0017F002073E4345F8246001278C4693
:10822000D0F800E05EF82C805FEA58085FEA480862
:10823000B9465FFA89F919F0010959EA08084EF8B8
:108240002C80FFE7BDE8F083F0B413000C00056854
:1082500055F8246036F4E0661F00FFB23F0217F4C1
:10826000E0673E4345F824601700FFB2002F0FD1AE
:1082700001230C00056855F8246036F004061F0041
:10828000FFB2BF0017F004073E4345F824600EE03C
:1082900000230C00056855F8246036F004061F0022
:1082A000FFB2BF0017F004073E4345F82460F0BC5E
:1082B000704730B443685B6901248C40A3431400C9
:1082C000E4B28C4023431C0045686C6130BC7047AD
:1082D00030B443681B6801248C40A3431400E4B20B
:1082E0008C4023431C0045682C6030BC704710B4A0
:1082F000030000245868006901228A400240002AD5
:1083000001D1002000E00120C0B210BC7047FEE7A0
:10831000010009B2002909D4012210F01F018A408E
:108320000C4903001BB25B0941F823207047000091
:1083300009480168012906DB0168491E01600068DF
:10834000012800DA62B6704772B603480168491C1A
:108350000160704700E100E03411002010B5040016
:10836000200000B2FFF7D4FF10BDFEE71CB50320CC
:1083700000F00AF8040000222100C9B2032000F036
:108380000BF80090009816BD10B50400002114F001
:108390007F0000F086FD10BDF8B505000E0014004A
:1083A0003100C9B255F08000C0B200F07AFD07007C
:1083B000002C00D027808DF800502800C0B2FFF7B5
:1083C000E3FF70408DF801008DF802600098F2BD67
:1083D0002DE9FC4705000E00170098460A9C28006E
:1083E000C0B2FFF7D1FF8146002C01D0A4F8009065
:1083F000CA463AEA060A4046C0B2B84050EA0A0AFB
:108400005146C9B255F08000C0B200F04AFD8DF867
:1084100000504046C0B2B8408DF802002800C0B2FB
:10842000FFF7B2FF010031409DF8020048408DF88F
:1084300001000098BDE8F6872DE9F04F97B01521AF
:10844000152400250800C0B291EA10110800C0B23E
:1084500091EA90010800C0B291EA50018DF8041031
:108460009DF8040010F00100012801DB95200400B4
:108470005FF0000A5FF0000B504680B2C0088DF834
:1084800009005FEA4A108DF8080000208DF8070007
:1084900000265846C0088DF806005FEA4B108DF89C
:1084A000050000275FF0000803A833495022FEF7BB
:1084B000C3FC0DF10C0989F801409DF809008DF805
:1084C00035009DF808008DF837009DF807008DF8FD
:1084D00039008DF83B609DF806008DF83D009DF851
:1084E00005008DF83F008DF841708DF843808DF8C0
:1084F000575000F0B1FC00280AD000208DF8000091
:10850000FF208DF8010000208DF80200009830E077
:108510005FF0000A5046C0B219F81000002807D1D9
:1085200003A85146C9B200EB41004078002816D09C
:10853000002203A85146C9B200EB410041785046E1
:10854000C0B219F81000FFF727FF00909DF8010056
:10855000002801D000980CE01AF1010ADAE70020A7
:108560008DF8000000208DF8010000208DF8020039
:10857000009817B0BDE8F08F9CCD00002DE9F843BE
:108580008AB00400474803904748049005900020B3
:108590000690002007900020089000200990434D8D
:1085A000434E444FDFF8108103A80190CDF80080BE
:1085B0003B003200290014F11800FCF74DFE3F4942
:1085C00014F17C0001F028FA00208DF80800032047
:1085D0008DF80900DFF8E89002A80190CDF800902E
:1085E0003B004246374914F19800F8F787F901201B
:1085F0008DF8080002208DF8090002A80190CDF83E
:1086000000903B004246304914F1AC00F8F776F98F
:1086100002208DF8080001208DF8090002A80190C1
:10862000CDF800903B004246284914F1C000F8F70D
:1086300065F9274A274914F59470FFF78BFD264A00
:10864000264914F59870FFF785FD254A254914F54C
:108650009C70FFF77FFD244A244914F5A070FFF7B2
:1086600079FD234A234914F5A470FFF773FD2A000E
:10867000214914F5A87001F0FBF9330042461F4967
:1086800014F5C270FCF79DFE1D4914F5F070FEF75D
:1086900069F91C4914F5FC7000F036F80BB0BDE820
:1086A000F08300BF006CDC0200127A0000F8074083
:1086B00000FC074000E0064000F0064000000240D9
:1086C00000F005400080034000C00340000004406B
:1086D00000F00F400000064040F00F400010064040
:1086E00080F00F4000200640C0F00F4000300640F0
:1086F00000F10F400040064000D0074000F0074066
:1087000000E0024000A0074001607047016809686E
:10871000C1F340110A00D2B2012A1CD10E4A0368EB
:108720005A600268126832F0800203681A604FF6DD
:10873000FF7203689A6002681268D20A12F001029E
:10874000D2B2002AF7D102681268520A12F001026E
:10875000D2B2002AF7D0704720C528D910B5DFF86B
:1087600054420320206103206061DFF84C02A061C5
:10877000DFF84812E1614FF4806121620021A162BB
:10878000002161620021E1622066DFF83402606648
:108790001020A066002020670020E06600206067AF
:1087A00053A1E01D01F068F9BFF35F8FDFF81412E9
:1087B000200001F061F9BFF35F8F2020A071BFF3AB
:1087C0005F8F10BD2DE9FE4F05000E0014005FF015
:1087D0000008D5F80C9028690700B94503D2B7EB1B
:1087E0000900401E04E0A868B0EB09003818401EDC
:1087F000A968B1EB0901884201D2824603E0D5F8AD
:1088000008A0BAEB090AA24500D3A246686848440A
:108810000090CDF808A00196DDF800B0029A019909
:108820005846FEF7F9FA1AEB08085644B4EB0A0466
:108830001AEB0909A868814501D100208146BFF3E0
:108840005F8FC5F80C90002CC5D14046BDE8FE8F67
:108850002DE9F84F84B004000D001600E768D4F845
:108860000880B8EB070846450FD2606800EB07099F
:108870000196AA46CB46019A51465846FEF7CCFAD5
:10888000BFF35F8FF019E06021E0CDF800806068F1
:1088900038440190009803900295DDF80490039A03
:1088A00002994846FEF7B8FAB6EB08000090D4F8F3
:1088B00004900098019005EB080ACB46019A5146B6
:1088C0005846FEF7A9FABFF35F8F0098E06005B045
:1088D000BDE8F08F01000A69CB68934204D3886831
:1088E000401EC01A101801E0D01A401E7047000048
:1088F000525454002DE9F04704000D001600A8461C
:10890000DFF8B000182101FB04F1084410F1180A47
:10891000DAF81400002803D0022820D010D325E074
:108920005046FFF7D7FF0700B74202D25FF00009B9
:1089300005E0B146320041465046FFF789FF17E097
:108940005046FFF7C7FF0700B74201D2B94600E023
:10895000B1464A4641465046FFF77AFF08E03200EA
:1089600041465046FFF72EFF814601E05FF00009C7
:108970004846BDE8F0872DE9F04104000D001600DF
:10898000DFF830703878002801D1FFF7E7FEEFF309
:108990001188202080F31188320029002000FFF781
:1089A000A9FF88F31188BDE8F08180B5FFF7D6FEF6
:1089B00001BD0000DC300020C8D000008431002060
:1089C00084350020D4D0000070B504000D00A668E6
:1089D0006068711C884206D320688555701CA060B1
:1089E000E068401CE060A068616888420DD1A26820
:1089F00021682069FFF7BFFFA168884203D05FF0BC
:108A0000FF30E06001E00020A06070BD2DE9FE4F66
:108A10000700884691461E000C9CC24601255FF067
:108A2000010BCA4504D3BAFBF9FA1BF1010BF8E7B5
:108A3000B34500D2B3460D98C0071AD4002C18D005
:108A40000D98800705D5002E03D130208DF8000049
:108A500002E020208DF80000002C0AD0A34508D2A7
:108A6000641E9DF800103800FFF7AEFFF86800287C
:108A7000F2D5F868002830D4022E01D3761E05E026
:108A8000B8FBF5F001900198484502D309FB05F5C4
:108A9000F2E7B8FBF5F00190019805FB108810484B
:108AA0000199415C3800FFF78FFFF868002803D474
:108AB000B5FBF9F5002DECD10D98C0070DD5002CB4
:108AC0000BD0002C09D0A34507D2641E202138000A
:108AD000FFF77AFFF8680028F3D5BDE8F78F0000AC
:108AE000B8D000002DE9FE4F06000F0090461D0093
:108AF0000C9CDDF83490002F02D5D7F1000A00E07D
:108B0000BA465FF0010BC24504DB9AFBF8FA1BF191
:108B1000010BF8E7AB4500D2AB46002C05D0002F87
:108B200002D45FEA497000D5641E5FEA897001D5FE
:108B3000002D10D05FEAC9700DD4002C0BD0002C92
:108B400009D0A34507D2641E20213000FFF73CFF67
:108B5000F0680028F3D5F068002831D4002F05D53F
:108B60007F422D213000FFF72FFF06E05FEA4970BA
:108B700003D52B213000FFF727FFF06800281FD412
:108B800019F0030002280FD1002D0DD1002C0BD0BD
:108B9000002C09D0A34507D2641E30213000FFF716
:108BA00013FFF0680028F3D5F068002808D4CDF84A
:108BB000049000942B00424639003000FFF726FF56
:108BC000BDE8F78F2DE9F14F98B08946150007A849
:108BD00002904020039000200490189806900020F6
:108BE000059099F80000060019F101093000C0B2A3
:108BF000002800F00F813000C0B2252840F001812C
:108C0000002080460120040099F800000600300092
:108C1000C0B2232815D02B280ED02D2802D0302802
:108C200005D013E058F0010819F1010910E058F0DF
:108C3000020819F101090BE058F0040819F10109C3
:108C400006E058F0080819F1010901E000200400CD
:108C5000002CD9D10020824699F80000060030008F
:108C6000C0B2302803DB3000C0B23A2808DB002055
:108C7000070099F800100800C0B22E2820D109E0A2
:108C800019F101090A2000FB0AFA5AFA86FABAF128
:108C9000300AE1E719F1010999F800000100080024
:108CA000C0B2302803DB0800C0B23A2800DB07E07E
:108CB00019F101090A20474357FA81F7303FEBE7E2
:108CC00099F800603000C0B26C2803D03000C0B208
:108CD000682805D119F1010999F800000600F1E7AB
:108CE0003000C0B2252800F08480582841D0632885
:108CF0000AD0642817D0702868D073284CD0752803
:108D000024D0782835D079E0286828602868006861
:108D10002968091D29600400A3465946C9B202A862
:108D2000FFF752FE6AE02868286028680068296812
:108D3000091D29600400CDF80480CDF800A03B0097
:108D40000A22210002A8FFF7CDFE57E0286828601C
:108D5000286800682968091D29600400CDF804808E
:108D6000CDF800A03B000A22210002A8FFF74EFE2A
:108D700044E028682860286800682968091D29607F
:108D80000400CDF80480CDF800A03B0010222100A3
:108D900002A8FFF73BFE31E0286828602868D0F879
:108DA00000B02868001D28609BF8000006001BF139
:108DB000010B3000C0B2002807D03100C9B202A8B0
:108DC000FFF702FE05980028EED517E02868286016
:108DD000286800682968091D2960040000200190A6
:108DE0000820009008231022210002A8FFF70EFEA1
:108DF00004E0252102A8FFF7E7FDFFE719F10109CB
:108E000004E03100C9B202A8FFF7DEFD0598002892
:108E10007FF5E7AE059801280BDB0498002804D005
:108E2000049A07A91898FFF7A6FD05990498411818
:108E30000591059819B0BDE8F08F0CB438B5040061
:108E40000D0004A800906A4629002000FFF7BAFE32
:108E500032BC5DF80CFB000018B589B000F041F899
:108E60006846FDF702FD01208DF808008548019055
:108E700001208DF80900844C6A46332114F1180052
:108E8000FCF70FFA0028F6D014F5F07469462000BC
:108E9000FDF726FD00212000FDF71BFF00200AB092
:108EA00010BD7CB504000D00784B1C705D70784ED1
:108EB0000096022201217748FDF7DDFD307800029F
:108EC0007178084380B276BD10B5724C0221200043
:108ED000FDF768FD012803D102212000FDF78CFE7B
:108EE00010BD2DE9F04F8FB0674C14F59C7503222F
:108EF0000E212800FFF7A8F901208DF805000E26A5
:108F0000D4F838010790079850F8260030F0400058
:108F10009DF80510890111F0400108430E900E984C
:108F2000079941F8260001208DF804000E27D4F897
:108F300038010690069850F8270030F020009DF880
:108F40000410490111F0200108430D900D98069975
:108F500041F8270003220F212800FFF775F90120AF
:108F60008DF803005FF00F08D4F8380105900598DC
:108F700050F8280030F040009DF80310890111F0EE
:108F8000400108430C900C98059941F828000120F5
:108F90008DF802005FF00F09D4F8380104900498AE
:108FA00050F8290030F020009DF80210490111F01E
:108FB000200108430B900B98049941F829000322E3
:108FC00000212800FFF740F901208DF801005FF033
:108FD000000AD4F838010390039850F82A0030F0C2
:108FE00040009DF80110890111F0400108430A90EA
:108FF0000A98039941F82A0001208DF800005FF0DB
:10900000000BD4F838010290029850F82B0030F091
:1090100020009DF80010490111F02001084309903B
:109020000998029941F82B00032201212800FFF73B
:109030000BF901200121D4F8382152F8213033F006
:1090400040030500EDB2AD0115F040052B43089338
:10905000089B42F8213001250123D4F8384154F807
:1090600023C03CF0200CAE465FFA8EFE5FEA4E1E37
:109070001EF0200E5EEA0C0C44F823C00FB0BDE8D1
:10908000F08F000040420F0038110020943500207E
:10909000A03500201813002038B504000D00290069
:1090A000200000F016FC0548A0600548E0600F2095
:1090B0006060044820610620A08231BD7CCC0000A5
:1090C000C4CE0000DC05FF1F2DE9F04704000D00B1
:1090D00016004FF48067B0465FFA88F817F104096C
:1090E000AA46424649465046FDF796FEBDE8F0873F
:1090F00043780B7070472DE9F04704000D0016000F
:109100004FF48067B0465FFA88F817F12809AA463D
:10911000424649465046FDF77FFEBDE8F0872DE9FF
:10912000F84F04000D0016004FF480675FF00C0844
:1091300017F118000090A946424600994846FDF7ED
:109140006BFE5FF0080917F10C0A15F10C0B4A468B
:1091500051465846FDF760FE2020E872BDE8F18FC9
:109160002DE9F04704000D0016004FF48067B0466B
:109170005FFA88F8B946AA46424649465046FDF786
:109180004BFEBDE8F08730B400231C001500E4B2AC
:10919000EDB2AC4205D220241D00EDB24C555B1C53
:1091A000F3E730BC704700004FF40060704770B5C3
:1091B00040F674040025DFF820662A002100300004
:1091C000FDF77EFE70BDE0B576208DF80000DFF87B
:1091D000082692F82C008DF801000221684652689A
:1091E0005269904707BD38B5DFF8EC45002084F898
:1091F0006408DFF8E8050068C4F84408DFF8E00513
:109200000068C4F85008DFF8DC050068C4F85408AA
:10921000E069DFF8D41588420ED1206AB0F5805F8E
:109220000AD10123226A121FE1695FF0FF306568ED
:109230006D68A847C4F83008D4F83008DFF8AC15DA
:109240000968884212D1D4F84408C4F85808D4F800
:109250005008C4F85C08D4F85408C4F860082068C2
:10926000D4F858188847012084F8640831BD80B5C7
:10927000DFF86415487A00281AD191F838080128D7
:1092800003D091F83C0801280FD10020C1F86C08E8
:10929000002081F86408012081F83C08022048720F
:1092A000022049680969884702E0042000F0C7F9F4
:1092B00001BD2DE9F843DFF82045607A002802D08F
:1092C000607A01285BD16069002858D0A069616983
:1092D000884254D20025E66894F8680803282DD007
:1092E000002061680968884794F86408012808D15B
:1092F0000121E06810F50060D4F85C289047050073
:1093000001E0042005002800C0B2002805D1012199
:10931000E068D4F85C28904705002800C0B2002817
:1093200007D16169891E16F58050D4F85C289047F2
:10933000050001206168096888470AE04FF48057FA
:109340005FF00008DFF8A094424639004846FDF778
:10935000B7FD2800C0B2002808D1022060720020AA
:109360006061002020610020A06108E000206061B1
:10937000002020610020A061032000F060F9BDE81A
:10938000F1832DE9F041DFF8504494F835080128C5
:1093900061D1607A002802D0607A01285BD194F80C
:1093A0003608012857D1606A216A884253D20025C5
:1093B00094F8680803281AD0002061680968884773
:1093C00094F8640801280BD14FF4006214F12D01C8
:1093D000E069636A1818D4F860389847050001E01E
:1093E0000420050001206168096888470DE04FF4FA
:1093F000006614F12D07E069D4F8248018EB00080A
:10940000320039004046FDF707FD2800C0B20028B1
:1094100012D1606A10F500606062606A216A884259
:1094200005D3002084F835080220607201E0012095
:109430006072FFF7C8FE09E0002084F835080020BC
:10944000206200206062032000F0F9F8002084F818
:1094500036080020A062BDE8F081F8B5DFF8784357
:10946000607A002802D0607A012870D101206072F1
:1094700094F86808012803D094F8680800284DD1B2
:109480005FF482300068DFF86813884208D001205A
:1094900084F83C0802206072002084F8340856E00A
:1094A000DFF850030568DFF85003066806F17F46D1
:1094B00016F57F06B6F5E02F0FD244F20100864282
:1094C0000BD3012332005FF480315FF0FF30676817
:1094D0007F68B847C4F8300802E00020C4F83008BC
:1094E000D4F83008854208D0012084F83C080220D6
:1094F0006072002084F8340829E0012084F83408E0
:1095000094F83C08002803D1052000F098F81EE0EC
:10951000012084F83C080220607218E094F8680882
:10952000022814D094F86808032810D1FFF75BFED6
:1095300094F86408012805D1012084F83408022039
:10954000607204E0002084F8340802206072F1BDEB
:1095500070B5A14C607A002802D0607A012827D12A
:1095600094F83A0801280DD16068C5696068066AF8
:10957000FFF71DFE94F83B08012801D1B04717E022
:10958000A84715E0D4F86C0832280FD394F83C08AB
:1095900000280BD16068C468FFF707FA97490020DC
:1095A000FFF74BFCFFF703FEA04701E001206072CC
:1095B00070BD70472DE9F24F82B0040040F674068A
:1095C0000027854DA8463A0031004046FDF778FC5B
:1095D000029868604FF480585FF00009DFF808A235
:1095E000D3464A4641465846FDF76AFC2C600020A7
:1095F000C5F83008CAF8004068688068804785F878
:109600003C0895F83C08012817D10020C5F86C08E3
:109610000220696809698847082100226E463000E7
:10962000FDF74EFC50208DF8000002208DF801005F
:10963000022168466A6852699047BDE8F78F66491B
:1096400000224A7208720022C1F86C2870476248F2
:10965000007A70476048407A70475F4890F8340855
:1096600070475D4A92F83C1800290AD182F8380800
:109670000021C2F86C18012182F83C18002182F800
:109680006418022151727047534A82F8390882F8EF
:109690003B18002382F86438704738B504000D0089
:1096A0004D480561C460002180F83618002180F81B
:1096B0003518B4F5803F0BD1B5F5E02F08D1012165
:1096C00080F86818016901F2FF71C90A41610EE072
:1096D00045498C420BD141F201018D4207D2032151
:1096E00080F86818002180F8641802214161012087
:1096F000FFF7A5FF31BD38B504000D003648012144
:1097000080F83518002180F83618C4610562002100
:1097100041620220FFF793FF31BD70B403000025C2
:10972000002000240D00ADB2AC4208D22A4DAE6A32
:10973000A61935441E5D85F82D60641CF2E7264DA0
:10974000AE6A16FA81F6AE6285F82C20AE6AB6F5DE
:10975000006F04D3012685F8366801252800C0B2C1
:1097600070BC70471C480021417204210172002125
:1097700080F834180021C0F83018704780B51649B9
:10978000087A062809DA1E4A087A52F820000028CA
:1097900003D0087A52F82000804701BD10B50400BC
:1097A0000D49087A002802D0087A052805D1D1F899
:1097B0006C0850FA84F0C1F86C0891F83908012857
:1097C00008D1002081F83908012081F83A080520E5
:1097D000FFF735FF10BD0000C008002004F0FF1F98
:1097E00008F0FF1F0CF0FF1F00F0FF1FFCFFFF1F22
:1097F000DDCCBBAAFCFF0700F8FF0700A8D00000E3
:109800002004FF1F0021016000214160002101723E
:109810000021417270470022026041600122027201
:10982000002242727047407A7047FEB504000D0076
:109830001600082100226F463800FDF741FB30007A
:10984000C0B2782805D0B4F88C1804F6A800FFF749
:10985000E2FF94F87900002814D03000C0B211283B
:109860000FD03000C0B212280BD03000C0B2312867
:1098700007D03000C0B27E2803D03000C0B27F28AD
:1098800000D10CE07F208DF800008DF801508DF89C
:1098900002600322694614F11800FDF75EFDF7BD72
:1098A00010B4020000200023180080B25468A042C7
:1098B0000CD290681C00A4B210F834000C00E4B282
:1098C000A04201D1012002E05B1CEDE7002010BCAA
:1098D000704738B504000D00290014F11800FDF799
:1098E00031FF012060700020A070002084F8780013
:1098F0000020002114F50862C2E90001A88DA4F837
:109900008808E88DA4F88A08288EA4F88C0814F535
:109910000960FFF777FF04F69C00FFF773FF04F67A
:10992000A800FFF76FFF0020002140F602008142EF
:1099300006D2002004EB010282F87B00491CF4E708
:1099400031BD2DE9FC4104000020ADF804005FF0BA
:1099500000080025002614F11800FDF73CFF01A8BF
:10996000009040F6020314F17B0214F1790114F126
:109970001800FDF7B1FE0700380040B200283AD1C8
:1099800094F87B0005002900C9B22000FFF788FF8A
:1099900000282AD000200600606886422BD2A068EA
:1099A00010F836002900C9B288421CD1A06800EB2B
:1099B000C6008078002806D094F87C00C0B2C009A8
:1099C00084F8780002E0002084F8780084F87A6057
:1099D000BDF8042014F17B012000A36803EBC6034B
:1099E0005B68984707E0761CD6E711222900C9B2C8
:1099F0002000FFF71AFF04F6A800FFF714FF012864
:109A000007D1012060700020A07004F6A800FFF7C5
:109A1000F9FEBDE8F381000038B504000D002560B3
:109A2000200000F015F82075002060605FF4002031
:109A3000A0600648E060207D002803D05FF48030FD
:109A4000206102E05FF44030206131BD0000011070
:109A5000010000200A681268120D12F00102D2B251
:109A6000012A01D1012000E00020C0B270470000AF
:109A700001604260704700005FEA000C11F8012BA2
:109A800000F8012B12B111F8012BF9E7604670477D
:109A9000002202604160012202720022427270477D
:109AA00070B504000D001600B4F88C1804F6A80078
:109AB000FFF7EEFF94F87800012806D0320092B24A
:109AC000290014F11800FDF748FC70BDFEB5040034
:109AD0000D001600082100226F463800FDF7F0F94E
:109AE0003000C0B2782805D0B4F88C1804F6A8006D
:109AF000FFF7CEFF94F87900002814D03000C0B2F0
:109B000011280FD03000C0B212280BD03000C0B2E4
:109B1000312807D03000C0B27E2803D03000C0B258
:109B20007F2800D10CE07F208DF800008DF80150D7
:109B30008DF802600322694614F11800FDF70DFC50
:109B4000F7BD30B400200422002108001300C0B289
:109B5000DBB298420BD20023DFF80C450D00EDB2CA
:109B60001420454304EB05000371491CEDE730BCAC
:109B700070472DE9F74F04001D000C9E00275FF091
:109B80000008002100220023002C02D10020308098
:109B900034E094F800905FFA89F95FEA191994F8B3
:109BA00000A01AF00F0A002001004A46C9B2D2B242
:109BB00091420AD20100C9B221444978D0F103028E
:109BC000D20091400F43401CEEE75FF0000B584677
:109BD0005146C0B2C9B288420CD25846C0B22044E5
:109BE0004079DBF10301C900884050EA08081BF105
:109BF000010BECE741463800FFF74FFDBDE8F78F5A
:109C000070472DE9F84304000D0016001F00DDF831
:109C10002080B8F80090FFF71AFD012817D1FFF750
:109C200019FD0100C9B202290AD101214A4692B2A6
:109C3000B15419F101090021DFF82C24117110E051
:109C400002214A4692B2B15419F1010909E00320F8
:109C5000494689B2705419F101090020DFF808144F
:109C60000871A8F80090BDE8F183F8B504000D0074
:109C700016001F00FFF776FDF1BD70472DE9F84390
:109C800004000D0016001F00DDF82080B8F80090D9
:109C9000FFF7DDFC042829D1FFF7DCFC012806D101
:109CA0000220494689B2705419F101091EE0FFF7FC
:109CB000D1FC02281AD1FFF7D0FC01280BD10120DA
:109CC000494689B2705419F101090020DFF8981350
:109CD00081F82C000AE00320494689B2705419F13A
:109CE00001090020DFF8801381F82C00A8F800900B
:109CF000BDE8F183F8B504000D0016001F00FFF762
:109D000031FDF1BD70472DE9F84304000D00160048
:109D10001F00DDF82080B8F80090FFF798FC0428B9
:109D200025D1FFF797FC012806D10220494689B2C8
:109D3000705419F101091AE0FFF78CFC022816D1C2
:109D4000FFF78BFC012809D10120494689B27054E4
:109D500019F101090020C449087608E003204946AA
:109D600089B2705419F101090020BF490876A8F89A
:109D70000090BDE8F1837047704770472DE9F64FBA
:109D8000ADF5037D04000D00002600208DF80800CD
:109D90000020ADF806005FF000085FF0000A04271D
:109DA0004FF40079494600220DF10C0B5846FDF79F
:109DB00087F80020ADF80400BDF81002A16894F8FF
:109DC0007A2001EBC201497889B2884205D2132278
:109DD00031212000FFF77AFE42E1687810F07F0021
:109DE0008DF80800A8780002E9784018ADF80A005C
:109DF000BDF81002001FADF80600BDF806000028EF
:109E000001D0281D06005FF0000840463900C0B2AE
:109E1000C9B2884232D21421934A4046C0B2484364
:109E2000105ABDF80A30984225D160784346DBB21B
:109E30004B4313449B78984217D14046C0B24843E5
:109E40001044C07800280FD04046C0B201FB00F19A
:109E500002EB0100C078A178884205D0332231217D
:109E60002000FFF733FEFBE008E022223121200032
:109E7000FFF72CFEF4E018F10108C6E74046390070
:109E8000C0B2C9B2884205D3312231212000FFF788
:109E90001DFEE5E0CA465FF0000B0DF10C095A46C5
:109EA00051464846FDF70CF871208DF80C000DF175
:109EB0000C09687889F80100A87889F80200E87828
:109EC00089F803000420ADF804009DF8080001287B
:109ED00005D0C0F09580032867D033D390E05FF0C1
:109EE000140ADFF884B14046C0B20AFB00F05844BF
:109EF000007901280CD17F208DF80C00312089F8E1
:109F00000100242089F802000320ADF8040018E0C5
:109F100001A800904FF4007303AABDF806103000AA
:109F2000C4465FFA8CFC0AFB0CFCDC44DCF808C07D
:109F3000E0474046C0B20AFB00FA0BEB0A000121E1
:109F400001716AE05FF0140ADFF81CB14046C0B24C
:109F50000AFB00F058440079002819D001A80090AD
:109F60004FF4007303AABDF806103000C4465FFA30
:109F70008CFC0AFB0CFCDC44DCF80CC0E0474046DF
:109F8000C0B20AFB00FA0BEB0A00002101710BE0E2
:109F90007F208DF80C00312089F80100242089F8F9
:109FA00002000320ADF8040037E05FF0140CDFF886
:109FB000B8E04046C0B20CFB00F0704400790028C5
:109FC00011D001A800904FF4007303AABDF8061049
:109FD0003000C2465FFA8AFA0CFB0AFCF444DCF853
:109FE00010C0E0470BE07F208DF80C00312089F88D
:109FF0000100242089F802000320ADF804000CE0E1
:10A000007F208DF80C00312089F80100122089F89A
:10A0100002000320ADF8040022E0BDF8040004288B
:10A020000ADB9DF80C00712806D1BDF8042003A9B5
:10A030002000FFF735FD13E0BDF8040003280AD126
:10A040009DF80C007F2806D199F8022031212000CC
:10A05000FFF73CFD04E0242231212000FFF736FD0C
:10A060000DF5057DBDE8F08F8C05FF1F0022026015
:10A0700041600122027200224272704770B50400F2
:10A080000D001600B4F88C1804F6A800FFF7EEFFD8
:10A0900094F87800012806D0320092B2290014F119
:10A0A0001800FDF75AF970BDFEB504000D0016004A
:10A0B000082100226F463800FCF702FF3000C0B2D2
:10A0C000782805D0B4F88C1804F6A800FFF7CEFF66
:10A0D00094F87900002814D03000C0B211280FD0B5
:10A0E0003000C0B212280BD03000C0B2312807D0E7
:10A0F0003000C0B27E2803D03000C0B27F2800D12B
:10A100000CE07F208DF800008DF801508DF8026082
:10A110000322694614F11800FDF71FF9F7BD2DE978
:10A12000FE4F04000D0016001F00DDF83080684669
:10A13000DFF814140A68026014F50860D0E9000121
:10A14000019001988DF8000069460198000A487056
:10A15000019A4B780720434353FAA2F08870019A82
:10A160009DF800300320434353FAB2F0C870380022
:10A17000C0B204281BD30420A8F800002800A1784E
:10A18000C0B288420AD15FF004095FF0000AB3460A
:10A19000524649465846FCF793FE08E05FF0040932
:10A1A000EA46B3464A4651465846FCF735FEBDE8F6
:10A1B000F78FFEB404002000C0B2012802D00928A5
:10A1C00049D094E0DFF884630D78307845408DF80D
:10A1D00000506D464F78707847406F708F78B07838
:10A1E0004740AF70CF78F0784740EF70E87810F0D4
:10A1F000F0008DF8040001A8EE78B60016F0BC0659
:10A200006F7817F003073E4346706E78F6B29DF8FC
:10A21000007017F0C00757EA960787709DF8006036
:10A22000AD7815F00F0555EA0615C5709DF8045078
:10A230001E78B5420BD145785E78B54207D1857856
:10A240009E78B54203D1C078DD78A84201D00020C5
:10A250004EE001204CE0BD4E0D78307845408DF841
:10A2600000506D464F78707847406F708F78B078A7
:10A270004740AF70CF78F0784740EF706878AE789D
:10A2800016F0F00656EA80068DF8046001A89DF8E5
:10A290000060F6B2B60816F03B066F7817F07E073E
:10A2A0003E434670EE78F6B29DF8007017F02C072A
:10A2B00057EA16178770AE78ED7815F07D0555EAE8
:10A2C0000615C5709DF804501E78B5420BD145782F
:10A2D0005E78B54207D185789E78B54203D1C078C3
:10A2E000DD78A84201D0002002E0012000E000203B
:10A2F000FEBC70472DE9F74F84B004005FF0000A00
:10A300000821002202AD2800FCF7DAFD0020ADF89C
:10A3100004005FF000095FF00008BDF81800A168B4
:10A3200094F87A2001EBC201497889B2884205D2BB
:10A33000132227212000FFF7B7FE02E160780128F1
:10A3400005D1222227212000FFF7AEFEF9E0059873
:10A35000457815F07F0567208DF808008DF80950C5
:10A36000E8077BD57A4E0020307000273800C0B255
:10A37000022839DADFF8DCC128003900C9B2090146
:10A380001CF80110C0B288422CD13800C0B20001C4
:10A39000604480783900C9B2090161444978884233
:10A3A0001FD214F50860D0E900233800C0B20001C4
:10A3B0006044D0E90201121A8B4142F21070002170
:10A3C0008B4208DC01DB824205D2362227212000A5
:10A3D000FFF76AFEB5E000203900C9B20901614407
:10A3E000487001E07F1CC1E73800C0B2022805DBDD
:10A3F000312227212000FFF757FEA2E006208146E8
:10A4000001A800904B46DBB20DF10A022900C9B247
:10A410002000FFF784FEBDF80400002818D0BDF826
:10A420000420921C92B202A92000FFF727FE35708B
:10A43000BDF8040048490880BDF804600DF10A0A1F
:10A44000DFF818B1320051465846FCF7E5FC78E0D9
:10A45000312227212000FFF727FE72E03C4E280022
:10A46000C0B23178491C884205D02422272120001F
:10A47000FFF71AFE65E0BDF81800801E80B200905C
:10A480000598831C3448028834493078FFF791FEE0
:10A4900080464046C0B201281ED1022202A92000F7
:10A4A000FFF7ECFD00203070681EA0700027380018
:10A4B000C0B2022845DA274829003A00D2B2120178
:10A4C000825CC9B2914205D100213A00D2B2120198
:10A4D000104441707F1CEAE7352227212000FFF756
:10A4E000E3FD00273800C0B202282ADA194A307882
:10A4F0003900C9B20901515C884220D13800C0B28C
:10A50000000110444078401C3900C9B209011144CF
:10A5100048703800C0B20001104480783900C9B2D8
:10A52000090111444978884209D214F50860D0E93C
:10A5300000013B00DBB21B011A44C2E902017F1C8F
:10A54000D0E707B0BDE8F08FDCD00000E0D000001D
:10A55000003600200004FF1FFC350020AC35002031
:10A5600000000000963007772C610EEEBA51099971
:10A5700019C46D078FF46A7035A563E9A395649ECD
:10A580003288DB0EA4B8DC791EE9D5E088D9D297F1
:10A590002B4CB609BD7CB17E072DB8E7911DBF904D
:10A5A0006410B71DF220B06A4871B9F3DE41BE8471
:10A5B0007DD4DA1AEBE4DD6D51B5D4F4C785D383CD
:10A5C00056986C13C0A86B647AF962FDECC9658A71
:10A5D0004F5C0114D96C0663633D0FFAF50D088DCD
:10A5E000C8206E3B5E10694CE44160D5727167A271
:10A5F000D1E4033C47D4044BFD850DD26BB50AA5CD
:10A60000FAA8B5356C98B242D6C9BBDB40F9BCACF0
:10A61000E36CD832755CDF45CF0DD6DC593DD1AB4C
:10A62000AC30D9263A00DE518051D7C81661D0BF70
:10A63000B5F4B42123C4B3569995BACF0FA5BDB8CC
:10A640009EB802280888055FB2D90CC624E90BB170
:10A65000877C6F2F114C6858AB1D61C13D2D66B6CC
:10A660009041DC760671DB01BC20D2982A10D5EF30
:10A670008985B1711FB5B606A5E4BF9F33D4B8E88C
:10A68000A2C9077834F9000F8EA8099618980EE130
:10A69000BB0D6A7F2D3D6D08976C6491015C63E68C
:10A6A000F4516B6B62616C1CD83065854E0062F2B0
:10A6B000ED95066C7BA5011BC1F4088257C40FF50C
:10A6C000C6D9B06550E9B712EAB8BE8B7C88B9FC30
:10A6D000DF1DDD62492DDA15F37CD38C654CD4FB8C
:10A6E0005861B24DCE51B53A7400BCA3E230BBD430
:10A6F00041A5DF4AD795D83D6DC4D1A4FBF4D6D38C
:10A700006AE96943FCD96E34468867ADD0B860DA2F
:10A71000732D0444E51D03335F4C0AAAC97C0DDD8B
:10A720003C710550AA41022710100BBE86200CC9AF
:10A7300025B56857B3856F2009D466B99FE461CE0B
:10A740000EF9DE5E98C9D9292298D0B0B4A8D7C72F
:10A75000173DB359810DB42E3B5CBDB7AD6CBAC08B
:10A760002083B8EDB6B3BF9A0CE2B6039AD2B174A7
:10A770003947D5EAAF77D29D1526DB048316DC7303
:10A78000120B63E3843B64943E6A6D0DA85A6A7AA7
:10A790000BCF0EE49DFF099327AE000AB19E077D03
:10A7A00044930FF0D2A3088768F2011EFEC2066927
:10A7B0005D5762F7CB67658071366C19E7066B6E83
:10A7C000761BD4FEE02BD3895A7ADA10CC4ADD67A7
:10A7D0006FDFB9F9F9EFBE8E43BEB717D58EB06003
:10A7E000E8A3D6D67E93D1A1C4C2D83852F2DF4FA7
:10A7F000F167BBD16757BCA6DD06B53F4B36B24803
:10A80000DA2B0DD84C1B0AAFF64A0336607A0441A6
:10A81000C3EF60DF55DF67A8EF8E6E3179BE694602
:10A820008CB361CB1A8366BCA0D26F2536E2685226
:10A8300095770CCC03470BBBB91602222F26055582
:10A84000BE3BBAC5280BBDB2925AB42B046AB35CA6
:10A85000A7FFD7C231CFD0B58B9ED92C1DAEDE5B02
:10A86000B0C2649B26F263EC9CA36A750A936D02E6
:10A87000A906099C3F360EEB856707721357000542
:10A88000824ABF95147AB8E2AE2BB17B381BB60C66
:10A890009B8ED2920DBED5E5B7EFDC7C21DFDB0BC2
:10A8A000D4D2D38642E2D4F1F8B3DD686E83DA1FE6
:10A8B000CD16BE815B26B9F6E177B06F7747B71842
:10A8C000E65A0888706A0FFFCA3B06665C0B0111E6
:10A8D000FF9E658F69AE62F8D3FF6B6145CF6C1642
:10A8E00078E20AA0EED20DD75483044EC2B30339E6
:10A8F000612667A7F71660D04D476949DB776E3E42
:10A900004A6AD1AEDC5AD6D9660BDF40F03BD83765
:10A9100053AEBCA9C59EBBDE7FCFB247E9FFB530C1
:10A920001CF2BDBD8AC2BACA3093B353A6A3B424E5
:10A930000536D0BA9306D7CD2957DE54BF67D92341
:10A940002E7A66B3B84A61C4021B685D942B6F2AE5
:10A9500037BE0BB4A18E0CC31BDF055A8DEF022D41
:10A960002DE9F04F93B040F2C710D549086001219E
:10A97000D44AD06A400840000B00DBB213F0010358
:10A98000184301900198D062CF4BDFF840B3CDF867
:10A9900000B00098C0F88030CD4CCE480500C5F816
:10A9A000804002265F46D7F800C03CF00C0CB6464B
:10A9B0005FFA8EFE5FEA8E0E1EF00C0E5EEA0C0C45
:10A9C000C7F800C05FF0010ED846D8F8089039F0FB
:10A9D0000409F2465FFA8AFA5FEA8A0A1AF0040A60
:10A9E0005AEA0909C8F808905946C968C1F38001B4
:10A9F000C9B20029F8D000218DF80010CDF824B09C
:10AA00000999896831F008019DF80020D20012F000
:10AA10000802114312911299099A91600221CDF80E
:10AA200020B0089A5268920892000B00DBB213F033
:10AA300003031A431192119A089B5A600022CDF821
:10AA40001CB0079B5B6833F00C031400E4B2A40055
:10AA500014F00C0423431093109B079C63605A234B
:10AA6000CDF818B0069C646834F4FE441D00EDB2C5
:10AA70002D0215F4FE452C430F940F9C069D6C602F
:10AA80000024CDF814B0059D6D6835F4803526009E
:10AA9000F6B2360416F4803635430E950E9D059EAB
:10AAA00075600325CDF810B0049E766836F0700608
:10AAB0002F00FFB23F0117F070073E430D960D9E29
:10AAC000049F7E6000260390039F3F6CFF08FF00F9
:10AAD000B4465FFA8CFC1CF0070C5CEA07070C9785
:10AAE0000C9FDDF80CC0CCF8407000270290DDF818
:10AAF00008C0DCF840E03EF0700EBC465FFA8CFC0B
:10AB00005FEA0C1C1CF0700C5CEA0E0ECDF82CE019
:10AB1000DDF82CC0DDF808E0CEF840C05FF0010E93
:10AB2000CDF804B0DDF804C0DCF8088038F008087F
:10AB3000F4465FFA8CFC5FEACC0C1CF0080C5CEA73
:10AB40000808CDF82880DDF828C0DDF80480C8F8B2
:10AB500008C0DFF884C14BF68038CCF80080DFF8FD
:10AB60007C815FF00009C8F80090DFF874915FF015
:10AB7000050AC9F800A0D9F80010B1F5803FFAD352
:10AB80000421C9F800100021CCF800100021C8F8F9
:10AB900000105946C968C1F3C001C9B20029F8D0F4
:10ABA0000021CDF804B0019A126932F0F0020B00D6
:10ABB000DBB21B0113F0F0031A430692069A019BC5
:10ABC0001A6101220090009B1B6833F4706314002B
:10ABD000E4B2240214F4706423430593059B009CA3
:10ABE00023600E23040025686D096D011E00F6B276
:10ABF00016F01F0635430495049D25600225394E45
:10AC0000776837F47067AC465FFA8CFC5FEA0C2C0F
:10AC10001CF4706C5CEA070777605FF0020ED846A0
:10AC2000D8F810905FEA99095FEA8909F4465FFA5B
:10AC30008CFC1CF0030C5CEA0909C8F810905FF06A
:10AC4000000ACDF80CB0DDF80CC0CCF880A05FF0A5
:10AC5000000B02900298C0F880B02348D0F800C0E2
:10AC60005CF4700CC0F800C00020DFF880C0CCF8A5
:10AC700000000020DFF878C0CCF800000020DFF8EA
:10AC800074C0CCF800000020DFF86CC0CCF80000E5
:10AC90000020DFF868C0CCF800000020DFF860C0BA
:10ACA000CCF800000020DFF85CC0CCF800000020E9
:10ACB000DFF854C0CCF8000013B0BDE8F08F00BF3F
:10ACC000002008E000F00540E42386FA00F8074081
:10ACD000656D435300E0064014E000E018E000E03A
:10ACE00010E000E00000024088ED00E0200000409D
:10ACF00024000040280000402C00004030000040AC
:10AD000034000040380000403C0000400022026057
:10AD100041600122027200224272704770B5040045
:10AD20000D001600B4F88C1804F6A800FFF7EEFF2B
:10AD300094F87800012806D0320092B2290014F16C
:10AD40001800FCF70AFB70BDFEB504000D001600EC
:10AD5000082100226F463800FCF7B2F83000C0B27C
:10AD6000782805D0B4F88C1804F6A800FFF7CEFFB9
:10AD700094F87900002814D03000C0B211280FD008
:10AD80003000C0B212280BD03000C0B2312807D03A
:10AD90003000C0B27E2803D03000C0B27F2800D17E
:10ADA0000CE07F208DF800008DF801508DF80260D6
:10ADB0000322694614F11800FCF7CFFAF7BD2DE91C
:10ADC000F44FADF5027D04000D0000270020ADF822
:10ADD00004005FF000095FF00008002600208DF8F5
:10ADE00000004FF4007100220DF1080A5046FCF7F4
:10ADF00067F8BDF80802A16894F87A2001EBC20157
:10AE0000497889B2884205D2132222212000FFF717
:10AE10009BFFF6E0BDF80802401EC00705D51322CF
:10AE200022212000FFF790FFEBE0BDF80802400868
:10AE3000ADF80600BDF80600002805D11322222136
:10AE40002000FFF781FFDCE0622002A94A4692B2AF
:10AE5000885419F1010901273800BDF8081280B2A1
:10AE6000884280F0BE80380080B2295C0902380038
:10AE700080B2284440780143ADF8041000208DF8DA
:10AE80000000002006003000A18A80B2884280F0D5
:10AE9000A2805FF014082069310089B208FB01F13B
:10AEA000405ABDF80410884240F09380A078216990
:10AEB000320092B208FB02F211440979884205D0AF
:10AEC000332222212000FFF73FFF9AE02069310062
:10AED00089B208FB01F10844808910FA89F0801CCE
:10AEE00040F20121884205DB142222212000FFF7D5
:10AEF0002BFF86E02069310089B208FB01F108448C
:10AF00008078052809D060782169320092B208FB68
:10AF100002F21144C978884205D22222222120005F
:10AF2000FFF712FF6DE02069310089B208FB01F1E3
:10AF300008448289D2B22069310089B208FB01F14C
:10AF40000844816820002369B4461FFA8CFC08FB82
:10AF50000CFC63441B69984701208DF8000002A98E
:10AF6000380080B2285C4A4692B2885419F101092F
:10AF700048463A0092B22A44527803009BB2CA541F
:10AF8000401CADF802002069310089B208FB01F1D4
:10AF90000844B0F80CA02069310089B208FB01F127
:10AFA0000844D0F808B002A8BDF8021000EB01096F
:10AFB000524659464846FBF72FFFBDF802902069DC
:10AFC000310089B208FB01F84044808910EB09097F
:10AFD00001E0761C57E79DF80000002801D0BF1C57
:10AFE0003AE79DF80000002806D04A4692B202A92E
:10AFF0002000FFF793FE04E0312222212000FFF71A
:10B00000A3FE0DF5037DBDE8F08F00000022026075
:10B0100041600122027200224272704770B5040042
:10B020000D001600B4F88C1804F6A800FFF7EEFF28
:10B0300094F87800012806D0320092B2290014F169
:10B040001800FCF78AF970BDFEB504000D0016006B
:10B05000082100226F463800FBF732FF3000C0B2F3
:10B06000782805D0B4F88C1804F6A800FFF7CEFFB6
:10B0700094F87900002814D03000C0B211280FD005
:10B080003000C0B212280BD03000C0B2312807D037
:10B090003000C0B27E2803D03000C0B27F2800D17B
:10B0A0000CE07F208DF800008DF801508DF80260D3
:10B0B0000322694614F11800FCF74FF9F7BD7047F9
:10B0C0007047704770472DE9F64FADF5037D0400DA
:10B0D0000D005FF000095FF0000A5FF0000B022630
:10B0E0004FF40071002203AF3800FBF7E9FEBDF812
:10B0F0001002A16894F87A2001EBC201497889B264
:10B10000884205D213222F212000FFF79DFFC2E0C5
:10B110006078012805D122222F212000FFF794FF1B
:10B12000B9E068780002A9784718E8788DF800003F
:10B130005FF0000840463100C0B2C9B2884224D254
:10B140001421574A4046C0B24843105A3B009BB2B4
:10B15000984217D14046C0B2484310448078002836
:10B160000FD04046C0B201FB00F102EB0100807835
:10B17000A178884205D033222F212000FFF764FFF9
:10B1800089E002E018F10108D4E740463100C0B27E
:10B19000C9B2884205D331222F212000FFF754FF86
:10B1A00079E06F208DF80C0003A869784170A978C8
:10B1B0008170E978C1709DF80000002802D0032852
:10B1C0001DD063E01421364A4046C0B248431044C3
:10B1D0000023C3724046C0B24843104400690028AF
:10B1E0000CD04046C0B201FB00F102EB0100006947
:10B1F0008047042203A92000FFF710FF4BE05FF017
:10B200001409DFF89CA0BDF810024146C9B209FB41
:10B2100001F15144097A091D884205DA22222F21C1
:10B220002000FFF711FF36E04046C0B209FB00F0F6
:10B2300050440121C1724046C0B209FB00F05044A5
:10B24000007A0290281D01904046C0B209FB00F030
:10B250005044D0F804B0029A01995846FBF7DCFD3F
:10B260004046C0B209FB00F05044C06800280CD032
:10B270004046C0B209FB00F90AEB0900C0688047EC
:10B28000042203A92000FFF7C9FE04E031222F2188
:10B290002000FFF7D9FE0DF5057DBDE8F08F000019
:10B2A0006405FF1F98490870704710B4010089B207
:10B2B000142926DA0C21954A03009BB24B43134410
:10B2C00000241C7103009BB24B4313441B1D1C78CC
:10B2D00054F010041C7003009BB24B4313441B1D1D
:10B2E0001C7854F040041C7003009BB24B43134481
:10B2F0000024DC8003009BB201FB03F11144002217
:10B300000A7210BC704770B40200002100240020B3
:10B310000023190089B2142911DA7C4D1E00B6B23F
:10B320000C214E4305EB0601097911F07F010C0059
:10B330002100C9B2114200D0401C5B1CE9E780B279
:10B3400070BC7047F0B504000023002500200026E3
:10B3500033009BB2142B41DA0C27DFF8B0C1330065
:10B360009BB27B4363441B791D002B00DBB213426D
:10B3700032D00B009BB286461FFA8EFE1EF1040EE1
:10B38000734528DB33009BB27B435CF803301B0C16
:10B3900086461FFA8EFE04F80E30401C33009BB226
:10B3A0007B435CF803301B0A86461FFA8EFE04F8C6
:10B3B0000E30401C33009BB207FB03F75CF80730EC
:10B3C0000700BFB2E355401C15F07F030700BFB272
:10B3D000E355401C00E001E0761CB9E780B2F0BD07
:10B3E000F0B4020000250023002000242500ADB2A7
:10B3F000142D37DA0C25454E2700BFB26F43374472
:10B400003F793B000F00BFB284461FFA8CFC1CF151
:10B41000040C674526DB2700BFB26F43F7593F0C8A
:10B4200084461FFA8CFC02F80C70401C2700BFB247
:10B430006F43F7593F0A84461FFA8CFC02F80C70E0
:10B44000401C2700BFB205FB07F575590600B6B2D0
:10B450009555401C13F07F050600B6B29555401C6B
:10B46000641CC3E780B2F0BC704738B50400002507
:10B4700020002749401A04D09D3818D02F3834D0E6
:10B480003FE000200500280080B214280EDA1F4992
:10B490002A0092B20C2042438858B0F5801F03D294
:10B4A000280080B2FFF701FF6D1CECE729E00020C7
:10B4B0000500280080B2142816DA0C2013492A004F
:10B4C00092B242438A58B2F5800F0BD32A0092B24F
:10B4D00000FB02F00858B0F5000F03D2280080B23C
:10B4E000FFF7E3FE6D1CE4E70BE0002005002800F9
:10B4F00080B2142805DA280080B2FFF7D6FE6D1C52
:10B50000F5E731BD00000000FF3500207404FF1F87
:10B5100033FFFF000022026041600122027200221C
:10B520004272704770B504000D001600B4F88C1814
:10B5300004F6A800FFF7EEFF94F87800012806D083
:10B54000320092B2290014F11800FBF706FF70BD1B
:10B55000FEB504000D001600082100226F463800D9
:10B56000FBF7AEFC3000C0B2782805D0B4F88C18D8
:10B5700004F6A800FFF7CEFF94F87900002814D055
:10B580003000C0B211280FD03000C0B212280BD04A
:10B590003000C0B2312807D03000C0B27E2803D0BE
:10B5A0003000C0B27F2800D10CE07F208DF8000071
:10B5B0008DF801508DF802600322694614F11800DD
:10B5C000FBF7CBFEF7BD10B50024FDF7EDFD801CA9
:10B5D00010BD10B402000021002001231900C9B2DF
:10B5E00005290CDAD3F10404E4001100E14000293C
:10B5F00003D0D3F10501080001E05B1CEEE7C0B207
:10B6000010BC70472DE9F44F84B005000E005FF0C8
:10B61000000900208DF8010000245FF0000B0020DD
:10B620008DF80000002001905FF0000A0027687884
:10B63000012805D1222234212800FFF789FF9CE050
:10B64000BDF81000A96895F87A2001EBC20149788D
:10B6500089B2884205D2132234212800FFF778FFEF
:10B660008BE096F8028018F00F08B078C0B200099D
:10B670008DF801004046C0B200280BD04046C0B251
:10B68000052807D29DF80100002803D09DF801008D
:10B69000052805D3312234212800FFF759FF6CE03B
:10B6A000002001004246C9B2D2B2914209D25FEAFB
:10B6B00009290100C9B23144C97859FA81F9401CFD
:10B6C000EFE75FF0000A50469DF80110C0B28842D3
:10B6D0000BD224025046C0B250FA88F03044C078F1
:10B6E00054FA80F41AF1010AEDE7002C05D1222268
:10B6F00034212800FFF72CFF3FE000F09AF848467D
:10B7000000F0A7F8200000F0A7F8012000F0AAF848
:10B71000FFF759FF01900198FFF75BFF8DF80000DC
:10B7200002A874213A0092B281547F1C9DF8001047
:10B7300009013A0092B281547F1C5FF0010B9DF821
:10B7400000105A46D2B291420DD301999DF80020C3
:10B75000B2EB0B02D200D1403A0092B281547F1C6E
:10B760001BF1010BEBE721004846FDF7C4FF3A004F
:10B7700092B202A92800FFF7D5FE05B0BDE8F08F10
:10B780000022026041600122027200224272704770
:10B7900070B504000D001600B4F88C1804F6A8006B
:10B7A000FFF7EEFF94F87800012806D0320092B23D
:10B7B000290014F11800FBF7D0FD70BDFEB50400A0
:10B7C0000D001600082100226F463800FBF778FBB9
:10B7D0003000C0B2782805D0B4F88C1804F6A80060
:10B7E000FFF7CEFF94F87900002814D03000C0B2E3
:10B7F00011280FD03000C0B212280BD03000C0B2D8
:10B80000312807D03000C0B27E2803D03000C0B24B
:10B810007F2800D10CE07F208DF800008DF80150CA
:10B820008DF802600322694614F11800FBF795FDBC
:10B83000F7BD0020534908700020534908700020CC
:10B8400052490860002052490860002051490860B0
:10B8500070474F49086070474E49086070474D482F
:10B86000006870474C49087070474B480078704733
:10B870004648006870472DE9FE4304000D0016009D
:10B880000A2100226F463800FBF71AFB6078012876
:10B8900005D1222236212000FFF790FF6FE0300013
:10B8A000A16894F87A2001EBC201497880B289B28C
:10B8B000884205D2132236212000FFF77FFF5EE089
:10B8C00035480078012802D002284DD052E02D4F93
:10B8D00068783870DFF8B080387898F800108842BF
:10B8E0000CD0387898F80010491CC9B2884205D0AD
:10B8F000732236212000FFF761FF40E0DFF88C90D3
:10B9000024480068D9F8001011FA86F1891E88428F
:10B9100005D2712236212000FFF750FF2FE0387842
:10B9200098F80010491CC9B288421CD13A78B11E5F
:10B9300089B2A81CFDF7F1FE012806D1D9F8000054
:10B9400010FA86F0801EC9F80000387888F80000E8
:10B9500076208DF8000038788DF8010002226946C3
:10B960002000FFF715FF0AE0312236212000FFF703
:10B9700025FF04E0242236212000FFF71FFFBDE849
:10B98000F78300000336002004360020C035002075
:10B99000B8350020BC35002002360020010005002B
:10B9A0000000000000000000000000000900050089
:10B9B0000000000000000000000000006F92000086
:10B9C000B392000083930000B39500005B940000E5
:10B9D000519500000100000032070000DF07000061
:10B9E000B2070000441300200002000044150020AC
:10B9F00008080000000000008F7B00001D7A000096
:10BA00003200F40188130000010203040506070850
:10BA10001A62040050000000000000001B630400D4
:10BA200050000000000000001603F000500000006D
:10BA3000000000001703F0005000000000000000AC
:10BA40008873C00050000000000000000100C10029
:10BA500050000000000000000101C1005000000083
:10BA6000000000000121C1005000000000000000A3
:10BA70000127C10050000000000000000128C100A3
:10BA800050000000000000000129C100500000002B
:10BA9000000000000131C100500000000000000063
:10BAA0000041C10050000000000000000151C10031
:10BAB00050000000000000000063C10050000000C2
:10BAC000000000000069C1005000000000000000FC
:10BAD0000181C10050000000000000000136C200DA
:10BAE00050000000000000000064C1005000000091
:10BAF000000000000067C1005000000000000000CE
:10BB000092F00000B435002002000000BFB0000039
:10BB1000C1B0000020F00000B63500200200000097
:10BB2000C3B00000C5B0000001FD02090000000024
:10BB3000739B0000019C0000039C000002FD0209B1
:10BB400000000000F59C0000059D0000079D00001E
:10BB500003FD0209000000006B9C00007B9C0000BC
:10BB60007D9C000004FD020900000000779D00009C
:10BB7000799D00007B9D000086F106010000000019
:10BB8000C435002001000000F190000087F106019B
:10BB900000000000C535002008000000F7900000FC
:10BBA00080F1060100000000CD35002008000000F3
:10BBB000C990000091F1060100000000D535002079
:10BBC000180000001F91000093F106010000000022
:10BBD000ED350020040000006191000095F10601A0
:10BBE00000000000F13500200800000087910000EF
:10BBF00000220260416001220272002242727047FC
:10BC000070B504000D001600B4F88C1804F6A800F6
:10BC1000FFF7EEFF94F87800012806D0320092B2C8
:10BC2000290014F11800FBF798FB70BDFEB5040065
:10BC30000D001600082100226F463800FBF740F97E
:10BC40003000C0B2782805D0B4F88C1804F6A800EB
:10BC5000FFF7CEFF94F87900002814D03000C0B26E
:10BC600011280FD03000C0B212280BD03000C0B263
:10BC7000312807D03000C0B27E2803D03000C0B2D7
:10BC80007F2800D10CE07F208DF800008DF8015056
:10BC90008DF802600322694614F11800FBF75DFB82
:10BCA000F7BD2DE9FE4304000D0016000821002217
:10BCB0006F463800FBF704F900273000A16894F8BC
:10BCC0007A2001EBC201497880B289B2884205D25C
:10BCD000132228212000FFF7A9FF8EE060780128B9
:10BCE00005D1222228212000FFF7A0FF85E095F84A
:10BCF000018018F07F0895F8029068208DF8000008
:10BD00008DF801804046C0B2002805D0022839D005
:10BD10001DD3032851D06BE04846C0B2012807D09C
:10BD20004846C0B2022803D04846C0B2032808D112
:10BD3000002033490870022269462000FFF760FFA7
:10BD400004E0312228212000FFF770FF55E048462B
:10BD5000C0B2012807D04846C0B2022803D04846E6
:10BD6000C0B2032808D10120254908700222694683
:10BD70002000FFF745FF04E0312228212000FFF7D3
:10BD800055FF3AE04846C0B2012807D04846C0B245
:10BD9000022803D04846C0B2032808D1022018491F
:10BDA0000870022269462000FFF72AFF04E03122D2
:10BDB00028212000FFF73AFF1FE04846C0B20128C3
:10BDC00007D04846C0B2022803D04846C0B2032874
:10BDD00008D103200A490870022269462000FFF7B3
:10BDE0000FFF04E0312228212000FFF71FFF04E0AD
:10BDF000122228212000FFF719FFBDE8F783000079
:10BE000001360020002202604160012202720022FD
:10BE10004272704770B504000D001600B4F88C181B
:10BE200004F6A800FFF7EEFF94F87800012806D08A
:10BE3000320092B2290014F11800FBF78EFA70BD9F
:10BE4000FEB504000D001600082100226F463800E0
:10BE5000FBF736F83000C0B2782805D0B4F88C185B
:10BE600004F6A800FFF7CEFF94F87900002814D05C
:10BE70003000C0B211280FD03000C0B212280BD051
:10BE80003000C0B2312807D03000C0B27E2803D0C5
:10BE90003000C0B27F2800D10CE07F208DF8000078
:10BEA0008DF801508DF802600322694614F11800E4
:10BEB000FBF753FAF7BD2DE9F04FADF5017D040016
:10BEC0000D00160000208DF8000000275FF000082C
:10BED0005FF000094FF4007100220DF1040A504692
:10BEE000FAF7EEFF3000A16894F87A2001EBC20166
:10BEF000497880B289B2884205D2132219212000E4
:10BF0000FFF79EFF76E095F801A01AF07F0A59200E
:10BF10008DF804000DF1040B8BF801A05046C0B25F
:10BF2000012804D0022827D00A2845D05DE030003F
:10BF300080B2032805D0132219212000FFF780FFCB
:10BF400058E0A87807003800C0B2FFF7DCF9804657
:10BF50007F208BF8020001208BF80300404680B25E
:10BF6000000A8DF8080040468DF80900062201A954
:10BF70002000FFF74FFF3DE0300080B2032805D0DE
:10BF8000132219212000FFF75BFF33E0A878070098
:10BF90007F208BF802003A00D2B240F2FD110DF181
:10BFA0000700FFF7CFF9814619F1030292B201A908
:10BFB0002000FFF72FFF1DE0300080B2022805D0DF
:10BFC000132219212000FFF73BFF13E040F2FD117F
:10BFD0000DF10700FFF704FA814619F1030292B24E
:10BFE00001A92000FFF716FF04E01222192120000A
:10BFF000FFF726FF0DF5017DBDE8F08F00220260FE
:10C0000041600122027200224272704770B5040042
:10C010000D001600B4F88C1804F6A800FFF7EEFF28
:10C0200094F87800012806D0320092B2290014F169
:10C030001800FBF792F970BDFEB504000D00160064
:10C04000082100226F463800FAF73AFF3000C0B2EC
:10C05000782805D0B4F88C1804F6A800FFF7CEFFB6
:10C0600094F87900002814D03000C0B211280FD005
:10C070003000C0B212280BD03000C0B2312807D037
:10C080003000C0B27E2803D03000C0B27F2800D17B
:10C090000CE07F208DF800008DF801508DF80260D3
:10C0A0000322694614F11800FBF757F9F7BD2DE993
:10C0B000FE4F04000D00160000275FF00008082165
:10C0C0000022E9464846FAF7FBFE3000A16894F8E2
:10C0D0007A2001EBC201497880B289B2884205D248
:10C0E00013222E212000FFF7A7FF81E095F8019091
:10C0F0005FEA0929A87850EA09096E208DF8000046
:10C10000684669784170A97881705FF0000A5046EE
:10C11000A18A80B2884266D214212069524692B226
:10C120004A43805A4A4692B2904259D120695246B7
:10C1300092B24A431044007900280ED0A0782269B8
:10C1400053469BB24B431A441279904205D0332296
:10C1500022212000FFF770FF4AE0300080B2C01EAD
:10C16000226953469BB24B431A449289904205D0B0
:10C1700013222E212000FFF75FFF39E0206952468D
:10C1800092B24A4310448078032808D0607822692C
:10C1900053469BB24B431A44D278904205D2222296
:10C1A0002E212000FFF748FF22E02069524692B27C
:10C1B0004A431044878915F103082069524692B218
:10C1C00001FB02F10844D0F808B03A004146584655
:10C1D000FAF722FE032269462000FFF717FF07E067
:10C1E0001AF1010A93E731222E212000FFF724FFE4
:10C1F000BDE8F78F00220260416001220272002236
:10C200004272704770B504000D001600B4F88C1827
:10C2100004F6A800FFF7EEFF94F87800012806D096
:10C22000320092B2290014F11800FBF796F870BDA5
:10C23000FEB504000D001600082100226F463800EC
:10C24000FAF73EFE3000C0B2782805D0B4F88C185A
:10C2500004F6A800FFF7CEFF94F87900002814D068
:10C260003000C0B211280FD03000C0B212280BD05D
:10C270003000C0B2312807D03000C0B27E2803D0D1
:10C280003000C0B27F2800D10CE07F208DF8000084
:10C290008DF801508DF802600322694614F11800F0
:10C2A000FBF75BF8F7BDFEB504000D001600082192
:10C2B00000226F463800FAF703FE3000A16894F8B8
:10C2C0007A2001EBC201497880B289B2884205D058
:10C2D000132210212000FFF7ABFF64E06F7817F006
:10C2E0007F0750208DF8000068464770B4F8881822
:10C2F00089B2090A8170B4F88818C170B4F88A0844
:10C3000080B2000A8DF80400B4F88A088DF80500A0
:10C31000FDF717FC3800C0B2012806D03ED3032831
:10C320000CD01AD304282AD038E00020A0706770FF
:10C33000062269462000FFF765FF34E00020A07068
:10C340006770062269462000FFF75CFFB4F88C187E
:10C3500004F6A800FFF74EFF25E00020A0706770EC
:10C36000062269462000FFF74DFFB4F88C1804F64A
:10C37000A800FFF73FFF0120FDF773F913E000204D
:10C38000A0706770062269462000FFF73BFFB4F8F3
:10C390008C1804F6A800FFF72DFF04E012221021EC
:10C3A0002000FFF745FFF7BDE12E00000B2F000036
:10C3B000C92F0000F32F0000692E0000932E00000B
:10C3C0003D3000002D310000C7320000173300005F
:10C3D000C733000017340000C934000019350000CD
:10C3E000C935000019360000CB3600001B370000AD
:10C3F000CB3700001B380000CD3800001F3900008B
:10C40000CF390000213A0000D33A00002B3B000056
:10C41000933B0000CB3B0000FF3B0000393C000099
:10C420006D3C0000B93C00000B3D0000593D000090
:10C43000C53D0000153F0000FF4100000000000066
:10C4400009420000274200005342000071420000F0
:10C450009D42000000000000A9420000FB420000D5
:10C460004143000085430000B34300002D44000019
:10C47000F3440000BD450000AF4600000147000046
:10C480004347000087470000B1470000F547000020
:10C490001F480000634800008D480000D14800009C
:10C4A000FB4800003F490000694900009149000035
:10C4B000BD490000E5490000114A0000394A00006A
:10C4C000654A00008D4A0000B94A0000E14A0000B8
:10C4D0000D4B00002F4B00005B4B00007D4B00001C
:10C4E000A94B0000CB4B0000F74B0000194C00009B
:10C4F000454C0000694C0000954C0000B94C000010
:10C50000E54C0000094D0000354D0000594D00007C
:10C51000854D0000A94D0000D54D0000F94D0000EB
:10C52000254E0000494E0000754E0000D94E000017
:10C530006B4F0000D14F000065500000CB50000051
:10C540005F510000C55100000022026041600122DD
:10C55000027200224272704770B504000D0016008E
:10C56000B4F88C1804F6A800FFF7EEFF94F87800F2
:10C57000012806D0320092B2290014F11800FAF70F
:10C58000ECFE70BDFEB504000D001600082100226F
:10C590006F463800FAF794FC3000C0B2782805D016
:10C5A000B4F88C1804F6A800FFF7CEFF94F87900D1
:10C5B000002814D03000C0B211280FD03000C0B213
:10C5C00012280BD03000C0B2312807D03000C0B2E2
:10C5D0007E2803D03000C0B27F2800D10CE07F203D
:10C5E0008DF800008DF801508DF802600322694635
:10C5F00014F11800FAF7B1FEF7BD2DE9FC41040073
:10C600000D001600002708210022E8464046FAF7F0
:10C6100057FC6078012805D1222237212000FFF73E
:10C62000B1FF3FE03000A16894F87A2001EBC2012D
:10C63000497880B289B2884205D21322372120007E
:10C64000FFF7A0FF2EE0772069463A0092B28854A7
:10C650007F1CFFF70AF9012802D0022814D019E044
:10C66000FFF706F98046FFF7FAF8804505D0132258
:10C6700037212000FFF786FF11E03A0092B26946A9
:10C680002000FFF769FF0AE0312237212000FFF781
:10C6900079FF04E0242237212000FFF773FF0020F8
:10C6A000FFF7E0F8BDE8F38100220260416001225B
:10C6B000027200224272704770B504000D0016002D
:10C6C000B4F88C1804F6A800FFF7EEFF94F8780091
:10C6D000012806D0320092B2290014F11800FAF7AE
:10C6E0003CFE70BDFEB504000D00160008210022BE
:10C6F0006F463800FAF7E4FB3000C0B2782805D066
:10C70000B4F88C1804F6A800FFF7CEFF94F879006F
:10C71000002814D03000C0B211280FD03000C0B2B1
:10C7200012280BD03000C0B2312807D03000C0B280
:10C730007E2803D03000C0B27F2800D10CE07F20DB
:10C740008DF800008DF801508DF8026003226946D3
:10C7500014F11800FAF701FEF7BD2DE9FC410400C1
:10C760000D001600082100226F463800FAF7A8FBDA
:10C77000FF273000A16894F87A2001EBC2014978C4
:10C7800080B289B2884205D0132211212000FFF720
:10C79000A9FF36E095F8018018F07F0851208DF848
:10C7A0000000684680F8018087704046C0B20128CA
:10C7B00004D021D3032815D00AD31DE003226946F3
:10C7C0002000FFF779FF01210120FCF75DFF18E051
:10C7D000032269462000FFF76FFF02210120FCF7CA
:10C7E00053FF0EE0032269462000FFF765FF032197
:10C7F0000120FCF749FF04E0122211212000FFF77D
:10C8000071FFBDE8F38100220260416001220272E3
:10C8100000224272704770B504000D001600B4F893
:10C820008C1804F6A800FFF7EEFF94F878000128B2
:10C8300006D0320092B2290014F11800FAF78DFDEB
:10C8400070BDFEB504000D001600082100226F46E1
:10C850003800FAF735FB3000C0B2782805D0B4F8BC
:10C860008C1804F6A800FFF7CEFF94F87900002892
:10C8700014D03000C0B211280FD03000C0B212283E
:10C880000BD03000C0B2312807D03000C0B27E28B3
:10C8900003D03000C0B27F2800D10CE07F208DF89B
:10C8A00000008DF801508DF802600322694614F1F2
:10C8B0001800FAF752FDF7BDFEB504000D00160092
:10C8C000082100226F463800FAF7FAFA3000A16812
:10C8D00094F87A2001EBC201497880B289B288428B
:10C8E00005D2132285212000FFF7ABFF2EE06078F0
:10C8F000012805D1222285212000FFF7A2FF25E093
:10C900006F7817F07F07C5208DF800008DF8017053
:10C910003800C0B2012802D0022809D011E001205D
:10C92000FEF7C0FC022269462000FFF774FF0DE00D
:10C930000020FEF7B7FC022269462000FFF76BFFDC
:10C9400004E0122285212000FFF77BFFF7BD0000E5
:10C95000002202604160012202720022427270478E
:10C9600070B504000D001600B4F88C1804F6A80089
:10C97000FFF7EEFF94F87800012806D0320092B25B
:10C98000290014F11800FAF7E8FC70BDFEB50400A8
:10C990000D001600082100226F463800FAF790FAC1
:10C9A0003000C0B2782805D0B4F88C1804F6A8007E
:10C9B000FFF7CEFF94F87900002814D03000C0B201
:10C9C00011280FD03000C0B212280BD03000C0B2F6
:10C9D000312807D03000C0B27E2803D03000C0B26A
:10C9E0007F2800D10CE07F208DF800008DF80150E9
:10C9F0008DF802600322694614F11800FAF7ADFCC5
:10CA0000F7BD2DE9FC4104000D00160000270821A8
:10CA10000022E8464046FAF753FA3000A16894F83D
:10CA20007A2001EBC201497880B289B2884205D0F0
:10CA3000132214212000FFF7A9FF20E0687857EAAD
:10CA40000047A87857EA0027E878074354208DF874
:10CA5000000038000B49401A03D09D3801D02F3810
:10CA600008D13800FEF701FD012269462000FFF7DA
:10CA700077FF04E0312214212000FFF787FFBDE893
:10CA8000F381000033FFFF000022026041600122B9
:10CA9000027200224272704770B504000D00160049
:10CAA000B4F88C1804F6A800FFF7EEFF94F87800AD
:10CAB000012806D0320092B2290014F11800FAF7CA
:10CAC0004CFC70BDFEB504000D00160008210022CC
:10CAD0006F463800FAF7F4F93000C0B2782805D074
:10CAE000B4F88C1804F6A800FFF7CEFF94F879008C
:10CAF000002814D03000C0B211280FD03000C0B2CE
:10CB000012280BD03000C0B2312807D03000C0B29C
:10CB10007E2803D03000C0B27F2800D10CE07F20F7
:10CB20008DF800008DF801508DF8026003226946EF
:10CB300014F11800FAF711FCF7BDFEB504000D0062
:10CB40001600082100226F463800FAF7B9F93000C4
:10CB5000A16894F87A2001EBC201497880B289B2C9
:10CB6000884205D013223E212000FFF7ABFF16E0DC
:10CB70006F7817F07F073800C0B200280AD17E20F6
:10CB80008DF800008DF80170022269462000FFF741
:10CB900083FF04E012223E212000FFF793FFF7BD40
:10CBA0002DE9F04F264FDFF89CC02748DFF89CE0C6
:10CBB000DFF89C802749284A284B294C294D2A4ECA
:10CBC000604507D09CF8009087F800907F1C1CF10E
:10CBD000010CF5E7414508D098F800908EF80090D8
:10CBE0001EF1010E18F10108F4E7934205D05FF041
:10CBF000000982F80090521CF7E7AE4206D095F883
:10CC0000009084F800906D1C641CF6E75FF000094A
:10CC1000DFF858A0B9EB9A0F0AD2DFF854A05AF8FF
:10CC200029A0DFF850B04BF829A019F10109EFE76E
:10CC3000DFF840A0DFF840B0CBF800A0BDE8F08FEF
:10CC40000004FF1F9CB90000F0BB00005406FF1F4A
:10CC5000E8D00000E8D000000000002005360020E9
:10CC600000000000000000000000000000040000C0
:10CC7000000000000000FF1F08ED00E010020100AE
:10CC8000A7C20000110201005BC7000027020100DB
:10CC9000F5A2000028030100A3BC00003E02010031
:10CCA0003BCB000085020100B9C800002203000050
:10CCB000BFAD00002E040000AFC00000140400004F
:10CCC00003CA000019030100B7BE00002F030000D3
:10CCD000C7B00000310401007D9D00003405000054
:10CCE00005B600003602000077B8000037010000EA
:10CCF000FBC5000072B6002100220023002400259D
:10CD000000260027B846B946BA46BB46BC460A4983
:10CD10000A4A521A013A05DD00200423086019442A
:10CD2000043AFBDA064885460648804706488047AD
:10CD300062B6FBF78BF8FEE70000FF1FEFEF002065
:10CD4000F0EF002061A90000A1CB0000000001006D
:10CD5000320700000001080001000000FFFFFFFF94
:10CD600001000100DF0700000001080001000000D1
:10CD7000FFFFFFFF02000100B207000000000800F3
:10CD800000000000FFFFFFFF03000100340200006D
:10CD90000000080000000000FFFFFFFF0300011378
:10CDA00002401D010B000600070008000C001C00DB
:10CDB000180017040E000F4004033D0121503E549B
:10CDC0003F4C3C05230024002500260027002800B6
:10CDD00029002A002C002D002E002F0030003100E9
:10CDE000320033002B0034000000000046697273EB
:10CDF00074206672616D652073686F756C64206E57
:10CE00006F7420757365206D756C7469706C652026
:10CE10006672616D65207472616E736D697373699A
:10CE20006F6E2E004D756C74692D6672616D652094
:10CE3000726573706F6E736520746F6F206C6172B2
:10CE4000676520666F7220726563656976696E67D3
:10CE5000206275666665722E000000004D65737372
:10CE60006167652073697A6520746F6F206C6172E9
:10CE700067652E205365742061206C61726765724E
:10CE80002073656E64206275666665720A00000034
:10CE900041626F72742070726576696F7573206D70
:10CEA0006573736167652C207472616E736D69734D
:10CEB00073696F6E20696E2070726F67726573732D
:10CEC0002E0A00000000000000000000000000002A
:10CED0000000000000000000000000000000000052
:10CEE0000000000000000000000000000000000042
:10CEF0000000000053696E676C652D6672616D6598
:10CF0000206C656E67746820746F6F20736D616C40
:10CF10006C206F7220746F6F206C617267652E00D9
:10CF20004669727374206672616D652073686F75EF
:10CF30006C64206265203820627974657320696EA4
:10CF4000206C656E6774682E00000000357E00005E
:10CF5000217D0000597D0000A37D0000E17D0000DF
:10CF60000B7E00001F7E0000E77D0000F77D0000C3
:10CF70004EF68851CEF20001086840F47000086057
:10CF8000BFF34F8FBFF36F8F4FF00170E1EE100AC8
:10CF900070470000436F6E73656375746976652032
:10CFA0006672616D6520746F6F2073686F72742E86
:10CFB00000000000466C6F7720636F6E74726F6CB8
:10CFC000206672616D6520746F6F2073686F727474
:10CFD0002E0000000100000002000000040000001C
:10CFE00008000000100000002000000040000000C9
:10CFF0008000000000F00DF8002801D0AFF30080A1
:10D00000AFF300800020AFF30080FAF71FFF00F0BD
:10D0100002F80120704700F001B8000007463846CA
:10D0200000F002F8FBE7000080B5AFF30080024A91
:10D0300011001820ABBEFBE72600020067437075A5
:10D04000436C6F636B4672657175656E6379203DE5
:10D050002025640A0000000025303464203A205363
:10D0600042435F57445F4354524C203D2025780A89
:10D07000000000000548014603B4684680F30988B3
:10D08000AFF30080FFF774FFFFF7B4FFA5EDF5FEE7
:10D090002D2D2D2D2D494E544F20424F4F542D2DC7
:10D0A0002D2D2D0A000000004A756D7020746F2030
:10D0B0004170700A000000003031323334353637A9
:10D0C00038394142434445465465726D696E616C1E
:10D0D0000000000053454747455200000102030489
:08D0E0004D535751FFF7FEBF4D
:040000050000D075B2
:00000001FF
